:020000040800F2
:1000000000000110D95A0708F92200083D30020803
:10001000795B0708795B0708795B07080000000037
:1000200000000000000000000000000091450008F2
:10003000954500080000000099450008FDCF000824
:10004000795B0708795B0708795B0708795B070824
:10005000795B0708795B070865A4000869A40008B4
:10006000795B07086DA4000871A400080126000848
:1000700015260008292600083D26000851260008FC
:100080006526000879260008795B0708795B070870
:10009000795B0708795B0708795B070875A4000896
:1000A000AD240008D5240008FD2400089924000888
:1000B00025250008392500084D250008795B07082B
:1000C000795B0708795B0708795B0708795B0708A4
:1000D000795B0708795B0708FD22000809230008FF
:1000E00079A40008795B07089D4500088925000868
:1000F000B1250008D9250008752500088D260008BF
:10010000795B0708795B070861250008795B0708B8
:100110001523000821230008795B0708795B07088D
:10012000A1260008B5260008C9260008DD2600081B
:10013000F1260008795B0708795B0708795B0708F7
:10014000795B0708795B0708795B0708E9450008D0
:1001500005270008192700082D2700082D2300086F
:10016000795B0708795B0708795B0708795B070803
:10017000795B0708795B0708795B0708795B0708F3
:08018000795B0708795B0708B1
:1001C000D0E907239A423CBFC1685218D01A704741
:1001D000D0E9092300699A4238BF1218D31A0138AE
:1001E000C01A7047D0E90902101AB0FA80F040092D
:1001F000704700BF0246036A4069D168C05C0133A2
:100200008B4228BF00231362704700BF436A826994
:10021000D154436A0169426B01338B4228BF0023EA
:100220004362D36843F08003D3607047436B188800
:1002300010F0100002D01A889B880120704700BF80
:10024000436B99891A88890610B504460AD592B27B
:10025000900607D5E26A002A2AD09888216B80B2DE
:100260009047636B99891A88090692B210D51006D7
:100270000ED5D4E909128A4215D0A1692069895C9A
:100280000132C9B29980B2FBF0F100FB1122A262E7
:10029000998A1A88C90592B204D5D20744BF4FF68D
:1002A000F7721A8010BDDA6822F08002DA60EFE798
:1002B0009B88E2696169DBB28B54E269E168636B38
:1002C0000132B2FBF1F001FB1022E261CAE700BF8C
:1002D000036942681F2B10B40AD95468A3F1200C9B
:1002E000202101FA0CF1214207D15DF8044B70473F
:1002F0001468202199402142F7D081690024C86800
:100300000C7480684C68016821F00101016020686C
:1003100094F805C00C4C818934F81C4089B221EA5C
:1003200004011F2B818107D9A3F1200120238B40D9
:100330005DF8044BD3607047202101FA03F35DF8A8
:10034000044B9360704700BF9062070882B0092297
:10035000274B8DF80720DA68D00319D4DA68D10664
:1003600040D4DA68D20541D4DA6812F0E00F3BD10C
:10037000DB6813F0020F0CBF092308238DF8073048
:100380009DF80730012B0AD09DF8070002B0704796
:1003900001238DF807309DF80730012BF4D1144A62
:1003A00012E0D368DB0519D4D36813F0E00F17D13E
:1003B000D36813F0020F0CBF092308238DF8073010
:1003C0009DF80730012BDFD1D168C8034FF001033E
:1003D000F4D4D368D906E4D50623EFE70223EDE78A
:1003E0000723EBE70623D4E70723D2E70223D0E76E
:1003F000003C0240704700BF704700BF01207047BB
:10040000034BD3E90003C01AC0F30A00704700BFD2
:10041000D81F0020054AD2E900139942FDD0D11817
:100420000133C3F30A03087A53607047D81F0020D2
:10043000064BD3F8080800B97047D3F80808A0F1B4
:100440000500B0FA80F04009704700BFD81F0020B7
:10045000012380F849307047044BD3E90003C01AE8
:10046000C0F30A00C0F50060704700BFD81F00202D
:1004700010B5D0F8E83504461B699847032384F883
:100480001231002010BD00BF08B5042290F81211EF
:10049000D0F8E83580F8131180F81221DB6898470E
:1004A000002008BD08B5D0F8E435DB6903B19847F2
:1004B000002008BD08B5D0F8E4351B6A9847002035
:1004C00008BD00BF08B5D0F8E4355B6A9847002046
:1004D00008BD00BF70B5037805460E461446DBB173
:1004E000013074F00DFA431CDBB201335B00DAB269
:1004F00023800323327073702C7864B12846022362
:1005000000215A1CD2B2F454B15410F8014F0233F6
:10051000DBB2002CF5D170BD02221346E8E700BF24
:1005200010B5074C2068FF2808D00649D1F80C28E0
:1005300001F5016100F080F8FF232360002010BD69
:1005400000000020D81F0020432301480B80704783
:1005500004000020122301480B807047480000204F
:10056000042301480B8070475C00002010B5044C48
:1005700004480A462146FFF7ADFF204610BD00BFE4
:10058000F02700202417080810B5044C04480A4638
:100590002146FFF79FFF204610BD00BFF027002037
:1005A0003017080810B5044C04480A462146FFF7E6
:1005B00091FF204610BD00BFF02700203817080823
:1005C00010B5044C04480A462146FFF783FF204635
:1005D00010BD00BFF02700204417080810B5044CD8
:1005E00004480A462146FFF775FF204610BD00BFAC
:1005F000F027002050170808704700BF704700BF61
:10060000704700BF704700BF704700BF704700BF12
:10061000044B00200522C3F80828C3F81809C3F8C2
:100620001C097047D81F0020024B0020C3F808089F
:10063000704700BFD81F0020212838B50C4625D0B0
:10064000222816D0202812D189B1072A0FD1174DA0
:10065000D5F81C3913B10968002098472168A28891
:10066000A379C5F82019A5F8242985F82639002092
:1006700038BD0029FBD0022AF9D10C4BD3F8183928
:10068000002BF4D0098800209847F0E70029EED02D
:10069000072AECD1054BD3F82019B3F8242993F895
:1006A00026392160A280A371E1E700BFD81F002096
:1006B00010B4114CD4E900329A1AC2F30A020A4467
:1006C000B2F5006F13D871B101444A1E013810F819
:1006D00001CFE118904203F1010381F808C0C3F390
:1006E0000A03F4D1236000205DF8044B7047022018
:1006F0005DF8044B704700BFD81F002010B5812162
:1007000004466AF0E5FA204601216AF0E1FA204643
:1007100082216AF0DDFAFFF787FF002010BD00BFDD
:10072000034610B4D9691A69002040F20114A3F8F5
:1007300044410860D1699C6D21F002014FF0010C29
:10074000D161A3F89CC32060D369044923F400332A
:1007500081F827095DF8044BD3617047D81F00204A
:10076000202301480B8070476000002012230148BD
:100770000B80704780000020042301480B807047E5
:10078000940000200A4608B5054920B90548FFF73E
:10079000A1FE034808BD0448FFF79CFE004808BDC1
:1007A00000290020601708087817080810B5044CC5
:1007B00004480A462146FFF78DFE204610BD00BFC3
:1007C00000290020901708081C48D0F8E837D0F816
:1007D000EC2710B59B184FF01A040C8001D1184873
:1007E00010BD174AD0F8EA0702F1100411464FF085
:1007F000000E4FEA137CB3F1204F34BF0CF1300CE4
:100800000CF1370C81F802C081F803E002318C4210
:100810004FEA0313EDD102F108040021030FB0F1F8
:10082000204F34BF303337339374D1740232944243
:100830004FEA0010F2D1024810BD00BF00F0FF1FC8
:100840009800002010B5044C04480A462146FFF7E2
:1008500041FE204610BD00BF00290020A417080853
:1008600010B5044C04480A462146FFF733FE2046E3
:1008700010BD00BF00290020B0170808034BD3F8B3
:10088000B42BB3F8B83B138300207047D81F002067
:100890004FF40070034B1060D3F8F03D0B60002064
:1008A000704700BFD81F002000207047012070470C
:1008B000012070470020704710B41C6994420CD38B
:1008C00094460A4661448C42996938BFA4EB0C02F5
:1008D00061445DF8044B70F043BB5DF8044B704716
:1008E000704700BF704700BFD0ED007AD0ED036ABB
:1008F00030EE677AE6EE877AB0EE670AC0ED007AEE
:10090000704700BF90ED017AB5EE407AF1EE10FA33
:10091000F0EE407A09D19FED0D7A60EE870AF7EE8E
:10092000006A86EEA07A80ED017A31EE077A90EDCA
:10093000000A80ED021AC1EE076A77EEC07AC0EDB8
:10094000036AA6EEA70A80ED000A7047DB0FC940D4
:1009500090ED017AD0ED036AD0ED027A30EE470ACD
:10096000A6EE807A90ED000A80ED017A37EE676A94
:10097000E6EE867A37EEC07AC0ED027AA6EE870AF6
:1009800080ED000A704700BFD0ED056AD0ED017A16
:1009900090ED066AD0ED025A90ED035AC0ED066A5A
:1009A000B0EE407A26EEA70AD0ED007A80ED057A07
:1009B000A7EE870AD0ED077AA5EE860A90ED086AC1
:1009C000D0ED045AC0ED087AA5EE670AA5EEC60A76
:1009D00080ED070A704700BFF0EE406AD0ED007A64
:1009E00090ED050A90ED037A90ED016AD0ED025A80
:1009F000A7EEA60AD0ED047A27EE407A67EEC07A19
:100A0000A6EE267AE5EEA67A90ED066AC0ED067AA5
:100A100036EE076A80ED056A704700BF03685A1C0E
:100A200002601970704700BF03685A1C0260197099
:100A3000704700BF024BD3F8200E03681B681847AD
:100A4000D81F0020007970470079C0F3401070472C
:100A500000794009704700BF90F83C20034602F03F
:100A6000FF0012B1002283F83C2070472DE9F843C3
:100A700045697DB90768C7F30D0804460E46B8F10D
:100A8000000F0AD0D6F80080FFF760FC09283BD0A1
:100A90006FF001052846BDE8F883514B9F422AD3E9
:100AA00003F580439F4224D303F580439F427FD3C5
:100AB0004C4B9F427FD903F580339F427ED903F58B
:100AC00000339F427DD903F500339F427CD903F563
:100AD00000339F4269D903F500339F4277D903F56C
:100AE00080239F4276D9B7F1016F76D305200DF0B0
:100AF00059F94FF00808FFF729FC092821D04FF0D9
:100B0000FF352846BDE8F883374E336923F4407338
:100B10003361336943F400733361336943F0010394
:100B20003361C7F80080FFF711FC3369092823F00F
:100B300001033361ACD12368043323602846BDE848
:100B4000F883DFF8A490D9F8103023F44073C9F883
:100B50001030D9F8103043F40073C9F81030D9F8C8
:100B6000103023F0F803C9F81030D9F8103043EAF8
:100B7000080343F00203C9F81030D9F8103043F4E9
:100B80008033C9F81030FFF7E1FBD9F8103023F0BB
:100B90000203C9F81030D9F81030092823F0F803FF
:100BA000C9F810303FF46EAFA9E74FF03808A2E75C
:100BB0004FF010089FE74FF018089CE74FF020080F
:100BC00099E74FF0280896E74FF0300893E74FF089
:100BD000400890E74FF048088DE74FF058088AE743
:100BE00000400008FFFF0008003C02402DE9F041F2
:100BF0000446D0E90030134483421DD80D4601EB72
:100C00000208B2B104F10C07002601E0A84510D09B
:100C100023695A1C2261234415F8011B1973042A05
:100C2000F4D139462046FFF721FFA845C4E9046006
:100C3000EED16069BDE8F0814FF0FF30FAE700BF08
:100C40002DE9F0411F4E80460B4696F8242E002ACF
:100C5000FBD19BB343445F1E08F1FF38D6F8283E12
:100C6000D6F82C2E0133C3F30A039A4216D10CF0A6
:100C700011FA04460D460CF00DFA001B61EB05015C
:100C8000B0F57A7F71F10001F5D3D6F8283ED6F899
:100C90002C2E0133C3F30A039342E8D0D6F8282E52
:100CA000D6F8283E18F8011F32440133C3F30A0373
:100CB000B84582F8301EC6F8283ECFD10020BDE8E6
:100CC000F08100BFD81F00200A4B10B5D3F80848A8
:100CD00004B910BDD3F80838052BFAD1064C002A08
:100CE0000846D4F838351146F3DDFFF7A9FFD4F8EC
:100CF000383510BDD81F0020D030002090F8482093
:100D0000531C0244DBB280F8483082F8341090F86B
:100D100049204AB1132B06D9002280F848200C4AFA
:100D2000D2F8081829B9704780F84820002BF6D16E
:100D30007047D2F80828052AF5D110B5054C194698
:100D40003430D4F83835FFF77BFFD4F8383510BD90
:100D5000D81F0020D030002090F848100023A0F8C1
:100D6000483001B97047094BD3F80828002AF9D058
:100D7000D3F80838052BF5D110B5054C3430D4F82C
:100D80003835FFF75DFFD4F8383510BDD81F002087
:100D9000D03000202DE9F047564E1F4606EB800369
:100DA0009C68002C00F0A28004F13E03A36104F5CE
:100DB0009F73E3614FF48073C4E9043328362368DA
:100DC00066600546E16094F83D00A363914609F032
:100DD000D9FB804694F8440294F83CA0261D0028D4
:100DE00053D194F8450250BBD4F840326BBB3B075B
:100DF00031D419F0020F5FD119F0010F48D1D4F8A6
:100E0000483294F9471294F847221B010029DBB2BB
:100E10000DDB3949881880F800335009012302F0AE
:100E20001F02934041F820303046BDE8F087334937
:100E300002F00F02114430460B76BDE8F08767F0F0
:100E4000ABFAD4F84032002BD1D02D4A116B0B43B2
:100E500013633B07CDD50135EDB207F01003B8F1B0
:100E6000000FCCD040F2067288F80850A8F806208F
:100E700094F84622002B34D117F0200F0CBF3221FA
:100E80001221404609F0C4FBB9E767F085FAA8E7EC
:100E9000504609F077FB6A1CD2B20028AFD002722C
:100EA00040F20662012DC28094F846220CBF322126
:100EB000022109F0ADFBA2E76B1CDBB2B8F1000F19
:100EC0009AD088F8083040F20653A8F8063094F813
:100ED00046224046022109F09BFB19F0010F8ED0FB
:100EE000D6E70221404609F093FB88E726463046C4
:100EF000BDE8F0879062070800E100E0FCEC00E04C
:100F0000003802402DE9F047038A8489A4B21C40CE
:100F100082B047D0814688464FF0004501F14C072A
:100F200001F13406B4FA84F325FA03F2D24391B204
:100F3000A9F8101014401B3BB8F1000F5FD0042B30
:100F40002ED8DFE803F052483D320300D8F80C30C9
:100F5000D9F82CA033B19B6823B11FFA8AF108F1AC
:100F600004009847D8F8243033B19B6823B11FFAA6
:100F70008AF108F11C009847D8F83C3033B19B68DF
:100F800023B11FFA8AF108F134009847D8F8543099
:100F900033B19B6823B11FFA8AF108F14C009847DE
:100FA000002CBFD102B0BDE8F087D8F80C30D9F8DA
:100FB00034105B6808F104009847002CB2D1F1E7C7
:100FC000D8F82430D9F838105B6808F11C0098472D
:100FD000002CA7D1E6E7D8F83C30D9F83C105B6884
:100FE00030469847002C9DD1DCE7D8F85430D9F82A
:100FF00040105B6838469847002C93D1D2E7042B09
:1010000007D8DFE803F01903140F0A00D9F83C30C1
:101010000193019B002C85D1C4E7D9F82C300193B2
:10102000019BF7E7D9F834300193019BF2E7D9F837
:1010300038300193019BEDE7D9F840300193019BD3
:10104000E8E700BFF8B5264C94F8242E012A0346A1
:1010500003D0022A09D00020F8BD224ED6F83C5514
:101060008DB984F8245E0020F8BD002540F20112FD
:10107000C0E95455C0E95655A0F8442100F5A271C5
:1010800069F022FFEDE7402D20D94027D4F82C1E2F
:10109000154AC3F858710A44C3E9542240F20112B8
:1010A000A3F844210022C3F85C2103F5A27118467D
:1010B00069F00AFFD4F82C3E3B44ED1BC3F30A034E
:1010C000C4F82C3EC6F83C550020F8BDAAB2402A10
:1010D00001D02F46DAE7022284F8242ED5E700BF9C
:1010E000D81F0020D0300020082E002001EB810105
:1010F00038B500EBC1010F4DB1F88C1304462846FA
:10110000FFF7D6FAE378C4F8A853012083424FF0E2
:1011100000024FF04001C4E9EC12A4F89C0304F56E
:101120006771204608BFC4F8AC5369F0CDFE0020BB
:1011300038BD00BF10360020F8B52A4CD4F88035F1
:101140000F2B04D05A1CC4F880250020F8BD264D72
:1011500095F8243E0022C4F88025002BF5D1D5F85F
:101160002C2ED5F8283E9A42EFD0D5F82C2ED5F863
:10117000283E9A422DD8D5F8286ED5F82C3EF61A7E
:10118000402E2BD8B3B2402B13BF37464027022343
:101190000123D5F82C2E85F8243E144BC0F8587145
:1011A0001344C0E9543340F20113A0F84431002342
:1011B000C0F85C3100F5A27169F086FED5F82C3ECE
:1011C0003B44F61BC3F30A03C5F82C3EC4F83C6548
:1011D000BBE7D5F82C6EC6F50066D1E701234027A2
:1011E000D7E700BFD0300020D81F0020082E0020F5
:1011F00010B5324B93F8902593F8A4C5D3F88C35ED
:10120000044613B152EA0C0231D00123E06984F89C
:10121000463140F20112A4F8442102682849002A0C
:10122000A8BFC2F380739B0301EA124143F020037D
:101230000B4363F31F42BCF1020F026000D010BDEC
:10124000E278204BC4F8A8331F200021C4E9EC0148
:10125000012A4FF00101A4F89C1308BFC4F8AC3375
:1012600004F567712046BDE8104069F02DBE0121EC
:1012700069F0F4FC0122E06984F8462140F2011390
:10128000A4F84431016800290A460CDBC1F38073DD
:101290000B4C9B0343F0200304EA11410B4363F31F
:1012A0001F42026010BD064B03EA114343F4804322
:1012B00043F0200363F31F42026010BDD0300020D2
:1012C000DFBFFFFF543600202DE9F041B0F8CC1508
:1012D000D0F8CE35B0F8D255B0F8D085C0F840512E
:1012E000012284B080F8112101F01F02012A044676
:1012F00000F2CC56ADF80810C1F3072ECDF80A3035
:10130000ADF80E504FEA134C51D0022A7746C9B2BD
:101310009BB210D0002A55D1BEF1090F4BD8DFE89F
:101320001EF08900AD004A00C8004A005C01DF00E1
:101330004A001301330101F0600120295FFA8CF2A9
:1013400072D0012F00F0B881032F00F0A181AFBB54
:1013500090F81231022B00F0E381032B2BD11CF00B
:10136000800F40F0E98102EB820200EBC20393F8A8
:101370007623003A18BF0122C24D02234FF4807138
:10138000C4E94E3384F81131C4F83031A4F81C118B
:1013900005F2B4530021C4F83411C4E94A3304F50A
:1013A0008E712046C5F8B42569F02CFD06E090F852
:1013B0001231032B0ED0204669F018FC002004B037
:1013C000BDE8F08101F0800169F048FC002004B024
:1013D000BDE8F0815FFA8CFCBCF1010FEBD8D0F8CE
:1013E000E43502A99B689847BDF80E30002BE5D183
:1013F000C4E94A33C4E94C3304214FF4807284F8C1
:101400001111A4F81C2104F58E71204669F0FAFC34
:10141000636D9D4A1A61E278012ACFD15E614FF077
:10142000802219681A60C9E7D0F8E43502A99B68E0
:101430009847C3E790F81231023B012BBBD8914B80
:10144000D0F818210021C3F8AC1512B10222C3F85C
:10145000AC258E4A02234FF480700021C4E94C3140
:10146000A4F81C01C4E94E33C4E94A2284F81131BE
:1014700004F58E71204669F0C5FC9FE790F81221B3
:10148000023A012A97D8012B98D1D0F8E4350025EB
:101490009B68C0F8185102A9984704224FF4807342
:1014A000C4E94A55C4E94C5584F81121A4F81C310B
:1014B000A9E7012B00F03B81022B7FF47FAF5FFA9D
:1014C0008CF3002B7FF47AAF03694FEA1C22023AB7
:1014D0005B68032A00F2BD81DFE802F0B6CED2D00D
:1014E0001E0A022EADF8065000F08A81032E00F08D
:1014F0004E81012E7FF45FAFD0F8EC3580781B6809
:101500000DF106019847BDF80630002B3FF456AFA9
:10151000BDF80E20002A3FF451AF934228BF134676
:101520004FF480720221A4F81C210022C4E94A0071
:1015300084F81111C4E94E33C4E94C3204F58E71BC
:10154000204669F05FFC39E7012D7FF434AF90F855
:101550001231022B00F00881032B7FF42CAF4FF4E3
:10156000807200F588730221A0F81C21002280F807
:101570001111C0E94E55C0E94A33C0E94C5200F59B
:101580008E7169F03FFC19E7DDB23E4F012D87F8FF
:10159000A5553FF610AF90F81231022B00F0D8801D
:1015A000032B7FF408AF002D00F0358190F8101167
:1015B000012910D0D0F8E4355B68984797F8A51555
:1015C000D4F8E43584F810111B6820469847D4F805
:1015D000E8359B68984700230AE758EA05027FF43C
:1015E000EAAE90F8121103293FF4E5AE03F07F054F
:1015F00080F814510069114663F30A110368194316
:101600000423016084F811314FF48073C4E94A2245
:10161000C4E94C22A4F81C3104F58E71204669F00F
:10162000F1FB636D184A1A61E278012A06D0002D99
:1016300000F0FC80022384F81231BFE65E614FF0B7
:10164000802219681A60F2E702210E4861F306133E
:101650000022C0F8B0350423C4E94A22C4E94C2270
:1016600084F8113101224FF4807304F58E7184F8EF
:101670001621A4F81C31C8E60321E6E70521E4E7BA
:101680000421E2E7D0300020180008607C360020FA
:1016900090F81211022943D003297FF48CAE23B9AC
:1016A000510602D0114669F0D9FAD4F8E4359B68A6
:1016B00002A9204698478EE790F8121102292FD0F0
:1016C00003297FF478AE002B7FF478AE12F07F010F
:1016D00081D01CF0800F40F0AD8002EB820100EB66
:1016E000C10181F8763381F87533282381F874239A
:1016F00003FB020300EB820193F87723496D0B682B
:10170000023A012A23F400138CBFC3F300720122B2
:1017100062F31C73D4F8E4250B60936802A9C8E750
:1017200053063FF44BAE114669F098FA46E6D0F8FE
:10173000E425C0F81831F0E702F07F0202EB8202E4
:1017400000EBC20393F81E21003A18BF012213E6F2
:10175000002D3FF4A2AE01210322D0F8E43580F839
:10176000101180F812212FE73B4A80F811314FF415
:1017700080710023A0F81C11C0E94E55C0E94A222F
:10178000C0E94C5300F58E7169F03CFB16E6DBB204
:10179000052B3FF610AEDFE803F02B231B130B03E2
:1017A000D0F8EC3580789B690DF106019847AAE6E0
:1017B000D0F8EC3580785B690DF106019847A2E618
:1017C000D0F8EC3580781B690DF1060198479AE650
:1017D000D0F8EC358078DB680DF10601984792E689
:1017E000D0F8EC3580789B680DF1060198478AE6C1
:1017F000D0F8EC3580785B680DF10601984782E6F9
:10180000D0F8E43580789B6A0DF106019847467060
:10181000C4F8F00577E60222D0F8E43580F812210A
:1018200080F810515B682946984736E6012384F812
:101830001231C3E5282202FB010080F81C1104EBE1
:10184000810180F81E3180F81DE190F81F2189691F
:1018500055E70121F9E600BF7836002010B50446AF
:1018600029B990F81121032A0DD0002010BDD0F81D
:10187000E4359B69002BF8D090F81221032AF4D1AB
:101880009847002010BDD0F890230B46D0F87C1369
:101890008A4219D9521AC0F8902394F803C0D0F89C
:1018A00080038A4228BF0A46BCF1010F92B234D0AD
:1018B000C4E9E22304F55D71C4F88003A4F874332D
:1018C000204669F09FFAD0E7D0F8E4351B691BB1D8
:1018D00090F81221032A1ED000234FF480720421B5
:1018E000C4E94A33C4E94C3384F81111A4F81C212B
:1018F00004F58E71204669F085FA636D0D4A1A6110
:10190000E278012AB1D104F2CC545C614FF080221C
:1019100019681A60A9E79847DEE70844C4E9E2239A
:1019200004F55D71C4F88003A4F87433C4F884032B
:10193000C6E700BF1800086038B5044649B990F8FA
:101940001131022B11D094F81631012B39D000201F
:1019500038BDD0F8E4355B69002BF8D090F812213F
:10196000032AF4D19847002038BDD0F83831D0F898
:10197000242193422FD990F803C09B1ABCF1010F88
:101980000D46C0F83831D0F828116ED09BB2C0F89F
:1019900030314FF48073C0E94A11C0F8345100F57A
:1019A0008E71A0F81C3169F02DFAC4E9E255C4F833
:1019B000805304F55D71A4F87453204669F022FA4F
:1019C000C1E73F4B2269D3F8B0155160002384F87A
:1019D0001631002038BDD0F83C31B3FBF2F502FBE4
:1019E00015350DBB9A421FD8D0F8402193421BD227
:1019F0004FF48073A0F81C3100F58E71C0E94A5590
:101A0000C0E94C5569F0FEF9E378C4F84051012B68
:101A1000C4E9E255C4F88053A4F8745308BFC4F86D
:101A2000845304F55D71C8E7D4F8E435DB681BB175
:101A300094F81221032A15D0E27800230521012A07
:101A400084F81111C4E9E233C4F88033A4F8743384
:101A500004F55D7124D0204669F0D4F9636D194A0C
:101A60001A6170E720469847E6E79BB21144C0F838
:101A700030314FF48073C0E94A11C0F8345100F599
:101A80008E71A0F81C3169F0BDF9C4E9E255C4F8C3
:101A9000805304F55D71A4F87453C4F884538CE743
:101AA000C4F88433204669F0ADF9636D05481861C8
:101AB00004F2CC525A614FF080211A68196042E753
:101AC000D03000201800086070B50B7813F0600269
:101AD0000D46044624D0202A04D0204669F086F81A
:101AE000022070BDCA8848781AB31B0640D5324E12
:101AF0003146FEF7A1FDEB884FF480720221A4F875
:101B00001C21002284F81111C4E94E33C4E94A664D
:101B1000C4E94C3204F58E71204669F073F906E091
:101B20004B780A2B10D00B2B08D0062BD5D00020D9
:101B300070BD02221144FEF77FFDF8E78B78C3BB2E
:101B40001E4AC2F8B835F2E7022180F811114FF4AD
:101B50008071A0F81C111A490123C0E94A11C0E99B
:101B60004E33C0E94C3200F58E7169F04BF9DEE777
:101B70001449154B0860E078C3F80C28002103F5E0
:101B8000016301284FF00305C4F88C13A4F8741303
:101B9000C4E9E42284F81151C4F88823C4F88033DE
:101BA00004F55D7108BFC4F88433204669F02AF952
:101BB000BDE769F01BF8BAE7E8270020D030002025
:101BC0008836002000000020D81F0020002310B518
:101BD00019460446402269F0ABF8802120460023D4
:101BE000402269F0A5F8D4F8E835A078012284F8FD
:101BF00012215B689847002010BD00BF10B502237A
:101C000004464022812169F093F8204602234022B5
:101C1000012169F08DF8204603230822822169F012
:101C200087F8104B0222A3F84C20FEF7F1FCE27873
:101C30000D4BC4F8A8334021C4F8B013012A4FF06B
:101C400000004FF00101C4F8B403A4F89C1320462F
:101C500004F5677108BFC4F8AC3369F035F90020AA
:101C600010BD00BF000000201036002030B58121DB
:101C700083B0044669F02CF80121204669F028F869
:101C80002A4900250223402281F827592046812134
:101C900069F04EF8012102234022204669F048F8FD
:101CA000234BD3F8BC2583F8A455126828469047E7
:101CB0000095009AE1681F4B42F010020092009AD2
:101CC0000A610A690092013B02D0009AD006F8D45A
:101CD00000230193019B43F020030193019A154BCC
:101CE000012060F38A120192019A0A610A69019245
:101CF000013B02D0019A9206F8D4E2780E4BC4F868
:101D0000A8331F200021C4E9EC01012A4FF0010192
:101D1000A4F89C13204604F5677108BFC4F8AC33DF
:101D200069F0D2F8002003B030BD00BFD81F0020FA
:101D3000D0300020410D0300543600202DE9F84337
:101D4000DDF820800F4615460021202204461E465D
:101D500070F01EFDB8F1000F0CD0D8F80030E38110
:101D60001B0C2382D8F80430B8F80A20E3821B0C3D
:101D700062822383384672F0C3FDEB0619D4431EFA
:101D8000B8B107EB000C01E0013B12D31CF801EDE8
:101D9000BEF12E0FF8D1C01A421E032AA8BF03229B
:101DA000082B03F10109A8BF08239046B9441A463D
:101DB00006E008280246B946A8BF08224FF00008EE
:101DC0004FF0203339462360636020466FF0C8F837
:101DD00004F10800154B23814246494683706FF099
:101DE000BFF8611EE21D11F801CFACF16103192BA0
:101DF0009CBFACF1200C81F800C09142F3D104F1FA
:101E00000A0011F8013FA3F16102192A9CBF203B8F
:101E10000B708142F5D118232373330CA382E57232
:101E2000099B6683E361BDE8F88300BF20202000A2
:101E30002DE9F04FDFF858B4DBF8B40B0C46BBF8D3
:101E4000B81B418385B0002B63D01344174604F5BB
:101E5000FE7A99461FE0002F69D0DBF8FC3DBB42BB
:101E600000F0CB80DBF8F83DBB4200F0FD80DBF8F2
:101E7000003EDBF8041EBB4250D8B94200F2758127
:101E8000791A204666F084F901374F4504F500744D
:101E90000AF5007A39D0DBF8083EBB42DBD8DBF824
:101EA000185EFB1A296BDA0802328A4203F0070631
:101EB00002D3AB6B9A420BD929461046029266F0C8
:101EC00037F9029A0546002800F06F81CBF8180E0A
:101ED0002B79002B40F02381D5F82880B8F1000F32
:101EE00000F05C812B6BD21AEB6806EBC20203EBAD
:101EF000422220462B464FF400710137C0474F4520
:101F000004F500740AF5007AC5D1DBF8B40BBBF810
:101F1000B81B0183002005B0BDE8F08FB942AFD9EE
:101F20004FF400720021204670F032FCACE74FF411
:101F300000723946204670F02BFC802384F8BE31B5
:101F40000C2384F8C231DBF8F81DC54ADBF8F03DFC
:101F5000C4F8C6119142C4F8CA3100F30B81C14ADA
:101F6000C14D82FB010285FB01050A44C817C0EB85
:101F70006212C0EB2530BD4D84F8C10185FB0265BE
:101F8000C2EB82168010891B013120F03F001544FE
:101F90000843D117C1EBE5110A4484F8BF21B04AC8
:101FA00084F8C001013B934200F3F080AD4AAE4893
:101FB00082FB031280FB03101A44D917C1EB621293
:101FC000C1EB2031A94884F8C51180FB0250C2EB57
:101FD000821589105B1B013321F03F011044194326
:101FE000D317C3EBE0131A4484F8C41184F8C32157
:101FF0004AF65523A4F8FE3146E74FF0FF3384F844
:10200000EC3184F8ED3184F8EE3184F8EF3152236D
:10201000237063706123A37084F8E7314123E37078
:1020200084F8E6317223002584F8E43184F8E53140
:10203000DBF8103EC4F8E8314FF4F0722946201D59
:1020400070F0A6FB552384F8FE316FF05503C4F8F9
:10205000F051C4F8F451C4F8F85184F8FC5184F8F4
:10206000FD5184F8FF310FE74FF400720021204644
:1020700070F08EFB7E4B03CB45F6EB032380902361
:10208000C4F80710A37002220821F823C4F8030043
:10209000617322746375DBF8F03D2273A27384F8D8
:1020A0002C20DBF8F82D9B1A2362DBF8002EDBF8DE
:1020B000043E9B1A63620023E372E3736377A377A2
:1020C000E37784F82D3084F82E3084F82F3084F8AC
:1020D0003130684BA361684BC4F842303E2323770C
:1020E000012384F83030654A802384F8403084F836
:1020F00046104AF65521A4F8FE1103CA604BC4F8F5
:102100004700C4F84B1003CB1388A4F84F309378E2
:10211000C4F85200C4F8561084F85130B4E64FF4B5
:1021200000720021204670F033FB002E44D12B6C4E
:1021300004F12008002B7BD02B6B52491122CDE9F2
:1021400000662046FFF7FAFD2B6C1A6C002A7ED041
:102150001B6B4D49CDE9006640461122FFF7EEFDAD
:1021600004F140084FF4E0736DE0F91A204666F080
:102170000FF889E6FF2284F8C1214FF6FF72A4F818
:10218000BF21374A013B93427FF710AFFF2384F80A
:10219000C5314FF6FF73A4F8C33129E741464FF428
:1021A0000072204670F0F4FA6EE6384A231F43F8B6
:1021B000042F9A45FBD167E6D5E910253301002AA3
:1021C00043D0023B002D3FF45FAE013BAD6CF9D133
:1021D000A0464FF40073002D3FF456AECDE9027ACD
:1021E00008EB0306A24608E00024CDE900C4FFF78F
:1021F000A5FDAD6CBDB1B04515D02C7929682B6B10
:10220000404605F11C0C112208F12008002CEBD1EE
:102210006A792C6942F02102CDE900C4FFF78EFDF6
:10222000AD6C002DE7D15446029FDDF80CA02BE6E3
:10223000CDE900663346DBF8F41D08222046FFF79F
:102240007DFD4FF4F0736D6CC5E7013BBAE7CDE956
:1022500000660D49334640461122FFF76FFD7FE7C8
:10226000FF03FB00832008829755454181808080D1
:10227000C01708083F00FF0029940E0DCC1708086E
:10228000D8170808901E0808341E0808DEADBEEFF7
:10229000D81F00208C46134601466246184646F079
:1022A000C3B900BF1049114BD1F8882042F4700225
:1022B00010B4C1F888201A680D4C002042F00102C9
:1022C0001A6098601A6822F0847222F480321A60D0
:1022D0005C601A68074C22F480221A60D8608C6017
:1022E0005DF8044B704700BF00ED00E0003802408D
:1022F0001030002400000008704700BF0148FDF7BF
:102300009FBF00BFB80000200148FDF799BF00BF84
:10231000040300200148FDF793BF00BF50050020D3
:102320000148FDF78DBF00BF9C0700200148FDF765
:1023300087BF00BFE8090020704700BF704700BF9B
:10234000B0B130B443688D685A791C680223934059
:102350004A689BB26AB1A2899DB192B2134381606F
:10236000A381A3899BB243F00103A38130BC7047D2
:102370007047A28992B222EA0303A38165B181600A
:10238000EFE722F001021204120CA281A2898160FF
:1023900092B21343A381E9E7A38923F001031B044D
:1023A0001B0CA3818160E1E738B5D0E9004007EE5E
:1023B000902A0068324A334B2468D3F8303C2468B2
:1023C000013990428DB210D002F5806290420CD05B
:1023D00002F57052904208D002F58062904204D01B
:1023E00002F58062904218BF5B0807EE103AF8EEE3
:1023F000677AB8EE477ADFED246A87EE270A30EE77
:10240000260A6AF033FE1E492388421E8C4292B28D
:102410009BB21AD01D498C4217D0B4F1804F1FD007
:10242000A1F580318C421BD001F580618C4217D020
:1024300001F580618C4213D015498C4219D123805B
:102440000123E5622285A38238BD23F45C739BB22D
:1024500023800023E562228523860123A38238BDE1
:1024600023F45C739BB223800123E5622285A3825F
:1024700038BD08498C42E2D023F440739BB2DEE7BA
:1024800000000140000000200AD7233C0004014066
:102490000010004000140040024B0348D3F8C01560
:1024A000FEF730BDD03000200000014010B5064CD2
:1024B0000648D4F8C015FEF725FDD4F8E015044809
:1024C000BDE81040FEF71EBDD030002000000140E6
:1024D0000040014010B5064C0648D4F8C015FEF780
:1024E00011FDD4F8E4150448BDE81040FEF70ABD1C
:1024F000D0300020000001400044014010B5064CDF
:102500000648D4F8C015FEF7FDFCD4F8E8150448D9
:10251000BDE81040FEF7F6BCD030002000000140BE
:1025200000480140034B4FF08040D3F8C415FEF73C
:10253000E9BC00BFD0300020024B0348D3F8C815D7
:10254000FEF7E0BCD030002000040040024B0348FE
:10255000D3F8CC15FEF7D6BCD030002000080040E0
:10256000024B0348D3F8D015FEF7CCBCD030002086
:10257000000C0040024B0348D3F8DC15FEF7C2BC48
:10258000D03000200004014010B5064C0648D4F8B5
:10259000DC15FEF7B7FCD4F8EC150448BDE8104094
:1025A000FEF7B0BCD030002000040140001800400D
:1025B00010B5064C0648D4F8DC15FEF7A3FCD4F899
:1025C000F0150448BDE81040FEF79CBCD030002058
:1025D00000040140001C004010B5064C0648D4F829
:1025E000DC15FEF78FFCD4F8F4150448BDE8104064
:1025F000FEF788BCD03000200004014000200040DD
:102600000348D0F8403C13B100F6344018477047F7
:10261000000000200348D0F8603C13B100F654409D
:1026200018477047000000200348D0F8803C13B1E1
:1026300000F6744018477047000000200348D0F8A7
:10264000A03C13B100F694401847704700000020EA
:102650000348D0F8C03C13B100F6B44018477047A7
:10266000000000200348D0F8E03C13B100F6D4404D
:1026700018477047000000200348D0F8003D13B110
:1026800000F6F44018477047000000200348D0F8D7
:10269000203D13B100F61450184770470000002089
:1026A0000348D0F8403D13B100F634501847704746
:1026B000000000200348D0F8603D13B100F65450EC
:1026C00018477047000000200348D0F8803D13B140
:1026D00000F6745018477047000000200348D0F8F7
:1026E000A03D13B100F69450184770470000002039
:1026F0000348D0F8C03D13B100F6B45018477047F6
:10270000000000200348D0F8E03D13B100F6D4509B
:1027100018477047000000200348D0F8003E13B16E
:1027200000F6F45018477047000000200348D0F826
:10273000203E13B100F614601847704700000020D7
:1027400002683649002310B422F001022124884295
:102750000260036043608360C3600361446138D0FA
:102760002F4B98422ED02F4B98423CD02E4B984264
:1027700040D02E4B984232D02D4B984241D02D4B19
:10278000984246D02C4B984217D02C4B98423CD0C4
:102790002B4B984216D02B4B984224D02A4B984270
:1027A00028D02A4B98421AD0294B984229D0294B3D
:1027B00098422ED0284B984208D14FF03D5243F812
:1027C000AC2C03E04FF4746243F8202C5DF8044B0A
:1027D0007047224B5DF8044B3D229A607047204AB7
:1027E00043F8642CF2E74FF474125DF8044B43F89D
:1027F000382C70474FF074625DF8044B43F8502C4E
:102800007047184A43F87C2CE0E73D2243F8082C37
:10281000DCE7154A43F8942CD8E700BF106002406B
:1028200028600240406002405860024070600240F0
:1028300088600240A0600240B8600240106402401C
:1028400028640240406402405864024070640240C0
:1028500088640240A0640240B86402400060024004
:102860003D000020400F002000003D202DE9F041F8
:102870006F4F00EB400307EBC30790B0054697F896
:10288000390E65F089FD97F8380E65F085FDD7F8AB
:102890003C8E4046FFF754FF0023D7F8344ED7F85C
:1028A000486E0493CDE90C33CDE90E330693D7F887
:1028B000403E604F01934FF48C7303FB0573039309
:1028C00006EB86039B00059304F14C034FF48062F2
:1028D00002934FF40063CDE907234FF400514FF406
:1028E0008073CDE909134FF4003301A90B9365F010
:1028F00027FDD8F800205049504B42F00102C8F89B
:1029000000204A68134043F440334B606368012E53
:1029100023F04073D4BF0022012223F4807343EAE2
:1029200002236360A268464B134043F00203A36096
:10293000E36A013EF6B223F4700343EA0653E3620E
:1029400007F5647007F55273012602E00C339842D4
:102950002DD05A7D002AF9D093F90D20AA42F5D145
:102960001A7C997D092A45D9A2F10A07D4F80CC02E
:1029700007EB47074FF0070EB9400EFA07F72CEAAE
:1029800007073943E160062E24D8711E676B01EBFF
:1029900081014FF01F0C8A400CFA01F127EA010176
:1029A0000A4362630C3301369842F6B2D1D1A36870
:1029B00043F40073A360A36843F48073A360A36827
:1029C00043F00103A360A36843F08043A36010B009
:1029D000BDE8F0810C2E1BD8F11F276B01EB8101A4
:1029E0004FF01F0C8A400CFA01F127EA01010A435B
:1029F0002263D7E7276902EB420E4FF0070C0CFA6F
:102A00000EFC01FA0EF127EA0C0739432161BAE7FF
:102A1000A6F10D01E76A01EB81014FF01F0C8A401E
:102A20000CFA01F127EA01010A43E262BAE700BFAA
:102A300000000020C836002000230140E030FCFFE9
:102A4000FDF7FFC0214A936803F00C03042B10B478
:102A50003AD0082B1FD01E4B1C4C0360A1681D4AA6
:102A6000C1F30311114491F85810CB404360A168A1
:102A7000C1F38221114491F8581023FA01F18160C9
:102A8000A1685DF8044BC1F342310A4492F8582022
:102A9000D340C36070475368516813F4800F536884
:102AA00014BF0D4A0A4AC3F3881301F03F01B2FB79
:102AB000F1F202FB03F3054A5268C2F3014201320C
:102AC0005200B3FBF2F3C7E7034BC5E700380240FF
:102AD0000024F4009062070800127A0070B5446B7D
:102AE0008668A38923F400531B041B0CA3818579FA
:102AF00090F805C02B0303F40051C5F380000CF0DF
:102B000001032A029B001CF0020F4FEA003002F47E
:102B1000806218BF43F0080302431A43238A9BB222
:102B200023F440530B432382A38923F4B05323F0AF
:102B30000C031B041B0C1343A381A38A23F44073CF
:102B40001B041B0C84B0A3826846FFF77BFF234B5A
:102B50009C4205D003F580639C4201D0029B00E0BB
:102B6000039BA2891E49120403EB83034CBF76002A
:102B7000B60003EB8303B3FBF6F3A1FB0302A089CA
:102B800052096426000406FB12334FEA02121CD4D9
:102B90001B013233A1FB0313C3F3431313439BB253
:102BA00023812A07A38A0AD59BB243F00803A38294
:102BB000A3899BB243F40053A38104B070BD23F0FA
:102BC00008031B041B0CA382F2E7DB003233A1FBDA
:102BD0000313C3F342131343E1E700BF00100140A6
:102BE0001F85EB512DE9F8431D46344B9DF82060BD
:102BF0009DF8249098428846174646D0304B98421C
:102C00004BD0304B984250D02F4B984235D02F4B61
:102C100098422ED14B46324629460520FEF7BAF897
:102C200004460023C4E90B87C4E90733C4E9093328
:102C30006671A56084F806902046FFF74FFFF10704
:102C4000626B0ED4B30707D493899BB243F400534D
:102C500093812046BDE8F883D36843F08003D360B6
:102C6000F2E74FF6DF731380D36843F02003D3609D
:102C7000E8E700242046BDE8F8834B463246294663
:102C80000420FEF787F80446CBE74B463246294638
:102C90000120FEF77FF80446C3E74B46324629463B
:102CA0000220FEF777F80446BBE74B46324629463A
:102CB0000320FEF76FF80446B3E700BF004400406E
:102CC00000480040004C004000500040001401400B
:102CD000816003E7417101E72DE9F043794F07EB8C
:102CE000C00985B005464FEAC00899F8800E07F084
:102CF00049FC044699F8810E07F044FC064699F811
:102D0000820E65F049FB6B1CDBB2002C00F0AB803F
:102D100040F60C122372E280002E00F0B68033726F
:102D200040F60C232046F38004223A2107F070FC81
:102D3000042230463A2107F06BFC07EB0803624A95
:102D4000D3F87C4E944200F09680604B9C4200F099
:102D5000A2805F4B9C4200F0A980474497F8833ED5
:102D6000022B32D0032B7CD05A495B4F012B08BF7A
:102D70000F46A6886846FFF765FE26F03F06029BD1
:102D8000564AB3FBF7F13604A2FB0323360C46EA9E
:102D90009346A680228822F001021204120C22809F
:102DA0008AB2C1F30B019B0C09B942F001024FF446
:102DB000967101FB03F34A49A1FB03139B090133FD
:102DC0009BB242F4004223841FE0A6886846FFF7C6
:102DD00039FE26F03F06029A404B3604A3FB02134D
:102DE000360C46EA9346A680218821F001010904A9
:102DF000090C21803B499209A1FB021292099B0C0C
:102E00000133042A238438BF0422A2832388364A4C
:102E10009BB243F001032380238823F4816323F0D2
:102E200002031B041B0C4FF4804143F48063238096
:102E30002181238823F080031B041B0C238023881B
:102E40009BB202EB451243F00103238001210023D2
:102E500082F8985982F8991982F89A3905B0BDE834
:102E6000F083224F85E7002E3FF467AF337240F6C0
:102E70000C23F3805CE71E4B1A6A42F400121A62BC
:102E80001A6A22F400121A6267E7042220463A21E5
:102E900007F0BEFB51E703F5F0331A6A42F48002F3
:102EA0001A621A6A22F480021A6256E703F5EE33B8
:102EB0001A6A42F400021A621A6A22F400021A62C2
:102EC0004BE700BF000000200054004000580040C5
:102ED000005C0040009F2400804F120083DE1B43F3
:102EE000D34D6210632D3E05D0300020C02709006D
:102EF000003802402DE9F047924E90F900108046CC
:102F0000807806EBC1050138CC0090B0D5F87C1E66
:102F100014282DD8DFE810F04C01200115005500D1
:102F20005F009E00A600C301B6017A0084003C0247
:102F30000402D701C000D0002F003700A301950183
:102F40005401888A0C8B81B27F4841EA044188434E
:102F500000F02081D8E90201101A42F2107263EBEE
:102F60000101904271F1000102D3152388F802306B
:102F700010B0BDE8F08798F813000882C8E9022372
:102F8000122088F80200888A0C8B80B240EA044044
:102F90006E4C844300F0B28000200E900F90012010
:102FA0000F910E900E99002900F017820F9914319D
:102FB0000F910F9909684905CCD5142388F8023080
:102FC000D6E798F8110000F0FE000882C8E9022355
:102FD000052088F80200888A0C8B80B240EA044001
:102FE0005B4C844300F0A180002000900190012000
:102FF000019100900099002900F0FB8101991431A2
:103000000191019909684F05D7D4A3E798F81100F9
:1030100040F001000882C8E902230B2088F8020072
:10302000888A0C8B80B240EA04404A4C84436DD0BD
:103030000020049005900120059104900499002936
:1030400000F0D181059914310591059909684D0564
:10305000B3D47FE798F813000882C8E90223072059
:1030600088F80200888A0C8B80B240EA0440374C12
:1030700084435ED0002002900390012003910290CF
:103080000299002900F0C181039914310391039939
:1030900009684E0591D45DE7088820F4806000043B
:1030A000000C088098F8110000F0FE000882C8E9C2
:1030B0000223102088F80200888A0C8B80B240EA34
:1030C0000440234C844312D000200C900D9001202A
:1030D0000D910C900C99002900F091810D991431FB
:1030E0000D910D99096848053FF567AF32E798F8EB
:1030F0001330FF2B06D198F810301BB1132388F83A
:10310000023035E7112388F8023031E7D8F814008F
:10311000012800F08F81022800F04382098B0E21E4
:10312000C8E9022388F8021022E7062388F8023053
:103130001EE7D8F81400002800F06D81082388F8F5
:10314000023015E7000000200100030084000700A2
:103150008200070002000300088820F400600004D9
:10316000000C0880088880B240F4806008800888DD
:1031700080B240F480700880032088F80200888ABA
:103180000C8B81B2A94841EA04418843C8E9022373
:103190007FF4EEAE98F81230002B40F0CE8198F814
:1031A0001330FF2B00F03F82042388F80230DFE663
:1031B000098889053FF5CEAE002388F80230D7E6AE
:1031C000344494F8800E07F0DDF9064694F8810E39
:1031D00007F0D8F9964AB2F8F83901339BB2824623
:1031E000A2F8F83916B13368B2881A83BAF1000F21
:1031F00004D0DAF80030BAF804201A8311213046DE
:1032000007F09CF91121504607F098F94FF0090991
:1032100065272EB13368B28819690A4240F02381CC
:10322000013F00F01D8109F035FF04460D4609F00D
:1032300031FF001B61EB0501052871F10001F6D398
:10324000E7E7088880B240F4007008804FF6FF304E
:1032500088820121C8E9022388F8021088E6D8F89C
:103260001400002800F06D81D8F8184014F8016BA4
:103270000E8201381225C8E90504C8E9022388F83E
:10328000025075E6888A0C8B81B2684841EA044195
:1032900088437FF45FAE0A2388F8023068E6088826
:1032A00080B240F480700880092088F80200888A83
:1032B0000C8B81B25D4841EA04418843C8E902238E
:1032C0007FF456AEE7E7002401250A940B940B9196
:1032D0000A950A98002800F047810B9814300B904B
:1032E0000B98006846077FF535AED8F81400032820
:1032F00000F06D81022800F24381088820F480608C
:103300000004000C0880088880B240F40070088037
:10331000098A88F81C40C8E9022388F8025027E689
:103320000020012408900990099108940898002829
:1033300000F0148109981430099009980068470733
:103340007FF508AEEFF31185102080F3128808880E
:1033500080B240F400700880D8F818000E8A471C2C
:10336000C8F81870EDB2067085F311880D8AD8F888
:1033700018106FF001004E1CC8F818600D70C8E9F5
:103380000223C8F8140088F81C4088F80240EFE5D2
:10339000002006900790012007910690069C002CC3
:1033A00000F0E880079C14340794079C24686406A6
:1033B0007FF5D0AD0C8AD8F818104D1CC8F81850FD
:1033C0000C70D8F8141088F81C000139C8E90223E1
:1033D000C8F8141088F80200CAE50F9918310F9147
:1033E0000F990968B6E5059918310591059909689D
:1033F000B0E501991831019101990968AAE50D9983
:1034000018310D910D990968A4E5039918310391BC
:10341000039909689EE5088880B240F4007008802E
:103420000121C8E9022388F80210A1E50100030088
:10343000D0300020088820F480600004000C088050
:10344000EFF31184102080F31288088B088880B273
:1034500040F40070E4B2088084F311880C215FE628
:1034600016B13368B2885A8309F014FE04460D463B
:1034700009F010FE001B61EB0501052871F1000148
:10348000F6D316B13368B2881A8309F003FE0446F6
:103490000D4609F0FFFD001B61EB0501052871F1E8
:1034A0000001F6D3B9F101097FF4B2AE16B1336869
:1034B000B2885A8309F0EEFD04460D4609F0EAFD94
:1034C000001B61EB0501052871F10001F6D3BAF18B
:1034D000000F04D0DAF80030BAF804205A8309F05B
:1034E000D9FD04460D4609F0D5FD001B61EB050131
:1034F000052871F10001F6D316B13368B2881A833A
:1035000009F0C8FD04460D4609F0C4FD001B61EB3F
:103510000501052871F10001F6D3BAF1000F04D0BE
:10352000DAF80030BAF804201A8398F90000441C35
:103530003FF442AEFFF7D0FB3EE60F2388F802309F
:1035400016E5088880B240F4007008800121C8E9BF
:10355000022388F81C1088F8021009E5099918312F
:10356000099109990968F5E40B9918310B910B99A8
:103570000968EFE407991831079107990968E9E4A8
:10358000D8F81800098A441CC8F818400170D8F807
:103590001410C8F808200139C8F81410C8F80C3005
:1035A000E6E4088880B240F400600880EFF31184FC
:1035B000102080F31288088B088820F480600004B3
:1035C000000CE4B2088084F311880D21A8E5088876
:1035D00020F480600004000C0880EFF311841020B8
:1035E00080F31288D8F818000D8A461CC8F81860B5
:1035F0000570088880B240F40070E4B2088084F35B
:103600001188D8F81800098A441CC8F818400170BD
:10361000D8F814100C200239C8E90223C8F8141095
:1036200088F80200A4E498F81030002B3FF4BCADF9
:1036300031E600BF38B5184D9DF814E005EB401495
:103640004FEA401C94F8990900B938BD84F8AB29B9
:10365000C4F8AC3901220023490005F6981584F816
:10366000AA2984F8B439049A84F8A8E9022384F8D2
:10367000A919C4F8B02984F89A39654409F00AFDFB
:1036800002460B462846FFF735FC94F89A39002B82
:10369000F4D194F8B40938BDD03000200068037923
:1036A000012B0BD0022B01D0002070478368DB0771
:1036B0004FF0F00219D5FF2105F022BA00B582685B
:1036C00090F910C0417C85B002F0010201920DF129
:1036D0000F0200926046FF224FF0F00C8DF80FC0F1
:1036E000FFF7A8FF05B05DF804FB7F2105F008BADD
:1036F00070B505682B79012B84B004460E4617D0AF
:10370000022B02D0002004B070BDAB68E122DB07C1
:103710004CBF11466121284605F0F2F90028F1D08E
:1037200020683246FF2104B0BDE8704006F09AB828
:10373000AA68697C95F9100002F001020DF10F05ED
:1037400001920095E1228DF80F20FFF773FFE5E766
:1037500070B505682B79012B84B004460E4618D04D
:10376000022B02D0002004B070BDAB68DB074FF025
:10377000C3024CBFE1216121284605F0C1F90028B0
:10378000F0D020683246FF2104B0BDE8704006F05A
:1037900069B8AA6895F91000697C02F001020192EB
:1037A0000DF10F020092C3228DF80F20E122FFF7E6
:1037B00041FFE4E700680379CA4341EA0211012BA3
:1037C000CAB209D0022B01D0002070478368DB0702
:1037D00017D5D22105F094B900B585B090F910C085
:1037E0008DF80F208268417C02F001020DF10F007C
:1037F000CDE90002D2226046FFF71CFF05B05DF85C
:1038000004FB522105F07CB970B505682B79012BBA
:1038100084B004460E461CD0022B02D0002004B017
:1038200070BDAB68DB074FF0F0024CBFE1216121B6
:10383000284605F065F90028F0D02246FF2152F80D
:10384000040B06F00FF80028E8D02379337004B099
:1038500070BDAA6895F91000697C02F0010201921E
:103860000DF10F020092F0228DF80F20E122FFF7F8
:10387000E1FEE0E700680379012B0BD0022B01D0B9
:10388000002070478368DB074FF0B40219D5FF2191
:1038900005F036B900B5826890F910C0417C85B05A
:1038A00002F0010201920DF10F0200926046FF2228
:1038B0004FF0B40C8DF80FC0FFF7BCFE05B05DF8FB
:1038C00004FB7F2105F01CB900680379012B0AD0A5
:1038D000022B01D0002070478368DB070A4617D50A
:1038E000A52105F00DB900B5826890F910C085B02A
:1038F00002F001028DF80F10417C0DF10F00CDE9AF
:103900000002A5226046FFF795FE05B05DF804FBB6
:10391000252105F0F5B800BF00680379012B0BD015
:10392000022B01D0002070478368DB074FF096021E
:1039300019D5FF2105F0E4B800B5826890F910C0F0
:10394000417C85B002F0010201920DF10F0200925C
:103950006046FF224FF0960C8DF80FC0FFF76AFE0D
:1039600005B05DF804FB7F2105F0CAB80068037953
:10397000012B0AD0022B01D0002070478368DB079F
:103980000A4617D5872105F0BBB800B5826890F9C3
:1039900010C085B002F001028DF80F10417C0DF1CE
:1039A0000F00CDE9000287226046FFF743FE05B015
:1039B0005DF804FB072105F0A3B800BF0068037998
:1039C000C901012BCAB206D0022B01D000207047DA
:1039D000782105F095B800B585B090F910C08DF844
:1039E0000F208268417C02F001020DF10F00CDE949
:1039F000000278226046FFF71DFE05B05DF804FB6B
:103A000000680379012B0BD0022B01D000207047F6
:103A10008368DB074FF0550219D5A52105F070B872
:103A200000B5826890F910C0417C85B002F00102B7
:103A300001920DF10F0200926046A5224FF0550C45
:103A40008DF80FC0FFF7F6FD05B05DF804FB2521EA
:103A500005F056B838B5184D9DF814E005EB401444
:103A60004FEA401C94F8990900B938BD490084F820
:103A7000AB29C4F8AC3984F8A9190023049984F857
:103A8000A8E9022205F6981584F8AA39C4F8B019F5
:103A900084F8B43984F89A29654409F0FBFA02469F
:103AA0000B462846FFF726FA94F89A39002BF4D1F2
:103AB00094F8B40938BD00BFD0300020F0B50446FA
:103AC00083B00D461746061D20680379012B1AD0D6
:103AD000022B02D0002003B0F0BD8368DB07324622
:103AE0004FF0FF015CBF3246FF2105F069FE002860
:103AF000F0D015B12379DB07E6D4002FEBD0237982
:103B00003B7003B0F0BD8268417C90F9100002F078
:103B10000102CDE90062FF22FFF79CFFE7E700BF4B
:103B200030B50446051D20680379012B83B017D0FA
:103B3000022B02D0002003B030BD8368DB072A4689
:103B40004FF0FF015CBF2A46FF2105F039FE002837
:103B5000F0D02379DB07EED520680379012BE7D17C
:103B60008268417C90F9100002F00102CDE9005218
:103B7000FF22FFF76FFFEAE730B50246044652F82E
:103B8000040B0379012B83B00ED0022B01D000204F
:103B900008E0FF2105F014FE0028F8D02079C0438A
:103BA00000F0010003B030BD8568417C90F9100041
:103BB000009205F001050195FF22FFF74BFFEBE7AF
:103BC00030B5B42283B00446FF21006804F0EEFF54
:103BD00010B9002003B030BD20680379012B04F137
:103BE000040514D0022BF4D18368DB072A464FF07A
:103BF000FF015CBF2A46FF2105F0E2FD0028E8D066
:103C00002379DB07E6D520680379012BEAD18268A6
:103C1000417C90F9100002F00102CDE90052FF2230
:103C2000FFF718FFEAE700BF30B50A4683B0044645
:103C3000A521006804F0BAFF10B9002003B030BD20
:103C400020680379012B04F1040514D0022BF4D170
:103C50008368DB072A464FF0FF015CBF2A46FF213D
:103C600005F0AEFD0028E8D02379DB07E6D5206813
:103C70000379012BEAD18268417C90F9100002F0AF
:103C80000102CDE90052FF22FFF7E4FEEAE700BFA0
:103C900070B582B0CDE900230446FFF791FF10B95B
:103CA000002002B070BD20685522A52104F07EFFDF
:103CB0000028F5D0251D20682A46FF2105F0D2FDF9
:103CC0000028EDD02379DB07F5D40DF1FF350DF198
:103CD000070615F8011F2046FFF7A6FF0028DFD0D2
:103CE000B542F6D1DDE700BF002A35D0F0B5044675
:103CF00083B00E468F18051D16F8012B2068A521EC
:103D000004F054FF90B9002003B0F0BD8268417CFC
:103D100090F9100002F00102CDE90052FF22FFF7F6
:103D200099FE0028EFD02379DB0710D520680379AE
:103D3000012BEBD0022BE6D18368DB072A464FF03C
:103D4000FF015CBF2A46FF2105F03AFDE9E7B742D3
:103D5000D2D1012003B0F0BD0120704770B596228A
:103D600082B004460E460068FF2104F01FFF10B920
:103D7000002002B070BD251D20680379012B1FD0E3
:103D8000022BF5D18368DB072A464FF0FF015CBFA9
:103D90002A46FF2105F014FD0028E9D02379DB072E
:103DA000EAD4E1222068114604F000FF0028DFD0A9
:103DB00020683246FF2102B0BDE8704005F052BDD8
:103DC0008268417C90F9100002F00102CDE90052B6
:103DD000FF22FFF73FFEDFE7002A43D0F0B504469D
:103DE00083B00E468F18051D20689622FF2104F02F
:103DF000DDFE90B9002003B0F0BD8268417C90F9EF
:103E0000100002F00102CDE90052FF22FFF722FE6E
:103E10000028EFD02379DB0710D520680379012B28
:103E2000EBD0022BE6D18368DB072A464FF0FF0177
:103E30005CBF2A46FF2105F0C3FCE9E7E1222068C8
:103E4000114604F0B3FE0028D4D020683246FF218A
:103E500005F008FD0028CDD00136B742C4D10120BD
:103E600003B0F0BD0120704770B505460B4604460F
:103E7000164655F8040B82B087211A4604F096FEC8
:103E800020680379012B1AD0022B02D0002002B047
:103E900070BD8368DB072A464FF0FF015CBF2A46EE
:103EA000FF2105F08DFC0028F0D02379DA07E7D454
:103EB000002EECD0C3F34013337002B070BD8268A3
:103EC000417C90F9100002F00102CDE90052FF227E
:103ED000FFF7C0FDE7E700BF70B5782182B0044668
:103EE00016460068002204F061FE10B9002002B0FE
:103EF00070BD251D20680379012B14D0022BF5D14C
:103F00008368DB072A464FF0FF015CBF2A46FF218A
:103F100005F056FC0028E9D02379DA07EAD45B09DA
:103F2000337002B070BD8268417C90F9100002F0DD
:103F30000102CDE90052FF22FFF78CFDEAE700BF46
:103F400030B5CC2283B00446A521006804F02EFED3
:103F500010B9002003B030BD20680379012B04F1B3
:103F6000040514D0022BF4D18368DB072A464FF0F6
:103F7000FF015CBF2A46FF2105F022FC0028E8D0A3
:103F80002379DB07E6D520680379012BEAD1826823
:103F9000417C90F9100002F00102CDE90052FF22AD
:103FA000FFF758FDEAE700BF30B5B42283B00446FE
:103FB000FF21006804F0FAFD10B9002003B030BD05
:103FC000251D20680379012B22D0022BF5D18368AF
:103FD000DB072A464FF0FF015CBF2A46FF2105F0B0
:103FE000EFFB0028E9D02379DA07EAD4CC21204678
:103FF000FFF71AFE0028E0D002E02379DB07DDD5C9
:1040000020682A46FF2105F02DFC0028F5D1D4E7D1
:104010008268417C90F9100002F00102CDE9005263
:10402000FF22FFF717FDDCE72DE9F04F8BB0CDE95C
:1040300007230446002004908A460390251D049B14
:10404000079A2046DE0002EBC30BFFF7B9FD20B94B
:1040500035E0237913F0010207D020682A46FF21BA
:1040600005F000FC0028F4D129E005929A07099098
:1040700040F1D880F0212046FFF7D6FDF8B1079B2C
:10408000DDF81480083E3344012606933746BAF122
:10409000000F54D0082F52D807F1FF394AFA09F916
:1040A00009F0010920684FEAC912782104F07EFD69
:1040B00028B120680379012B50D0022B06D00020B4
:1040C000089B049A1A700BB0BDE8F08F8368DB0779
:1040D0002A464FF0FF015CBF2A46FF2105F070FB26
:1040E0000028ECD0237913F00102E2D1C3F3801C45
:1040F000D9099B0646D5BCF1000F60D1BAF1000F7B
:104100005AD0082F58D8894540F08880B9F1000F5F
:1041100048D01BF8083033430BF8083076000137DD
:1041200016F0FF06FFB2B2D108F101085FFA88F875
:10413000B8F1080F43D00126BAF1000FAAD1049BB1
:10414000C3B1039BBB4215D9069B13F808301E422E
:1041500014BF4FF001094FF00009A3E78268417CCA
:1041600090F9100002F00102CDE90052FF22FFF7A2
:1041700071FCB5E7039BA3EB0709B9FA89F94FEA8C
:1041800059198FE7BAF1000F13D0082F11D88945BC
:1041900096D1B9F1000FBCD1059BBCF1000F08BF4F
:1041A0003B4605931BF8083023EA06030BF808305A
:1041B000B4E70029ADD1EFE70029AAD1F2E7402FFB
:1041C00006D8089B049A1B7893423FF638AF77E7EE
:1041D0009BF807700BF1FF360BF1060B16F801CFB9
:1041E000082182EA0C0343F30003013923F073032F
:1041F00083EA520211F0FF01D2B24FEA5C0CF0D117
:10420000B345EBD19742DCD1049B0133DBB204937D
:10421000059B002B3FF454AF0393D2E7DDF82480D5
:1042200040464DE7804640464AE700BF10B500686B
:104230000379012B84B00C461AD0022B02D0002047
:1042400004B010BD836813F0010F03AA4FF00303FD
:1042500014BF2221A22104F043FE0028EFD0BDF9B3
:104260000D3003EB83031B12E633238004B010BD33
:104270008368417C90F9100003F00103019303ABC4
:10428000009322220323FFF7E5FBE6E7F0B589B0B0
:104290000023904A02930393136843F4803313601E
:1042A00003E0029BB3F5A04F09D0136803F4003379
:1042B0000393029B01330293039B002BF1D0854BA8
:1042C0001B6813F4003318BF01230393039B012BD6
:1042D00001D000BFFDE77F4B7F491A6C7F4842F059
:1042E00080521A640A6842F440420A609A689A60EE
:1042F0009A6842F400429A609A6842F4A0529A6026
:1043000058601A6842F080721A601A689001FCD5F1
:10431000734A40F205711160996821F003019960B8
:10432000996841F00201A2F580629960936803F0F8
:104330000C03082BFAD1936803F00C03042B00F054
:10434000C680082B00F0AB80664A624B66499868CD
:10435000664D674E674FC0F303100144002491F887
:104360006810CA406449E9606449586FA960596B94
:10437000C6F8302C21F080015963596F604A6148BA
:1043800041F080715967196B0A431A635A6B5A637B
:104390009A6B9A631A6C5C490A431A64596C5B4ABB
:1043A0000A435A6448F2FF7123462246CDE900448D
:1043B00067F026F95648234622464FF6FF71CDE9AD
:1043C000004467F01DF95348234622464FF6FF711B
:1043D000CDE9004467F014F94F48234622464FF6D2
:1043E000FF71CDE9004467F00BF94C4823462246A3
:1043F0004FF6FF71CDE9004467F002F948482346C3
:1044000022464FF6FF71CDE9004467F0F9F84548C0
:10441000234622464FF6FF71CDE9004467F0F0F8DD
:104420004148234622464FF6FF71CDE9004467F02C
:10443000E7F8234622464FF6FF713C48CDE9004499
:1044400067F0DEF804A8FEF7FDFAD5F8FC20049921
:10445000D6F8303C364842F08072C5F8FC20354A28
:10446000C2F8B00F5460106840F0010010604FF4C3
:104470007A72B3FBF2F3013BB3F1807F2E4AB1FBBA
:10448000F2F2C7F8FC2908D24FF0E022F021536184
:10449000072385F823109461136109B0F0BD5168BA
:1044A000536852684902C2F388124CBF23490D4930
:1044B00003F03F03B1FBF3F303FB02F2054B5B6830
:1044C000C3F3014301335B00B2FBF3F23DE71B4A48
:1044D0003BE700BF0038024000700040085440072E
:1044E000003C02400024F4009062070800ED00E068
:1044F00000000020D03000200003FA050000000872
:10450000FF91670000000240FFC9FE10335707000B
:104510000004024000080240000C0240001002406B
:104520000014024000180240001C0240002002401B
:1045300055CEACC5001000E040420F0000127A00DA
:1045400082B0064B002201920193019B03EB800392
:104550000193019B196002B0704700BF50280040D2
:1045600010B51C2006F00EF81121044605F0E6FFF8
:104570004CB12368A2885A83C82008F0B9FD23688B
:10458000A2881A8310BDBDE81040C82008F0B0BD55
:10459000704700BF704700BF704700BF10B5104C98
:1045A00094F80A3A23B90F4B4FF480225A6110BD98
:1045B0004FF0E022D2F8103D23F00603C2F8103D80
:1045C000FDF770FED4F8103A9B68DB07EBD5D4F802
:1045D0000C2B136823F0030161F307031360E2E778
:1045E000D0300020003C01402DE9F04FA34CD4F81E
:1045F0000C3A5A69D5078BB002D50BB0BDE8F08FE5
:104600005A699B6912EA0301F7D0C1F30743080313
:10461000019300F1E180019B5D073FD48807CEB292
:1046200003D5D4F80C3A02225A610029C0F24A821A
:104630000A05C1F3072500F19981370708D5904B8A
:104640009048D3F8A03E9847D4F80C3A08225A6113
:10465000F60600F10F82E80600F1BE81A80600F11F
:104660001781019BDA0609D5854B8648D3F8B03E01
:104670009847D4F80C3A4FF480125A61019B9B067C
:10468000BBD57F4B7F48D3F8B43E9847D4F80C3A5B
:104690004FF400125A610BB0BDE8F08FD4F8103A15
:1046A0009E69DB691E40B6B2002EB7D0754D4FF043
:1046B000000B05F118080F46F00740F18280D4F88E
:1046C000101AD8F8002008694B6B23FA0BF3DB01B2
:1046D000DBB203439068034013F00109D8B200F045
:1046E0000F824B6B012000FA0BF023EA00034B63AF
:1046F00001239360624B6348D3F8983E5FFA8BF1D5
:10470000984794F8033A012B00F07E8219F0800F4D
:1047100057D0D5E94CC1D5F82431D8F800E0ACEB3E
:1047200001029342DEF8180028BF134680B203331B
:10473000B0EB930F45D9D4F8103A94F8039ACDE929
:10474000026BBA4667469C46B94237D2D5F8243147
:10475000781A984228BF184600F1030BD5F8283183
:104760004FEA9B0BB9F1000F10D182B203329210C5
:10477000D8F8B8600AD04946013153F8047B376055
:104780008A42F9D1D5E94C71D5F828310144034466
:104790008F42C5F82831C5F83411DEF818300AD137
:1047A00095F81C01012202FA00F0DCF8342022EA1C
:1047B0000002CCF834209BB29B45C5D3DDE9026BE7
:1047C000574676080BF1010B05F1280508F104089E
:1047D0007FF472AF394621E7D4F8103A9D69DB695E
:1047E0001D402D0C3FF417AF04F52068DFF890B0A2
:1047F000029104F6542600274FF00109C24608E052
:104800006D0807F1010706F1040608F1280800F019
:104810009181EA07F4D53068D4F8101A83684969A1
:104820000B40D9B2DB0740F1708194F8033AC0F82D
:104830000890012B07D10169D8F87C33C1F312012C
:104840005B1AC8F88C33DBF8943EF9B250469847AF
:1048500094F8033A012BD3D1002FD1D194F8113B16
:10486000052BCDD1D4F8543A07491961074959614C
:1048700019684FF080211960C2E700BFD0300020D6
:1048800000000020D03A0020180008609C40002062
:10489000D4F8105AD4F8182AAB68C3F34103022B9A
:1048A000136814BF0021032161F30A0313606B68CE
:1048B00043F4807306A86B60FEF7C4F8D4F80C2AA2
:1048C000079ED36823F47053D360A86810F0060FD6
:1048D000C0F3410100F03C819F49A048314481422E
:1048E00040F2AE819E48A6F57401A1F510518142B7
:1048F00040F2AA819B499C4831448142C0F0A88182
:104900009A48A6F18C71A1F54341814240F2A481FD
:104910009749984831448142C0F0A281964997480E
:1049200031448142C0F0A0819548A6F1B771A1F54C
:1049300058518142C0F0A08192499348314481424C
:10494000C0F09681914892493044884234BF062095
:1049500005204025012160F38D23D3604FF40053DF
:1049600084F8021AA4F8045A53617AE600238DF8F9
:10497000133094F8123B8DF81330864B8648D3F8E9
:10498000A83E9847D4F8103AD4F80C2A986894F8BE
:104990000A3A4FF400615161002B3FF44EAEC30759
:1049A0007FF54BAE94F8153B012B7FF446AE9DF896
:1049B0001330032B7FF441AED4F80C3B77491A68CF
:1049C00042F001021A601A6842F003021A600B6991
:1049D00043F006030B6130E6D4F8106AD4F80C1AE1
:1049E0007368002723F0010373600597059B43F06C
:1049F00020030593059B67F38A130593059B0B61C1
:104A0000674BBC460A690592013B02D0059A9206A3
:104A1000F8D494F8012A52B1624B03EB820EFF22C4
:104A200053F8040F8260D86B73458260F8D10B2372
:104A300063F3070763F3070C4FF0FF33B3614FF0E5
:104A40000113F3617761C6F810C03368564823F448
:104A5000FE63336094F8032AD4F8543A012A1861AB
:104A60006FD04FF480534B614A4B4B48D3F8A43E70
:104A70009847F3E5D4F80C3A9A6922F010029A614B
:104A80001A6AC2F34340022802F00F0100F090803E
:104A9000062812D101EB810104EBC101D4F8D06AE0
:104AA000D1F88C0DC2F30A1210443268C4F8CC2F2E
:104AB0003268C4F8D02FC1F88C0D9A6942F0100208
:104AC0009A61C8E594F80A3A3BB1D4F80C2B136804
:104AD00023F0030060F307031360D4F8102A2D4B72
:104AE0002D48D3F8AC5E5368029123F00103536064
:104AF000A847D4F80C3A02994FF000425A6197E562
:104B0000010707D5082393605BE68A0707D50223D0
:104B1000836075E6C3060FD51023936051E60B073B
:104B20007FF56EAEDBF89C3E50469847336808210F
:104B3000996065E602996EE5410679D54023936058
:104B40003FE61A4A5A611A684FF080221A6088E7D5
:104B50004FF400750920FEE6401E1BFF3F420F0088
:104B6000DFC810002013FBFE20D61300FF691800D9
:104B700000D3CEFE40771B00C05BB3FEC091210086
:104B800040AC2700C01D6AFE40E13300803C36FE89
:104B9000E09C410000000020D03A002000ED00E041
:104BA000410D0300E43A0020180008609C400020FA
:104BB00047F6F070104280D0C2F30A1201EB810078
:104BC00004EBC00002F1030C5FEAAC0CD0F8806D7E
:104BD000D4F8D0EA4FEA810818BF002006D001308F
:104BE000DEF8007046F8047B8445F8D1414404EBBC
:104BF000C101D1F8800D1044C1F8800DD1F88C0DA1
:104C00001044C1F88C0D58E7BBF1000F7FF47EAD66
:104C100094F8113B042B7FF479ADD4F8543A184A38
:104C20001A61184A5A611A684FF080221A606DE5BD
:104C3000830758BF81467FF569AD02239360C0E5C5
:104C4000012140250E2086E6012140250D2082E627
:104C5000012140250C207EE6012140250B207AE62B
:104C6000012140250A2076E601214025092072E62F
:104C70000121402507206EE60121402508206AE633
:104C8000180008609C40002070B5194D194BC5F8FC
:104C9000F43F05F5805300261970174BC0F85C618E
:104CA00083F8276940F20113A0F8443105F6F47344
:104CB000C0E954330D230446C0F8583100F5A27101
:104CC00066F002F91F23C4E9EC36E378012205F20D
:104CD00084559342C4F8A853A4F89C2308BFC4F891
:104CE000AC5304F567712046BDE8704066F0ECB83F
:104CF000D030002055534253D81F002070B50B7898
:104D000013F0600282B004462BD0202A30D14A78BA
:104D1000FE2A39D0FF2A2DD14A88002A3BD1CA88E1
:104D2000002A38D11B0636D46148624B80F8272907
:104D3000C4F8B423E278012183F8A415A4F89C13E5
:104D400003F284531F21012AC4F8B013C4F8A83316
:104D500004F5677108BFC4F8AC33204666F0B4F8B8
:104D600006E04B780A2B1AD00B2B08D0012B2AD047
:104D7000002002E065F03AFF022002B070BD4E4B09
:104D80004A8803F8F32CF3E74E8826B9CD88012D25
:104D900001D11A0642D4204665F028FFECE7022133
:104DA00080F811114FF48071A0F81C1143490123C0
:104DB000C0E94A11C0E94E33C0E94C3200F58E71AA
:104DC00066F020F8D4E78B88C0681E06DDB244D4B4
:104DD0000192019A3A4B42F010020192019A02614B
:104DE00002690192013B02D0019AD206F8D4314EF9
:104DF0002946204665F06CFF294696F8A455022303
:104E00004022204665F094FF022DB1D18121204639
:104E100065F024FF002386F8A435A9E7254BD3F8D5
:104E2000BC359B699847244BC0B203F8F40C0028AA
:104E3000B1D00222F43B84F811214FF48072C4E90E
:104E40004E55C4E94A33C4E94C56A4F81C2104F574
:104E50008E71204665F0D6FF8AE70092009A184BC3
:104E600042F020020092009A65F38A120092009AA2
:104E7000026102690092013B02D0009A9106F8D4C7
:104E80000C4E2946204665F023FF294696F8A45586
:104E900002234022204665F04BFF022DB6D0012DA3
:104EA0003FF466AF01212046FFF7EEFE60E700BF4A
:104EB000D81F0020D0300020C8410020D54000205D
:104EC000410D030010B50D4B93F82739022B07D085
:104ED000033B012B02D80021FFF7D6FE002010BDB6
:104EE000074B93F89115044666F0A2F80028F5DA0E
:104EF00001212046FFF7C8FEF0E700BFD81F0020C1
:104F0000D0300020F8B53F4C94F8276905467EB1B3
:104F1000012E01D00020F8BD3B4B93F8911566F0AF
:104F200087F80028F6DA31462846FFF7ADFEF1E7AC
:104F3000354FB0F8B433D7F88C25C7F8FC2F1F2BAA
:104F4000D7F88825C7F8F82F08D1304BD7F8842533
:104F50009A4203D197F8911501291AD92C4911F8D1
:104F6000F23C5A1CD2B201EBC303042A18BF164606
:104F70000222284687F8A42505244FF4005203F89E
:104F8000F04C01F8F26C43F8EC2CFCF731F90020FE
:104F9000F8BD97F89235013B0F2BDFD866F048F843
:104FA00000282ADB94F82739013B022BB2D9184B91
:104FB00033F8D01C0029B7D0D7F88C35C5F85C6120
:104FC000994228BF1946D7F8FC3FC5F858115B1A1B
:104FD000C7F8FC3F07F5805340F201111E700D4BDE
:104FE000A5F844110422C5E9543305F5A2712846F9
:104FF00084F8272965F068FF8CE72846FCF7F8F865
:1050000088E700BFD81F0020D0300020555342430E
:10501000C8410020886F002010B54FEA511E02449D
:1050200000EB8E0C624529D901F01F034FF0FF34CD
:1050300050F82E1004FA03F30B4093FAA3F3B3FADB
:1050400083F3DBB2202B16D10CF104018A4202D883
:1050500017E08A4212D98C460431DCF8003093FA0A
:10506000A3F3B3FA83F3DBB2202BF2D0ACEB000C4A
:1050700003EBCC0010BD03EB4E1010BD4FF0FF3022
:1050800010BD204610BD00BF0369416890ED067A4F
:10509000F0B4C56A3B4E876853EA010204BFD6F8F4
:1050A000381541606A1C30EE077A0133012A80ED21
:1050B000067A0361C26241D090ED075AD0ED096AC9
:1050C000D6F8384507EE902A70EE455AB8EEE76AF2
:1050D000611AC5EE867AB94277EE857A30EE670AB4
:1050E000C0ED087AE5EE806AC0ED077AC0ED0A6A85
:1050F000C0ED096A01D8F0BC7047012A2ADD07EE2D
:10510000905AF8EEE77A86EEA76AB5EEC06AF1EE3D
:1051100010FA1FDBF1EEC67AF4EE677AF1EE10FAC0
:1051200018D6D0ED056AF4EEE76AF1EE10FA14D560
:10513000037BF3B10323F0BC03707047D6F8382526
:1051400080ED080A521ABA424FF0000180ED070ABA
:105150004162D0D9DFED0C7AE3E707EE903AF8EE42
:10516000677A0223C7EE276AF0BC0370C0ED066AB7
:105170007047D6F838154160002203618261C3622E
:10518000B9E700BFD030002000000000DFED504A3A
:1051900010B5844600F1480E0346B1EC017AD3ED18
:1051A000067ADA6A77EE877A0132012AC3ED067A47
:1051B000DA6255D093ED075A93ED096A07EE902A0B
:1051C00077EE455AF8EEE77AC5EEA76A76EE857A6D
:1051D000F0EE466A37EE677AC3ED087AE5EE876A45
:1051E000C3ED0A6AC3ED077AC3ED096A1833734544
:1051F000D3D1384C4168D4F838250369521A8168F4
:1052000001338A4203612AD990ED056A00F1300E1C
:10521000DCF82C20DCED0A6A012A02F1FF3126DDE0
:1052200007EE901AF8EEE77A86EEA77AB5EEC07A26
:10523000F1EE10FA1BDBF1EEC77AF4EE677AF1EECD
:1052400010FA14D6E645B4EEE76A0CF1180C16D045
:10525000F1EE10FADCD5037B6BB30323037010BDB2
:10526000F0EE477AF0EE646A83ED087ABAE7DFED94
:10527000187AE645B4EEE76A0CF1180CE8D1F1EEC5
:1052800010FAE8D407EE903AD0ED066A90ED0C7A69
:10529000D0ED125AF8EE677A022386EEA76A037001
:1052A000C7EE276A85EEA77A80ED066AC0ED0C6A24
:1052B00080ED127A10BD0022D4F8381541600361E8
:1052C0008261C362026343648264C36510BD00BF30
:1052D00000000000D0300020B0EEC06AF0EEE05ACE
:1052E000F4EEC65AF1EE10FAF0EE407A0EDCB5EEAE
:1052F000400AF1EE10FA4BD0F4EEC65AF1EE10FA75
:10530000F0EE466A50D5B0EE655A03E0F0EE656AFD
:10531000B0EE465A85EE267A9FED252A9FED253A76
:105320009FED254ADFED254ADFED252ADFED253A01
:10533000DFED256AA7EE023AE7EE223AA7EE034A2E
:10534000B7EE005AE7EE044AA7EE235AE7EE246AC6
:10535000F4EEC65AB1EE667A87EE050AF1EE10FA5F
:1053600048BF9FED1A7AF5EEC00A48BF37EE400AF3
:10537000F1EE10FA48BF9FED167AF5EEC07A48BFFD
:1053800037EE400AF1EE10FA48BFB1EE400A70471E
:10539000DFED107A9FED100AF5EEC00AF1EE10FA7B
:1053A00058BFB0EE670A7047B0EE465AB2E700BF8A
:1053B00039094E3DE3B59EBE88FA16BE45FE7FBF55
:1053C00099FB243F69A2163EA7DFA8B4DB0FC93FB3
:1053D000DB0F4940A7DFA834DA0F494091ED007A8E
:1053E000D0ED047A90ED054AD0ED064A90ED075ACB
:1053F000D0ED085A90ED096AD0ED0A6AE7EE077A17
:10540000F7EE003AC0ED047A91ED007AD1ED017A21
:10541000A7EE274A90ED0B7A80ED054A91ED024AFE
:1054200091ED003AD0ED0C7AE3EE044AC0ED064A65
:10543000D1ED004A35EE245A80ED075AD1ED014AEC
:1054400091ED005AE4EE855AC0ED085AD1ED015AAB
:10545000A5EEA56A80ED096AD1ED015A91ED026AC7
:10546000E5EE866AC0ED0A6AD1ED016A37EE267A6A
:1054700080ED0B7AD1ED026A91ED007AE6EE877A43
:10548000C0ED0C7A91ED026AD1ED016AD0ED0D7A92
:1054900090ED0E7A90ED0F4AD0ED104A90ED115A32
:1054A000D0ED135AE6EE267A75EEA35AC0ED0D7ACA
:1054B000D1ED026AD0ED127A90ED006AA6EEA67ADE
:1054C000D0ED016A80ED0E7A91ED027A34EE074A52
:1054D00090ED027A80ED0F4A91ED004A74EE844A15
:1054E000C0ED104AD1ED014A35EE245A80ED115A33
:1054F00091ED025AC0ED135A77EE857AC0ED127A1B
:10550000D1ED017AD1ED005A91ED025A67EEA77AFA
:10551000E5EEA57AE5EE057AA5EEA76A80ED006ACC
:1055200091ED016AE6EE276AC0ED016AD1ED026AEB
:10553000A6EEA77A80ED027A90ED037A77EE277ACD
:10554000C0ED037A704700BF2DE9F04F4FF000091E
:1055500089B0864600F110050646034600F1300882
:10556000074648462C46CDF80CE08B469C46B24692
:1055700000283CD10CF1040CA445FBD1032800F118
:10558000010151D09C46AA46029398B1DCED047A01
:105590000192AAEB0903B6467246F3EC016A92ED5A
:1055A000007AE6EEC77A53450EF1100ECCED047A80
:1055B000F2D1019ADCED046A15ED047AC6EE877A21
:1055C0000CF1100CC4450AF1100ACCED007ADCD1C4
:1055D000029B04361433084608F1040814351034CD
:1055E000103709F104099C46B2460028C2D0DCED10
:1055F000007A0192D64639467246F1EC016A92ED84
:10560000007AE6EEC77A99420EF1100ECCED007AE0
:10561000F2D10CF1040CA445019A0AF1040AE6D176
:10562000032800F10101ADD1DDF80CE0002359465B
:1056300004930593069307937646774604AD0020BE
:10564000F2EC017AE5EC017AB0B104AC3B46B4EC83
:10565000017AF3EC016AE6EEC77AB34245ED017ACE
:10566000F5D1013004280BD0F2EC017A1037143652
:10567000E5EC017A0028E8D1103714360120DFE785
:1056800008AD75ED017A10310EF1400E0428744614
:10569000A1F1040241ED017A1ED07346F3EC016AD8
:1056A000B1EC017AE6EEC77AA342C2ED007AF5D1F9
:1056B0005EED016A87EEA67A013882ED007A17D096
:1056C000AEF1140E103C114675ED017A0428A1F1DB
:1056D000040241ED017AE0D15EED016A87EEA67A1F
:1056E000103CAEF1140E032001ED017A1146EBE7F8
:1056F00009B0BDE8F08F00BFDFED297AB4EEE70A0C
:10570000F1EE10FA28DD9FED277A30EE470AB4EE6D
:10571000E70AF1EE10FAF8DCDFED237AB4EEE70ADF
:10572000F1EE10FA2FDD30EE670A37EEC00A60EEB8
:10573000007A9FED1E7A9FED1E6ADFED1E6AA7EECE
:10574000876A9FED1D7AE7EE866A60EE275AA7EE1C
:10575000A67AA5EE870A7047DFED187AB4EEE70A5D
:10576000F1EE10FAD8D59FED0F7A30EE070AB4EEBD
:10577000E70AF1EE10FAF8D4DFED0B7AB4EEE70A9F
:10578000F1EE10FACFDC9FED0E7AB4EEC70AF1EE1F
:1057900010FA44BF30EE270A37EE400AC7E700BFD1
:1057A000DB0F4940DB0FC940DB0FC93F9A7C2E3627
:1057B000FAAF4FB93587083CA4AA2ABEDB0F49C00F
:1057C000DB0FC9BF10B5404CB4FBF2F4A14219D3B2
:1057D000DFED3E7AF7EE005AB0EE677AB0EE676A18
:1057E000F0EE676A0023C0ED005AC0ED017A80ED4B
:1057F000027A80ED036AC0ED046A8361436103624B
:10580000C36110BD07EE902AB8EE677ADFED307AFB
:1058100027EE277AB7EE006AC6EE076A07EE901AFF
:105820009FED2C7AF8EE677AB0EE405A67EE877AF1
:10583000C7EEA64AFDEEE47A17EE902A2032402AFF
:105840003FD8B0EE640AFFF757FFB0EE404ADFEDF5
:10585000227A34EEA70AFDEEC07A17EE902A2032A3
:10586000402A29D8FFF748FFF8EE006A60EE266A62
:10587000012B1CD0B7EE006A36EE406AF6EE004A05
:1058800066EE244A35EE055AF7EE007A84EE057A84
:1058900077EE275A37EEC75A84EEA57AC6EE257AF8
:1058A00086EEA56AC5EE256AF0EE475A9AE7B0EE95
:1058B000666AF7EE004AE5E7DFED086A9FED030A46
:1058C000D6E79FED024AC2E720A1070000000000D2
:1058D000BD378635DB0FC940DB0FC93F00000080B4
:1058E000DFED077A30EE270AFDEEC07A17EE903A28
:1058F0002033402B00D8FFE69FED020A704700BF1F
:10590000DB0FC93F000000002DE9F84FDDF82CB097
:105910009DF828408946002C1BF8011B0CBF4FF056
:1059200020084FF030081C1E0546174608463ADB93
:1059300000295CD0002C55D04FF0000A5B4600E0F7
:1059400064B313F8016B013C002EF9D1BAF1000FDA
:105950002FD1264644B14D454146284600D2B8478E
:10596000013CF8D10B9B18780146A0B14FF0FF34F1
:105970004FF0000A00E09B464D45284600D2B8474C
:105980005B4613F8011B0029F5D10B9BF61A5E4408
:10599000BAF1000F10D13046BDE8F88FBAF1000F10
:1059A0001BD15646E0E7634229B31C464FF0010A7B
:1059B000C4E70028E0D10646002C04F1FF3AEADDF6
:1059C00054464D454146284600D2B847013CF8D2DE
:1059D000013656443046BDE8F88F06460028DAD036
:1059E0002646C9E72646A2464FF0FF34C4E72646BE
:1059F000002CB0D1CFE76FEA040A0E46E0E700BF03
:105A00000FB430B583B006AB0B4853F8042B0193A9
:105A1000D0E9320166F05CF9084C0546D4F8200E56
:105A200003685B6998470028F8D0284603B0BDE8B2
:105A3000304004B0704700BFC8410020D81F00208C
:105A40000EB410B583B005AB044653F8042B0749D8
:105A5000009301A8019466F03BF9019B00221A70A3
:105A600003B0BDE8104003B0704700BF290A00082A
:105A70000CB470B5334CD4F8D030A4B0002B5CD04B
:105A800094F8D83099420AD9D4F8DC200123834015
:105A9000134204D124B0BDE8704002B070472A4BD5
:105AA0002A4AD3F83835A2FB030292094FF47A71DF
:105AB00001FB123304A82649FFF7C2FF04AA29AB51
:105AC0000244CDE902322349289A064603A866F02B
:105AD000FFF8039B0A22591C03911A70039B0022B2
:105AE000591C03911A70D4F8D050ADB12B681B6AC1
:105AF0001BB128469847D4F8D0509DF810100029C3
:105B0000C8D00DF111042B6828461B68984714F87B
:105B1000011B0029F7D1BDE7D4F8D430002BB9D050
:105B200030440222009204A98218FD2036F054F875
:105B300024B0BDE8704002B07047D4F8D430002BD8
:105B40009ED1A7E7C8410020D0300020D34D62107D
:105B5000E41708081D0A0008184A10B5D2F8E040FA
:105B6000033004EB9003B3F5007F17D802EB8101FB
:105B7000C2F8E030E43202EB8404D1F8E42820F0EB
:105B800003001044C3F50073C1F8E4080C4A9B00FD
:105B900004210020FFF76CFF204610BD00210846BD
:105BA000084AFFF765FF084AD2F89430002443F012
:105BB0000073C2F89430204610BD00BFC8410020D9
:105BC000F017080814180808000000102DE9F0412B
:105BD0000268214D0746002455F834309A4209D016
:105BE00001340E2CF8D11D4A00210520FFF740FF9B
:105BF000002013E01A4B03EB8408D8F8C0657EB18F
:105C0000797901EB410306EBC30300221820C3E9B5
:105C1000032200FB01609F601A750430BDE8F0812B
:105C200007216420FFF798FF0146C8F8C00568B156
:105C3000314664226CF0ACFDD8F8C06505EBC405B4
:105C4000C6E90056F6617663F664D9E7054A052091
:105C5000FFF70EFFCCE700BF1863070824180808F9
:105C6000D03000204C18080870B50668F46982B07E
:105C70000546002C3FD03379012B04F103022DD0CF
:105C8000022B26D1B36813F0010F30464FF00D03FD
:105C900014BF0C218C2103F023F9A070D8B1B4F902
:105CA0000A3007EE903AF8EEE77AC5ED077AB4F9D4
:105CB0000C3007EE903AF8EEE77AC5ED087AB4F9C1
:105CC0000E3007EE903AF8EEE77AC5ED097A02B0A9
:105CD00070BD0023A370002002B070BDB368717C5A
:105CE00096F91000009203F0010301930C220D239A
:105CF000FDF7B0FED1E709211420FFF72DFFF06179
:105D000004462E68B7E700BF38B50568EB6904465E
:105D1000E3B1987800B938BDB3F9042007EE902AB2
:105D2000F8EEE77A0120C4ED047AB3F9062007EE15
:105D3000902AF8EEE77AC4ED057AB3F9083007EE59
:105D4000903AF8EEE77AC4ED067A38BD09211420BE
:105D5000FFF702FF0346E861DBE700BF03681A466E
:105D6000591C016012F8021B0260587841EA0020B9
:105D7000704700BF10B402681346511C016013F84D
:105D8000021B0360D31C5478036093781B0443EA1E
:105D90000423141D0460D0785DF8044B0B4343EAE0
:105DA0000060704712B370B50446864604E0981B45
:105DB00017D114EB0C0C15D01EF8013BA3F14100D8
:105DC000192811F8010BA0F1410598BF2033192DB6
:105DD000A2EB0E0C00F12006E9D91B1A04D1002811
:105DE000E7D170BD604670BD184670BD1046704763
:105DF00010B402888378184C02F0030101EB4101D2
:105E0000013B03EB810304EB4303C178B3F8F830A3
:105E1000A2F5FA62920840F2B55404FB02334A1E1E
:105E20001344017942798479008903EB430301EB40
:105E3000C301C1EB0111094B02EB8102C2EB02125B
:105E4000234403EB820300214FF47A72C3FB020167
:105E50005DF8044B704700BF9062070880436D38BF
:105E6000F8B516461F460446394630464FF47A7256
:105E700000236FF055FC3C4D3C4B054483FB056013
:105E80002844E917C1EB601183FB01030B44384E32
:105E9000C817C0EB631086FB003CC317354EC3EB3D
:105EA000AC0386FB03764FEAE37ECEEBE61EC1EB46
:105EB0000116A5EB860CC0EB0015A1EB8501617105
:105EC00003EB4301A0EBC10040F2B55101FB1E33CF
:105ED000B3F5896F84F806C020714FEA8E0637DA71
:105EE00040F2DA218B4239DCB3F5B77FB4BF4FF013
:105EF000000E4FF0010E20490EEB4E0001EBC001E9
:105F00007546B1F80E014FEA4E071C4907EB0E0C1F
:105F100001EBCC0C0CF1160C0B2101E03CF8020D4E
:105F2000984212DD0139F9D11349774401EBC701D9
:105F3000B1F8F8000121013306F5FA6E1B1A754419
:105F4000A170E37022812580F8BD0131C9B2F2E76A
:105F5000032540F29650AE460627D6E7022540F2CA
:105F60002940AE460427D0E780BC92C7898888883C
:105F7000ABAAAA2A73B06D16906207088863070857
:105F800030B52F4C86460D460FCC8DB0EC46ACE8B4
:105F90000F000FCCACE80F0094E80F001EF0030FC9
:105FA0008CE80F000FD1274B274A03FB0EF3B2EB0F
:105FB000B30F43D3254AB2EB331F34BF0122002273
:105FC000C2F11D0200E01C220EF1FF33002B0192F2
:105FD00040F26D12194602FB0EF2B8BF0EF102013B
:105FE00002EBA1021A491B4C81FB0301DB17A3EB57
:105FF00061100244C3EBE1131A44253284FB0231E1
:106000001144D317C3EBA103C3EBC303D31AADF100
:106010000402EE4602EB85015EF8040FC21884FB11
:10602000023C9444D317C3EBAC03C3EBC3037145E9
:10603000A2EB0303F0D1C01A0DB030BD1D22C3E79F
:10604000E8630708295C8FC2285C8F020AD7A30087
:106050001F85EB51932449920E4B10B5D3F870492C
:10606000D3F8743954EA030209D1014640F201130E
:106070000020C1F8023088710880088110BD064AEE
:10608000D2F83825121943F10003FFF7E9FE012089
:1060900010BD00BFC8410020D030002088422DE94B
:1060A000F0414FF001043DD301FB04F4B0FBF4FCDC
:1060B0008C45F9D23CB3002616E0BCF1090F274607
:1060C00098462C4623DD002A0CBF4FF0570E4FF0A8
:1060D000370EF444B94288F800C003F1010306F119
:1060E000010610D8B0FBF5FCB4FBF1F504FB1C0075
:1060F000002EE2D1BCF1000FDFDCA1420AD90CF185
:10610000300C03F801CB00221A70BDE8F0814FF08B
:10611000300EDEE7B0FBF5FC2C4605FB1C00B5FBA2
:10612000F1F5E7E78446C6E72DE9F04104469442DD
:106130001546084609D2B4FBF2F6154B05FB16448A
:106140001B5D00F8013BBDE8F081B4FBF2F696421E
:10615000B6FBF2F70CD20E4B05FB176705FB164496
:10616000DA5D00F8012B1B5D00F8013BBDE8F08112
:10617000BA42B7FBF2F807D9054B05FB187813F8BC
:10618000082000F8012BE7E74046FFF7CDFFF3E7D3
:1061900068180808B5EEC00ADFED347AF1EE10FA9F
:1061A000CCBF30EE270A30EE670ADFED317A20EE01
:1061B000270A30B5FDEEC07A87B017EE904A054643
:1061C00084EAE470002303A9A0EBE470CDE9003376
:1061D000029362F003F9002CB4BF2D23202303A8FF
:1061E0008DF800306EF08CFB012829D0022833D0C6
:1061F00003281DD003A968466EF0C2FA68466EF007
:106200007FFBC41EE4B22246694628466AF0A8FE17
:1062100000232B5528466EF073FB2E232B540130A0
:106220000DEB040128446EF0CBFA284607B030BDD0
:10623000302303A968468DF801306EF0A1FADDE73E
:1062400043F23002302303A96846ADF801208DF8EF
:1062500003306EF095FAD1E743F2300303A96846A4
:10626000ADF801306EF08CFAC8E700BF6F12033A48
:1062700000007A440278202A034600F10100F9D098
:10628000092AF7D02D2A29D02B2A03BF5A78B7EE36
:10629000000A0346B7EE000AA2F13001C8B209288D
:1062A000DFED4C7A10D8F2EE046A07EE101AB8EE61
:1062B000C77A13F8012FA7EEA67AA2F13001C8B26F
:1062C0000928F0EE477AF0D92E2A49D0197801F042
:1062D000DF01452907D020EE270A70475A78BFEE24
:1062E000000A0346D8E710B459782D2962D02B292B
:1062F00054D0A1F13002092A03F1010355D800243A
:10630000002202EB820201EB420213F8011FA1F10D
:1063100030000928A2F13002F3D9B2F59A7F134672
:1063200028BF4FF49A73072A50D9DFED2B6A1A461B
:10633000B7EE007A083A072A27EE267AFAD803F051
:1063400007032BB1F2EE046A013B27EE267AFBD15C
:106350006CB3C7EE877A5DF8044B20EE270A7047CE
:106360005978A1F13002D0B2092803F10103AED867
:10637000F2EE046AF0EE665A07EE102AB8EEC77A1B
:1063800013F8011F87EE266AA1F13002D0B2092866
:1063900066EEA56A77EE867AEED998E79978A1F14C
:1063A0003002092A03F10203A9D9B7EE007A67EE99
:1063B000877AD0E79978A1F13002092A03F1020324
:1063C00088BFB7EE007AC4D8012499E7B7EE007A07
:1063D000B7E700BF0000000020BCBE4C0378202BB4
:1063E000024600F10100F9D0092BF7D02D2B08BF90
:1063F0005378A3F13001CBB206BF02464FF0FF3C09
:106400004FF0010C092B4FF0000000D9704712F833
:10641000013F00EB800001EB4000A3F13001CBB263
:10642000092BF4D90CFB00F0704700BF2DE9F04FA9
:1064300091B042F0ABF942F06DF9B0F1000A40F3CF
:106440003C810024DFF80C93B54D27462646A04634
:1064500004E006F50066B24540F3958020220DEB7E
:106460000201304642F0E0F8AE49122208A86BF073
:10647000B1F883460028ECD1BE4222D0AA4BAB49EA
:1064800008EB480203EB820308F10108424601933E
:106490001846F31B0293FFF7D3FA4A46019B42F8D2
:1064A0004C3B029BC9F80C70C9E90433D9F81C3085
:1064B000C9E908339E4BC9F828300123C9F80830D0
:1064C00091469C4BD3F8D034C9F81C303746122281
:1064D00002F140030DEB03012B5D11F8201C9942E2
:1064E00002F101020BD00024202AF1D12037BA4555
:1064F00008A938463EDB42F097F80022E8E701346D
:10650000152CF1D1D01920220DEB020142F08CF8AC
:10651000894907AA08A86AF0AFFC58B30023CDE95F
:106520000133CDF814B0039304931F469B467B1EA2
:10653000042B00F2BA81DFE803F082728A8603003E
:10654000CDF814B0FFF74AFF059B8346049989B143
:10655000DDE9012042EA401203985B0143EAC023CF
:10656000A1F2BC7143EA6B0342EA412243EA0243CF
:10657000C9F81C30B8F1640F6DD0374606F50066D7
:10658000B2453FF76BAFB8F1640FC34663D0BE426C
:106590001BD0654C65490C2303FB084408F1010B33
:1065A0005A462046FFF74CFA614BC9F82830F61BD3
:1065B000D9F81C30C9F80040C9E90376C9E90833A5
:1065C0000123C9F81460C9F80830BBF1000F0BF1C2
:1065D000040143DC594C574A4FEA4A03B3F1805F48
:1065E000D2F8D0546EDB564954484FF498726AF092
:1065F000B7FC544BA3F11C0203F598719D60C3E9ED
:1066000000554C338B42F9D1A06828B923791BB1CE
:106610002368002B40F0A28011B0BDE8F08FFFF797
:10662000DDFE01904449002007AA01376AF024FCEE
:1066300000287FF47CAF5B46DDF814B086E7FFF7F7
:10664000CDFE0290EEE7FFF7C9FE8346EAE7FFF7CB
:10665000C5FE0390E6E74FF0640B6821374C354ADE
:10666000D4F84C61C2F8D0644C2707FB01F56319DC
:106670003A46002118466CF08BF83A4600216CF03F
:1066800087F8314A625105F11002DFF8CC80284FBB
:10669000C0F820804FF00109C0F80890876244F8E4
:1066A00002A022441835C2F804A0221D0BF10501F6
:1066B000565115446E6046628DE71E4B1F4CD3F851
:1066C000D05404214FF04C0808FB01F6A7194246AC
:1066D000002138466CF05CF84246002138466CF0E8
:1066E00057F81A4BA3514FF0010906F11002DFF8D9
:1066F0006880C7F80890CAF1006303FA09F34FF005
:10670000020BC7E9078887F805B01148A35006F1C6
:10671000180122445360455001444D607D6262E798
:10672000B418080890180808404B0020A41808085E
:1067300095220008F8100020CC18080810500020FE
:10674000186407082C500020D4180808E41808081A
:1067500014500020405100200068994F0026002767
:106760005449A064C4E91067E063064607469646AC
:10677000CD6C01F14C036DB39D689F6406F1FF3C45
:106780006545C1E92377DF630ED006F1010C65454D
:106790001DD113F8486C002E3FF43EAF196443F846
:1067A000083C2E461946E3E7002E3FF435AF53F878
:1067B0000C1C2E46002E3FF42FAF0D6CEA6B02F13D
:1067C000010CC5F83CC01D648B641946D0E7B54286
:1067D000F0D021E7724602272E46A64615E0D36B7D
:1067E00017635B0118BF03F6FF73C2E9046614BFA9
:1067F00001EB13333B4653631946916352F84C4FF8
:10680000CB1A1D444F1C0130CCB11379791E002BDB
:10681000E5D1136917635BB103F6FF73546901EBAC
:10682000133353634CB104F6FF7C01EB1C31E4E7F6
:1068300054693B465363002CF5D13946DDE71E4AC7
:106840001E4BC2F81C0E013902F55F60C2F8F43D20
:106850003E2640233F27C2F8105EC2F8003EC0E942
:1068600002677446C2F80C1E8D0F8B00D9B140F23E
:10687000FF169B1945F100055B0A43EAC553C0E9C1
:10688000094403F14004234403EBC101C2F8083E6C
:10689000C2F8F01DCB0D490240F8043CC2F8044E8A
:1068A00040F8081CB8E60123E9E7FFF797FD0490DC
:1068B000B8E600BF10500020D81F0020F4180808C8
:1068C00070B5344D2B787E2B01D0002070BD08228E
:1068D0004FF4FC4341F2210019B200294FEA43036F
:1068E000B6BF80EA41019BB28BB2013AF4D1B5F850
:1068F000011069B32848294CA042E6D20638461850
:10690000A642E2D241F2210C0529DED9864214D0FA
:10691000013806F1FF3E10F8012F082183EA022317
:106920001AB2002A4FEA4303B6BF8CEA42029BB276
:1069300093B20139F4D17045EDD1318849B1B21D1E
:10694000A242C2D27218A2423046BED21646DBE73D
:10695000134E741E41F22100A44614F8012F0821A1
:1069600083EA02231AB2002A4FEA4303B6BF80EA41
:1069700042029BB293B20139F4D16645ECD17288E0
:10698000D01A084A331D5B1BB0FA80F04009A2F808
:10699000283E70BD00000E0807000E080000100819
:1069A00001000E08C84100202DE9F04F914B924A9A
:1069B0008BB00020D21ACDE90600CDE90800D1182D
:1069C00005928E4A0393049110690028C0F28181D8
:1069D0008A4AF320D060002008908948012288422A
:1069E0008DF8242000F271817E2007928DF8180026
:1069F0004FF4FC42082041F2210514B2002C4FEA6A
:106A00004202B6BF85EA440492B2A2B20138F4D180
:106A10007C48ADF802207C4A90427CD2804641F20C
:106A20002105B8F80200B8F80020C0F30B07C2F344
:106A30000B04120BBE1D4FF000098DF80820020454
:106A4000ADF80460ADF806408DF8099000F1C38000
:106A500006338B4200F2398101AE0DF10A0B344648
:106A600001E0A34513D0079B14F8011B03F1280292
:106A70006A440133042B079302F8101CF1D106A9D4
:106A800003A8F9F7F3FFA345CDE90790EBD1089BE5
:106A9000002BC0F21A81BDF8024016F8013B082213
:106AA00084EA032423B2002B4FEA4404B6BF85EAEC
:106AB0004303A4B29CB2013AF4D1B345EDD1D8F866
:106AC00004603A46314603A8FAF790F80028C0F26D
:106AD000FC80F019864213D0711E013811F8013F75
:106AE000082284EA032423B2002B4FEA4404B6BFF1
:106AF00085EA4303A4B29CB2013AF4D18142EDD1BC
:106B0000DDE90302ADF8024011463F4A08F11408DE
:106B10009045034685D302334FF000089942ADF803
:106B20000480C0F0D28001AD2E460DF106042F4640
:106B300001E0BC4213D0079B17F8011B03F12802A8
:106B40006A440133042B02F8101C0793F1D106A903
:106B500003A8F9F78BFFBC42CDE90780EBD1089B76
:106B6000002BC0F2B280BDF8023041F2210016F8CD
:106B7000012B83EA0223082219B200294FEA4303BA
:106B8000B6BF80EA41019BB28BB2013AF4D1B44264
:106B9000EDD10399ADF80230049B0231994200F225
:106BA00094800DF10206144602E0B54200F08A809E
:106BB000079B16F8011B03F128026A440133042BDA
:106BC00002F8101C0793F0D106A903A8F9F74EFFAD
:106BD000CDE90740E9E7CB460BF1010B06335FFA3D
:106BE0008BFB99428DF809B06FD301AE0DF10A0A03
:106BF00034460DE000000E0800001008003C024082
:106C000001000E081C870808088C0808A24515D04A
:106C1000079914F801CB01F128030DEB03000131B2
:106C20000429079100F810CCF0D106A903A8F9F7C0
:106C30001DFF0023A24508900793E9D1089A002A76
:106C400043DBBDF8024016F8012B082184EA022438
:106C500022B2002A4FEA4404B6BF85EA4202A4B237
:106C600094B20139F4D1B245EDD1D8F8041001EB5A
:106C700009063A46314603A8F9F7B8FF002824DB95
:106C8000F019864213D0711E013811F8013F082215
:106C900084EA032423B2002B4FEA4404B6BF85EAFA
:106CA0004303A4B29CB2013AF4D18142EDD1DDE9B3
:106CB0000302BBF1030FADF8024003461146B9448D
:106CC0008AD121E7089B002B09DA00200BB0BDE830
:106CD000F08F1548506000F18830506078E60798D2
:106CE00040B912490A6942F000420A61B3FA83F0DE
:106CF0004009EBE7DDE9033203449342E5D806ABF4
:106D0000C0F10402002118446BF042FD06A903A85B
:106D1000F9F7ACFE002803460890D6DB9DF8242046
:106D2000002AE3D0DDE700BF23016745003C0240B5
:106D300008B5FFF739FE40B9FFF736FE28B9FFF76F
:106D400033FE10B9052007F02DF8FFF7B9FD002834
:106D5000F8D008BD70B545880B460446C5F30B0551
:106D60002A46002118466BF013FD0A4A2169914218
:106D7000034606D3084A914206D3BDE87040184640
:106D800008470029F9D170BD2A46BDE870406AF075
:106D9000E7B800BF088C0808BB9008082DE9F0414F
:106DA00003EB4306964602EB460612F9067B86B0D5
:106DB0000346754692F80080A3EB0804A3EB070C8A
:106DC000002CB8BF6442BCF1000FB8BFCCF1000C7E
:106DD0006445B8BF154602F10602B8BF4FFA88F7FE
:106DE000B242E7D16A889EF80000B842144614D136
:106DF000BEF80200A1EB0008A1EB020CB8F1000FF5
:106E0000B8BFC8F10008BCF1000FB8BFCCF1000C4E
:106E1000E045BEBF7546024604460EF1060E7645B5
:106E2000E1D16A7904922A79CDE902422878054AAB
:106E3000CDE9001003210120FEF71AFE284606B016
:106E4000BDE8F081FC1808084FF4006383817047A7
:106E50004FF4006383817047012070470120704721
:106E60002DE9F04F734D2868AB88B5F910E0B5F9FE
:106E70000CC0B5F80A80B5F9126085B0C3EB2014D8
:106E8000009204FB04F4B5F90820CDF80CE02413BB
:106E900002FB04F45B00B5F906200296C3EBE003A5
:106EA00002FB03F3A41304EBE3242B6A0193A4F580
:106EB000FA30B5F90E30EC6180FB00EA4FEAE37B73
:106EC00003FB0AF98CFB00C20EFB0B99A3FB0E3BE4
:106ED000CB4412031B0A42EA1C5243EA0B634FEAFB
:106EE0000C3C13EB0C0342EB2B22A3FB083C02F5FA
:106EF000004208FB02CC4FEAEC734FEA6C0953EAFC
:106F00006C0C0F46B5F9141000F09180029E019AA6
:106F100086FB0008C2F5801C01FB0AFA4A464FEACC
:106F200048484FEAE17948EAD0380EFB09A9400405
:106F3000A1FB0E1E4118F14449EB080900200CF09A
:106F40000048039E411848EA5C084FEACC7CBCEB41
:106F5000010C09EBC60968EB09081CEB0C0E48EBA9
:106F600008011EEB0C0E48EB010188014FEA8E1957
:106F700040EA9E601EEB090E41EB0001890041EAE8
:106F80009E714FEA8E0E1EEB0C0E48EB01014FEA8C
:106F90008E00890010EB0C0041EA9E7148EB010164
:106FA0006EF0BEFBB5F91A304FEA61384FEA503E39
:106FB0004EEAC14EDA1703FB08F984460EFB02992C
:106FC000B5F91800B5F91620A3FB0E35A94403FB4B
:106FD00008F50EFB0955A3FB0E3E75445B0E43EA14
:106FE000C51313EB0C0341EB65654FEAE07E00FB34
:106FF00001F10EFB0C11A0FB0C0C6144C00C40EA2B
:1070000041301B1845EBE1451B0A43EA056303EBDE
:1070100002130FB11B0A3B60009B23B104EB8404F5
:10702000803424121C60012005B0BDE8F08F0023DD
:10703000EFE700BF887F002031B10A4BD3ED0F7A14
:10704000FDEEE77AC1ED007A52B1064B9FED067A6C
:10705000D3ED107A67EE877AFDEEE77AC2ED007A1B
:1070600001207047887F00200000C842012070473F
:1070700010B40E4B0E4C1B68606C1B1AFA2B09D80F
:1070800009B1E36C0B600AB1236D136001205DF858
:10709000044B7047074A1368002023F0040384F868
:1070A000480013605DF8044B704700BF08360020AD
:1070B000887F00209800001001207047044B0022B8
:1070C00000215A659A65DA6519660120704700BF8C
:1070D000887F00200F4B104A1B68116E5B1AFA2B39
:1070E00016D8D2ED156A92ED167AD2ED177AFDEE2A
:1070F000E66ABDEEC77A16EE903AFDEEE77AC386F1
:1071000017EE103A038717EE903A43870120704735
:107110000020704708360020887F00200048704714
:10712000CC15002000487047EC7F0020437913F015
:10713000010306D0D0E90731C268581A531E18401F
:1071400070471846704700BF437913F0020307D019
:10715000D0E909130269581E401A531E184070479F
:10716000184670474379024613F0010014D0106AA4
:10717000D168D36901F1FF3C1B1A13EA0C030AD052
:1071800053691B5C00F1010CD8B2BCFBF1F301FBAD
:1071900013C3136270471846704700BF43799B07BB
:1071A0000AD5436A8269D154436A02690133B3FB49
:1071B000F2F102FB11334362704700BF4171704727
:1071C000D0E90920101AB0FA80F04009704700BFDA
:1071D000014B5B6F5B681847887F0020024B5B6F39
:1071E00008309B68184700BF887F00200120704747
:1071F000012070470120704701207047012070472F
:1072000031B10C4BD3ED1E7AF8EEE77AC1ED007A7E
:1072100072B1084BDFED086ADB6FA3F5D543333B52
:1072200007EE903AF8EEE77A87EEA67A82ED007ADA
:10723000704700BF887F00200000C84201207047CF
:107240000120704710B4754C0023224692F90410B7
:10725000012902F10C023AD00133072BF6D1224664
:10726000002392F90410022902F10C0245D00133E7
:10727000072BF6D12246002392F90410032902F1CC
:107280000C0255D00133072BF6D12246002392F988
:107290000410042902F10C025ED00133072BF6D151
:1072A000002394F90420052A04F10C0468D001336A
:1072B000072BF6D15A4B5B685B067BD401795DF8EE
:1072C000044B203901298CBF002001207047554A0A
:1072D00003EB430302EB8303D3F8803003B3524A3A
:1072E000037992F83DC09C4503D092F83C209A4225
:1072F000B5D101205DF8044B70474A4A03EB4303C4
:1073000002EB8303D3F8803063B1484A037992F8E3
:107310003D109942EDD092F83C209A42AAD1E8E77C
:1073200022469EE722460C3212F9081C0329A9D1F5
:107330003C4A03EB430302EB8303D3F88030002B7A
:1073400036D03B4A037992F83D109942D1D092F859
:107350003C209A4299D1CCE7324A03EB430302EB3B
:107360008303D3F88030002B9BD0324A037992F804
:107370003D109942BDD092F83C209A4290D1B8E796
:10738000284A03EB430302EB8303D3F88030002B3E
:1073900090D0294A037992F83D109942A9D092F8E9
:1073A0003C209A42A5D01E4B5B685B0686D501E067
:1073B00022466CE7214B00229C4619460C791A2C78
:1073C00001F1140104D001320C2AF7D1002403E0AA
:1073D00002EB82020CEB820400221979192903F1D5
:1073E00014030BD001320C2AF7D1002C3FF466AF06
:1073F000226803689A427FF461AF7AE701681CB1A2
:1074000023688B423FF475AF0D4B02EB820203EB16
:1074100082031B698B427FF451AF6AE7088000202A
:1074200098000010887F0020B40000200003002096
:107430004C05002098070020E4090020DC150020FE
:10744000CC1500200C4B10B5844603F1F00E002043
:1074500002E014339E450ED01A686245F9D1DA680D
:107460008A4218BFD96000F1010403F1140318BF68
:10747000E0B29E45F0D110BDDC150020044B03EBBB
:107480008003D3F8D8300BB19B681960704700BFF8
:10749000887F0020044B03EB8003D3F8D8300BB176
:1074A0009B68196027F026BC887F0020704700BFCA
:1074B000044B40F2FF7203EBC0039142A8BF114698
:1074C00099807047404100200D4A92F8003183B105
:1074D0000C4B93F8181161B193F8191161B1D2F8FE
:1074E00004010022FA2883F81921A8BF4FF0FF30C9
:1074F00070476FF0010070476FF00200704700BFE7
:10750000CC150020887F00200C4B93F81A218AB1FB
:1075100093F81B215AB10A49D1F808010022B0F5AD
:10752000967F83F81B21A8BF4FF0FF3070476FF0A4
:10753000020070476FF00100704700BF887F002095
:10754000CC150020024BD3F81C315B68184700BFF4
:10755000887F0020024BD3F81C319B68184700BF7E
:10756000887F0020024BD3F81C31DB68184700BF2E
:10757000887F0020014BD3F80C017047CC15002008
:10758000054B93F820311BB1044BD3F81001704721
:107590006FF00100704700BF887F0020CC150020ED
:1075A0004B1EDBB2062B98BF214A30B598BF32F88C
:1075B0001350204BA3F1580488BF4FF48075002866
:1075C00008BF1C46A44620893CF8082B87B04FFA18
:1075D00082FE90B1A5EB0E022B1A002AB8BF5242D0
:1075E000002BB8BF5B429A42C4BF64464FFA80FE8C
:1075F0003CF8080F0028EDD122880F4B0F4893F874
:1076000021C1A3790593A38804930D4BBCF1000F0E
:1076100018BF0346A078CDE90015CDE9022003216B
:10762000084A0120FEF724FA204607B030BD00BF0B
:107630004070070838170020887F0020E42D0808D4
:10764000001A0808041A080870B50668F0690D46A3
:107650001446A0B3D0F80130CDB1D0F805209FED8D
:107660001B7ADFED1B5ADFED1B6A07EE902AF8EE5E
:10767000677AB7EE006A77EEC77A77EEA77A87EE79
:10768000A57A77EE467A67EEE67AC5ED007AACB178
:1076900007EE903A9FED107ADFED106A9FED106AC9
:1076A000F8EEE77A67EE877A87EEA67ADFED0D6A65
:1076B00077EE467A77EEA67AC4ED007A70BD09219E
:1076C0001420FEF749FAF061C4E700BF9AC9CC4420
:1076D0009AC94C460E76D7450000484300E0FF4467
:1076E000000048423393884370B50668F06982B061
:1076F0000D461446002848D0D0F80530DFED266A44
:107700009FED267A07EE903AF8EE677AD0F80130CE
:1077100077EEE67AF3EE096A67EE877AB2EE047ADC
:1077200067EEA67AF4EEC77AF1EE10FA20DCBAEE34
:10773000047AF4EEC77AF1EE10FA19D42DB19FED68
:10774000187A67EE877AC5ED007A7CB107EE903A39
:107750009FED146ADFED146AB8EE677ADFED137AF5
:10776000E7EE067A77EEA67AC4ED007A02B070BD35
:1077700017EE900A6DF018FB0D4ACDE900010421C7
:107780000320FEF775F902B070BD09211420FEF741
:10779000E3F9F061B0E700BF000000460000803868
:1077A0000AD778430319C83D33938843000048C281
:1077B000501A0808244B254A30B5D3F8244194F9CF
:1077C0001030A16803EB830302EB830283B08DF8D2
:1077D0000700D2F8CC018A070AD501230DF1070270
:1077E000002164F04DF9A3689B0714D503B030BDA8
:1077F000636913B11A689B885383154B15491A683E
:10780000154B4D68D200A3FB023292094B685B1BFB
:107810009A42FBD2E1E70E4B0E491A680E4B4FF429
:10782000FA7000FB02F2A3FB0232486892094B682F
:107830001B1A9A42FBD26369002BD7D01A689B8827
:10784000138303B030BD00BF887F0020CC1500201B
:10785000CC3A0020001000E0D34D621070B52B4CE4
:1078600094F8283182B023B9012084F8283102B07D
:1078700070BDD4F82451264A95F91030A96803EB5D
:10788000830302EB83030522ADF800208A07D3F8B7
:10789000CC0111D502236A4601A964F0F1F8AB6866
:1078A0009B071CD59DF8053003F0010383F0010010
:1078B00084F8283102B070BD6B6913B11A689B88D7
:1078C0005383144B14491A68144B4E68D200A3FB1F
:1078D000023292094B689B1B9A42FBD2DAE70D4BAE
:1078E0000D491A680D4B48684FF4FA7606FB02F210
:1078F000A3FB023292094B681B1A9A42FBD26B69B6
:10790000002BCFD01A689B881383CBE7887F002099
:10791000CC150020CC3A0020001000E0D34D6210BE
:107920002DE9F04782B060B9364D95F82831D5F889
:107930002C7173B900230120C5F82C3102B0BDE8C9
:10794000F087314B2F4D1F6895F828310744002BE5
:10795000F0D0DFF8BC802D4CDFF8B8A0DFF8B8908D
:10796000D5F8246196F9103003EB830308EB830309
:107970000522D3F8CC01B368ADF800209A072FD5C3
:1079800002236A4601A964F07BF8B3689B0712D50D
:107990009DF8053013F0010302D185F82831C9E7BD
:1079A000194B1B6801229F4285F82821D8D8002056
:1079B00002B0BDE8F087DAF8002061684FF4FA738E
:1079C00003FB02F2A9FB0232920963685B1A9A4236
:1079D000FBD27369002BDBD01A689B881383D7E72F
:1079E000736913B11A689B885383DAF800206168C1
:1079F000D200A9FB0232920963685B1A9A42FBD259
:107A0000BEE700BF887F002008360020001000E09D
:107A1000CC150020CC3A0020D34D621010B50020C8
:107A2000FFF77EFF00B910BD084C0620FFF7C2FE2D
:107A30000123C72084F82831FFF7BCFE044B1B68E4
:107A400003F5A4430833C4F82C3110BD887F00200F
:107A500008360020F0B5044689B000200E461546D1
:107A6000FFF75EFF10B9204609B0F0BD1D4F06209C
:107A7000FFF7A0FE012387F8283197F83021CDF8D1
:107A80000CD00223009300238DF804300293E2B15E
:107A9000CDE9066505930522230E8DF80130049289
:107AA0000DF10203220C1A70D7F824019C70220AEF
:107AB0005A700379022B10D00B4B1B682C440633F1
:107AC0002046C7F82C3109B0F0BDCDE905260422C7
:107AD00007950DF101030492E4E702A964F020F890
:107AE000EAE700BF887F00200836002070B5054611
:107AF00088B000200E461446FFF712FFE8B10322BB
:107B00000092164ACDF80CD092F830110596002359
:107B10008DF80430029391B9CDE9061404210DF1DA
:107B200001030491D2F824019D702A0C1A702A0ACC
:107B30005A700379022B0CD0204608B070BD290E74
:107B40008DF801100521CDE9063404910DF10203F1
:107B5000E8E702A963F0E4FF2046EEE7887F002013
:107B6000F0B5064683B00020FFF7DAFE08B903B08F
:107B7000F0BD324C0620FFF71DFE012294F8303193
:107B800084F82821D82100228DF80420D4F824512B
:107B90000091C6F307420BBB70BA8DF80120ADF817
:107BA0000200042395F91020254902EB820201EB23
:107BB0008202A968D2F8CC018A0714D56A4600214E
:107BC00063F05EFFAB689B0720D51E4B1B6803F577
:107BD0009C530833C4F82C3103B0F0BD30BACDF853
:107BE00001000523DEE76A6912B1116892884A83B1
:107BF000154A164E1168164A7768C900A2FB012182
:107C000089097268D21B9142FBD2D7E70E4B0F490C
:107C10001A680F4B48684FF4FA7606FB02F2A3FB92
:107C2000023292094B681B1A9A42FBD26B69002BF5
:107C3000CBD01A689B881383C7E700BF887F0020DA
:107C4000CC15002008360020CC3A0020001000E0BF
:107C5000D34D6210244B254A30B5D3F8344194F902
:107C60001030A16803EB830302EB830283B08DF82D
:107C70000700D2F8CC018A070AD501230DF10702CB
:107C8000002163F0FDFEA3689B0714D503B030BD4F
:107C9000636913B11A689B885383154B15491A6899
:107CA000154B4D68D200A3FB023292094B685B1B57
:107CB0009A42FBD2E1E70E4B0E491A680E4B4FF485
:107CC000FA7000FB02F2A3FB0232486892094B688B
:107CD0001B1A9A42FBD26369002BD7D01A689B8883
:107CE000138303B030BD00BF887F0020CC15002077
:107CF000CC3A0020001000E0D34D6210274B284AF8
:107D000030B5D3F8344194F9103003EB830383B0DA
:107D100002EB8302A3688DF804000025D2F8CC01A1
:107D20008DF8055049BA9A07ADF806100AD5042314
:107D30000DEB0302002163F0A3FEA3689B0714D59B
:107D400003B030BD636913B11A689B885383154B28
:107D500015491A68154B4D68D200A3FB02329209EF
:107D60004B685B1B9A42FBD2E1E70E4B0E491A6847
:107D70000E4B4FF4FA7000FB02F2A3FB023248688C
:107D800092094B681B1A9A42FBD26369002BD7D029
:107D90001A689B88138303B030BD00BF887F002022
:107DA000CC150020CC3A0020001000E0D34D62102A
:107DB00070B52D4D2D4AD5F8344194F9103003EBB0
:107DC000830302EB8303A26882B000204CF205011A
:107DD00092078DF80200ADF80010D3F8CC0119D548
:107DE00003236A4601A963F04BFEA3689B0724D5D1
:107DF00095F838319DF806203BB102F0010383F07D
:107E0000010085F8383102B070BD012085F83831A5
:107E100002B070BD636913B11A689B885383144B19
:107E200014491A68144B4E68D200A3FB023292091F
:107E30004B689B1B9A42FBD2D2E70D4B0D491A6847
:107E40000D4B48684FF4FA7606FB02F2A3FB0232B0
:107E500092094B681B1A9A42FBD26369002BC7D068
:107E60001A689B881383C3E7887F0020CC15002005
:107E7000CC3A0020001000E0D34D621070B55A4D8E
:107E80005A4E82B0FF20FFF7E5FE2C68012304F56F
:107E9000FA74C6F83C4186F8383103E02B681B1BA6
:107EA000002B06DAFFF784FF0028F7D00023C6F87E
:107EB0003C31D6F834414E4D94F91030A2684AF264
:107EC000010103EB830305EB8303ADF804100021EC
:107ED0008DF806109107D3F8CC0120D5032301AA11
:107EE000002163F0CDFDA3689A0743D594F91030C3
:107EF00003EB830305EB83034BF20102ADF804208F
:107F0000D3F8CC0118228DF80620032301AA002102
:107F100063F0B6FDA3689B0714D502B070BD63691A
:107F200013B11A689B885383324B33491A68334B19
:107F30004E68D200A3FB023292094B689B1B9A4207
:107F4000FBD2CBE72B4B2C491A682C4B4FF4FA7021
:107F500000FB02F2A3FB0232486892094B681B1A2D
:107F60009A42FBD26369002BD7D01A689B8813838F
:107F700002B070BD1F4B20481A68204B46684FF472
:107F8000FA7102FB01F1A3FB0131890943689B1BD4
:107F90009942FBD294F91030616903EB830305EB3E
:107FA0008305D5F8CC01B1B10B6889881983598351
:107FB0004BF20103ADF8043018238DF806300E495A
:107FC0000E4B4D68D200A3FB023292094B685B1B3B
:107FD0009A42FBD299E74BF20103ADF80430182323
:107FE0008DF80630EBE700BF08360020887F0020C0
:107FF000CC150020CC3A0020001000E0D34D6210D8
:1080000070B50B4D0B4E2C6801230444C6F83C415F
:1080100086F8383103E02B681B1B002B06DAFFF7CC
:10802000C7FE0028F7D00023C6F83C3170BD00BF62
:1080300008360020887F00202DE9F04FDFF8C4814A
:1080400098F840918BB007468B461646B9F1000F61
:1080500000F0A480D8F84451684CA8423AD1FFF708
:10806000A7FE48B92268D8F83C11521A002A06DA4D
:10807000FFF79EFE0028F5D00022C8F83C2106201C
:10808000FFF7E8FD0122ABB288F838210193C5F370
:108090000A0AB9F1000F4FD105E02268D8F83C1167
:1080A000521A002A03DAFFF783FE0028F5D08DF874
:1080B0000EA04FEA1A2AD8F83401CDF820B08DF876
:1080C0000DA00996022248E02268D8F83C11521A05
:1080D000002A06DAFFF76CFE0028F5D00022C8F867
:1080E0003C210620FFF7B6FD012288F83821D8F898
:1080F00048214FEAD22905E02268D8F83C11521AEB
:10810000002A03DAFFF754FE0028F5D04946102074
:10811000FFF7F4FD226802324FF00009C8F83C2155
:10812000012288F8409188F83821A1E72268D8F820
:108130003C11521A002A03DAFFF73AFE0028F5D064
:10814000019BCDF820B0D8F834018DF80EA0C3F310
:10815000022B8DF80DB0099684228DF80C20017940
:1081600000220492079203AA059202294FF003020B
:1081700006923ED022680232C8F83C2101223544E2
:1081800088F83821012288F84021C5F30A02C8F88E
:10819000445142B1B8190BB0BDE8F08FC8E95100A5
:1081A000164C054664E7D8F848214FEAD229144A0C
:1081B000C2F81C9205E02268D8F83C11521A002A35
:1081C00003DAFFF7F5FD0028F5D049461020FFF748
:1081D00095FD2268C8F848510232C8F83C210121B7
:1081E0000022B81988F8381188F840210BB0BDE892
:1081F000F08F04A963F094FCBCE700BF08360020B0
:10820000CC150020887F002070B5134C94F84031C5
:1082100003B970BDD4F84861104B114DF60AC3F88C
:108220001C6205E02B68D4F83C219B1A002B03DA72
:10823000FFF7BEFD0028F5D031461020FFF75EFDA8
:108240002B6801210022023384F83811C4F83C3134
:1082500084F8402170BD00BF887F0020CC1500202D
:1082600008360020F0B5314D314C83B0064605E0AC
:108270002B68D4F83C219B1A002B03DAFFF798FDFA
:108280000028F5D0D4F834712A4A06238DF8073037
:1082900097F9103003EB830302EB8303D3F8CC018F
:1082A000BB689A0715D501230DF10702002163F081
:1082B000E7FBBB689B0721D5F10AD820FFF71EFD1D
:1082C0002B6801220F3384F83821C4F83C3103B005
:1082D000F0BD7B6913B11A689B885383164B17490D
:1082E0001A68174BD1F804C0D200A3FB02329209DE
:1082F0004B68A3EB0C039A42FAD2D4E70E4B0F491A
:108300001A680F4B4FF4FA7000FB02F2A3FB023223
:10831000486892094B681B1A9A42FBD27B69002B72
:10832000CAD01A689B881383C6E700BF08360020AE
:10833000887F0020CC150020CC3A0020001000E0FF
:10834000D34D62102DE9F04F5D4DB5F8643083B028
:10835000002B55D0D5F834715A4EDFF874A15A4C21
:10836000DFF870B14FF000094FEA494805E0336883
:10837000D5F83C219B1A002B03DAFFF719FD0028E2
:10838000F5D097F91030BA6803EB830306210AEBA6
:1083900083038DF804109107D3F8CC017ED5012317
:1083A00001AA002163F06CFBBB684FEAD8209A0752
:1083B000C8F3C748C0B23CD5D823ADF8043097F90C
:1083C00010308DF8070003EB83030AEB83038DF86D
:1083D0000680D3F8CC0104230DEB0302002163F0E7
:1083E0004FFBBB689B070ED501213368B5F86420AD
:1083F00085F8381189440F334A45C5F83C31B3D864
:1084000003B0BDE8F08FDBF8003061684FF4FA721A
:1084100003FB02F22D4BA3FB0232920963685B1A45
:108420009A42FBD27B69002BDED01A689B881383AB
:10843000DAE7DBF80020254BD4F804C04FF4FA71DA
:1084400002FB01F1A3FB013189096368A3EB0C0373
:108450009942FAD24FF0000368F3070360F30F2349
:10846000ADF8063097F91030796903EB83030AEB16
:108470008303D3F8CC0119B10B6889881983598318
:10848000D823ADF80430114B6168D200A3FB02324F
:10849000920963685B1A9A42FBD29CE77B6913B12D
:1084A0001A689B885383DBF800306168DA00074B59
:1084B000A3FB0232920963685B1A9A42FBD26EE711
:1084C000887F002008360020001000E0D34D6210A5
:1084D000CC150020CC3A00202DE9F04FDFF8AC811C
:1084E000D8F81C32B3EBD02F8BB00546894617461F
:1084F00061D1614C614ECDF81C90D6F834910023C7
:10850000C5F30A05C5F5006003228DF80F3004930A
:10851000089399F804308DF80C20B84203AAB4BF30
:1085200087B2BFB28DF80E5005922D0A0422022B9D
:108530008DF80D500997069200F099802568012367
:108540000235C6F83C5186F8383103E023685B1BDE
:10855000002B2CDAFFF72CFC0028F7D04CF2050397
:10856000ADF8043099F9103003EB830308EB83086E
:10857000D9F80830D8F8CC010022C6F83C218DF893
:1085800006209A075FD5032301AA02A963F078FAAF
:10859000D9F808309B073ED59DF80A30C3F3011384
:1085A000013B022B33D938460BB0BDE8F08F0020D9
:1085B0000BB0BDE8F08F304C304E4FEAD02A05E0CA
:1085C0002368D6F83C219B1A002BF0DAFFF7F0FB6A
:1085D0000028F5D04FF0FF3351461320C8F81C3265
:1085E000FFF78CFB012386F83831236803F1020B77
:1085F000C6F83CB104E02368A3EB0B03002BD6DAEA
:10860000FFF7D6FB0028F6D0C8F81CA273E7FFF7E7
:1086100035FC3846C8E71A4B1A491A681A4B48689D
:108620004FF4FA7404FB02F2A3FB023292094B6886
:108630001B1A9A42FBD2D9F81430002BACD01A681E
:108640009B881383A8E7D9F8143013B11A689B8864
:1086500053830B4B0B491A680B4B4C68D200A3FB9E
:10866000023292094B681B1B9A42FBD28BE704A98A
:10867000484663F055FA61E708360020887F0020FD
:10868000CC3A0020001000E0D34D6210CC15002041
:108690002DE9F0410C4E356873691D4011D0DFF8AB
:1086A0002C800127B5FA85F4C4F11F0408EB84037C
:1086B00007FA04F4D3F84C0103689847A5437461A2
:1086C000F0D1BDE8F08100BF003C0140887F002070
:1086D00070B583681C686379DB0748D5A37994F883
:1086E0005C22E06B03F001010E461ABB94F85F3286
:1086F000012B3DD0002B3FD194F85E3294F85DE21F
:108700009E450ED9B4F86622012505FA03FC013313
:1087100042EA0C025FFA83FCE64592B2F5D8A4F86F
:108720006622012384F85F3286EA0301BDE87040C7
:108730005FF07CBD43681A68D36AC3F34E0353628B
:1087400094F86D32012B07D094F8613223B1B4F85C
:1087500068320133A4F8683286F001015FF066FDEB
:1087600000224FF08073A4F86622C4F85C3270BD1A
:1087700094F85D3284F85E32002384F85F32BDE8FD
:1087800070405FF053BD00BFF0B52DED028B4D4E34
:1087900096F8AC31022B83B00D46144619D0DFEDAC
:1087A0004A7A7DB19FED497A9FED496ADFED496ACA
:1087B00067EEA77A67EE877A87EE867A77EE267A73
:1087C000C5ED007A0CB1444B236003B0BDEC028BC5
:1087D000F0BD424B96F808229B6803F002032ABBC7
:1087E0002BB3B6F9383207EE903AB6F93632F8EED6
:1087F000E77A06EE903A27EEA77AF8EEE66AB6F93F
:108800003A32A6EEA67A07EE903AF8EEE77AA7EEAD
:10881000A77AB5EEC07AF1EE10FAC0DBF1EEC77AB6
:10882000F4EE677AF1EE10FABBD7B8E723B9D6F8C1
:108830005032D3ED347AB4E7294F0DF106002DF014
:10884000BFFCBDF80630D7F8EC23DFED265ADFED8C
:10885000266A9FED267A9B1A07EE903AF8EEE77AA1
:10886000B0EE408A87EEA56AA6EE267AFDEEC77ABC
:10887000B0EE470A17EE903A2033402B1ED8FCF793
:108880003BFF1B4B797CD6ED857AA3F12C02184671
:10889000443B002918BF134693ED057AD0ED006ADA
:1088A00077EE877AE8EE406A27EEA77AA6EEA67AF8
:1088B000B5EEC07AF1EE10FAB0DA70E79FED020A79
:1088C000DFE700BF887F002000000000CDCC9C3F88
:1088D00000409C4682E6C547331390439800001041
:1088E000389300200000C84235FA8E3CDB0FC93FA8
:1088F0003897002010B50B4B82B053F830400191EF
:108900006CB107EE901A94ED047A94ED030AF8EE38
:10891000E77AA7EE870A64F0A9FBA368186002B0A3
:1089200010BD00BF40410020174A02EB8000D0F884
:10893000540228B3154B00EB400003EB800393F97E
:1089400001C0BCF1FF3F1CD0587AC8B110B56244D9
:108950008C200F4C197A92F864E20023142200FB59
:108960000CFC0CEB0100013A34F81000714413FACE
:1089700080F3F6D1074AA2FB0320C0F30F1010BD0D
:1089800070470020704700BF887F0020103A002009
:10899000C8360020CDCCCCCC30B5032083B00D46FA
:1089A0001446FFF7C1FF01909DB107EE900A9FEDBD
:1089B0000B7AF8EE677AF0EE006A67EE877AB8EE27
:1089C000047AA7EEA67ADFED067A67EE277AC5ED80
:1089D000007A0CB1034B236003B030BD6740533ABB
:1089E00000007A4433139043074B10B403F1100195
:1089F000002453F8042B824208BF43F8044C8B42F6
:108A0000F7D15DF8044B7047DC81002070B5104B46
:108A1000104CA3421AD2054602E00C33A34215D2F1
:108A200093F805C08C45F8D193F804C0AC4501D04B
:108A3000002DF2D1D8799042EFD1186890F804E077
:108A4000E645EAD106689E42E7D170BD002070BDC0
:108A5000BC900808609208080379022B00D0704788
:108A600010B490F910201D481D4C83B002EB820217
:108A70000831694400EB82020094D2F8CC2111F84D
:108A8000084C18498A4225D0A1F578418A4223D062
:108A900001F580618A4219D1118821F04001090451
:108AA00003EB8303090C118000EB83001388D0F8DB
:108AB000D81123F0380331F824101B041B0C0B438E
:108AC000138013889BB243F04003138003B05DF81A
:108AD000044B70470023DFE70123DDE7CC150020BE
:108AE000000102030030014010B50446C06900B126
:108AF00010BD09211420FDF72FF8E06110BD00BF63
:108B0000034690F910002DE9F041244C00EB800061
:108B100016469A6804EB80009207D0F8CC8109D5FC
:108B2000404663F093F83146404663F08FF80120E9
:108B3000BDE8F0815D69084615B12B68AA885A83A3
:108B4000174B184F1C68184B7A684FEAC40CA3FBEC
:108B50000C3C4FEA9C1C7B689B1A9C45FBD201464F
:108B6000404663F073F83146404663F06FF80E4BB1
:108B700078680C494FF4FA7204FB02F2A3FB02324C
:108B800092094B681B1A9A42FBD2002DCFD02B685A
:108B9000AA881A830120BDE8F08100BFCC1500200F
:108BA000CC3A0020001000E0D34D621010B50379DC
:108BB000012B84B08E460DD0022B02D0002004B0D1
:108BC00010BD8368DB0758BF01F07F0104B0BDE82A
:108BD000104095E7144682688DF80F4002F00102BC
:108BE00001920DF10F020092417C90F91000724643
:108BF000FAF720FD04B010BD10B504460022212173
:108C00000068FFF7D3FF2068FC222021FFF7CEFF8A
:108C1000206840222421FFF7C9FF20680C2223216D
:108C2000FFF7C4FF206800222221FFF7BFFF0120C9
:108C300010BD00BF10B5044694220B210068FFF759
:108C4000B5FF206871220121FFF7B0FF20680022E4
:108C50000421FFF7ABFF2068C8220521FFF7A6FF1C
:108C6000206800220621FFF7A1FF2068C822072103
:108C7000FFF79CFF206800220821FFF797FF20687C
:108C8000C8220921FFF792FF012010BD00B500683E
:108C90000379012B85B012D0022B03D0012005B03F
:108CA0005DF804FB8368DB074FF031024CBFF42111
:108CB0007421FFF725FF012005B05DF804FB8268F1
:108CC00090F910C0417C02F0010201920DF10F02F7
:108CD00000926046F4224FF0310C8DF80FC0FAF785
:108CE000A9FC012005B05DF804FB00BF10B50446E7
:108CF00000680379012B84B011D0022B02D0002030
:108D000004B010BD01220B21FFF7FAFE0028F6D0B7
:108D100020681D22092104B0BDE8104046E78268A2
:108D200090F910C0417C8DF80F3002F001020192E1
:108D30000DF10F02009260460B22FAF77BFCE5E78B
:108D40002DE9F04105461F4695F91030244803EB04
:108D5000830300EB8300AB68D0F8CC8116469A07FA
:108D60000ED5404662F072FF3B4632460021404637
:108D700062F086FEAB689B0718D50120BDE8F08144
:108D80006B6913B11A689B885383164B164A1B688C
:108D90004FEAC30E154BA2FB0E2E5A684FEA9E1ED9
:108DA0005C68A4EB020CE645FAD2DAE70D4B0F49FA
:108DB0001A680D4B4FF4FA7000FB02F2A3FB02326B
:108DC000486892094B681B1A9A42FBD26B69002BC8
:108DD000D3D01A689B8813830120BDE8F08100BFBF
:108DE000CC150020CC3A0020D34D6210001000E0DA
:108DF00030B50579012D83B08E460DD0022D02D0FD
:108E0000002003B030BD8468E40758BF41F0800102
:108E100003B0BDE8304093E714468268009402F046
:108E20000102417C90F9100001927246FAF702FCAF
:108E300003B030BD10B5164C84F86912017984F87E
:108E40006A2201294FF0000282B084F8682210D013
:108E5000022903D06FF00C0002B010BD032304F50B
:108E60001A72FF21FFF76CFF0028F3D0002002B038
:108E700010BD8268417C90F9100004F51A7402F06C
:108E80000102CDE900420323FF22FAF7D3FBEBE70F
:108E9000887F002000680379012B0AD0022B00D0C4
:108EA000704783680D4A13F0010314D00023512149
:108EB00046E700B58368094A417C90F9100083B009
:108EC00003F00103CDE9002300235122FAF7B2FB9E
:108ED00003B05DF804FBD12132E700BFF08200202F
:108EE0002DE9F04105461F4695F91030244803EB63
:108EF000830300EB8300AB68D0F8CC8116469A0759
:108F00000ED5404662F0A2FE3B4600223146404666
:108F100062F0B6FDAB689B0718D50120BDE8F08173
:108F20006B6913B11A689B885383164B164A1B68EA
:108F30004FEAC30E154BA2FB0E2E5A684FEA9E1E37
:108F40005C68A4EB020CE645FAD2DAE70D4B0F4958
:108F50001A680D4B4FF4FA7000FB02F2A3FB0232C9
:108F6000486892094B681B1A9A42FBD26B69002B26
:108F7000D3D01A689B8813830120BDE8F08100BF1D
:108F8000CC150020CC3A0020D34D6210001000E038
:108F900030B50579012D83B08E460DD0022D02D05B
:108FA000002003B030BD8468E40758BF41F0800161
:108FB00003B0BDE8304093E714468268009402F0A5
:108FC0000102417C90F9100001927246FAF742FDCD
:108FD00003B030BD10B504460068037982B0022B9F
:108FE0000CBF4321032106236A46FFF7D1FF68B176
:108FF000BDF80010BDF80220BDF8043049BA52BADD
:109000005BBAE1866287238702B010BDC4F83600E0
:10901000608702B010BD00BF70B50668F56982B008
:109020000446002D59D000232B7004230DEB0302BE
:109030003046FF21FFF7ACFF10B9002002B070BD31
:10904000206804236A46FF21FFF7A2FF0028F4D01E
:109050009DF804309B09023B012BEED9BDF804308A
:10906000BDF80620BDF80010BDF802605BBA43F6FB
:10907000FF74C3F30D03A342DFD0002BDDD052BA3F
:10908000C2F34A1240F2FF7C6245D6D0002AD4D007
:1090900049BAC1F30D01A142CFD00029CDD076BA93
:1090A000C6F34A166645C8D0002EC6D05C1A002CFE
:1090B000B8BF6442FF2CC0DC941B002CB8BF6442D4
:1090C000FF2CBADC0B445B1032445210C5F805305B
:1090D0000123C5F801202B70B0E709211420FCF70B
:1090E0003BFDF061054626689DE700BF70B5066848
:1090F000F46982B0F4B10023237004230DEB030262
:10910000FF213046FFF744FF10B39DF804309B0960
:1091100019D1BDF80420BDF8063052BA5BBA92B23C
:10912000C3F34A1301212170C4F80520C4F80130AB
:1091300002B070BD054609211420FCF70DFDF06159
:1091400004462E68D7E7044A04210320FCF790FC6C
:10915000002002B070BD00BF741A08082DE9F0416C
:10916000104C04F51A7884F869121746002502237A
:109170004246FF21064684F86852FFF739FE68B17F
:10918000424630460223FF21FFF702FF30B1B4F818
:1091900068325BBA28463B80BDE8F0816FF00C0076
:1091A000FAE700BF887F002030B5194D95F81A31D5
:1091B00083B00BB903B030BD04460DF10501006862
:1091C00060F088FB9DF8053073B92068114A0121D1
:1091D0004FF4064485F86A120323FF21A5F868427C
:1091E00003B0BDE8304003E60DF106029621206889
:1091F000FFF7B4FF084ABDF806300849A2FB032375
:10920000DB080122C1F8083185F81B21DDE700BF2A
:10921000887F0020F0810020CDCCCCCCCC15002064
:1092200010B5044600680379012B84B02DD0022BC1
:1092300001D0002027E0836813F0010F02AA4FF04D
:10924000060314BF1F219F21FFF74AFE0028F0D01C
:10925000BDF80810BDF80A20BDF80C30C9BA07EEF9
:10926000901AD2BAF8EEE76A07EE902ADBBAB8EEA7
:10927000E77A07EE903AF8EEE77AC4ED046A84EDF7
:10928000057AC4ED067A04B010BD8368417C90F97C
:10929000100003F00103019302AB00931F22062389
:1092A000FAF7D8FBD2E700BF10B50446006803798F
:1092B000012B84B02DD0022B01D0002027E0836841
:1092C00013F0010F02AA4FF0060314BF2521A521B8
:1092D000FFF706FE0028F0D0BDF80810BDF80A2000
:1092E000BDF80C30C9BA07EE901AD2BAF8EEE76AA8
:1092F00007EE902ADBBAB8EEE77A07EE903AF8EE7E
:10930000E77AC4ED076A84ED087AC4ED097A04B0FF
:1093100010BD8368417C90F9100003F001030193B4
:1093200002AB009325220623FAF794FBD2E700BF95
:1093300000B500680379012B85B02FD0022B08D02F
:109340001D49D1E9DA3200200A600B6205B05DF8F0
:1093500004FB062302AAF721FFF7C2FD0028EFD085
:109360009DF809309DF808C09DF80C209DF80A1062
:109370009DF80BE01B0143EA0C3312019DF80DC070
:1093800043EA111342EA0E320B4942EA1C12C1E9C8
:10939000DA320A600B6205B05DF804FB8368417C39
:1093A00090F9100002AA03F00103CDE9002306237F
:1093B000F722FAF74FFBD1E7887F002010B504466B
:1093C00000680379012B84B042D0022B07D0002221
:1093D00013461046C4F83620638704B010BD836876
:1093E00013F0010F02AA4FF0060314BF11219121BF
:1093F000FFF776FD0028EAD0BDF9083006EE903A76
:10940000BDF90A30F8EEE66A07EE103ABDF90C3005
:10941000B7EE086A07EE903A66EE866AB8EEC77A4B
:10942000FDEEE66A27EE067AF8EEE77A16EE903A57
:1094300067EE867ABDEEC77AFDEEE77AE38617EE31
:10944000103A238717EE903A1BB2638704B010BD21
:109450008368417C90F9100003F00103019302AB93
:10946000009311220623FAF7F5FAC3E710B5044674
:1094700000230068C4F8363063870379012B84B079
:1094800022D0022B01D000201CE0836813F0010FD2
:1094900002AA4FF0060314BF03218321FFF720FD2A
:1094A0000028F0D0BDF90A30BDF80810BDF80C2036
:1094B0005B4201EB410103EB430302EB4202E18615
:1094C0002387628704B010BD8368417C90F9100047
:1094D00003F00103019302AB009303220623FAF782
:1094E000B9FADDE710B504464FF0000C0068C4F887
:1094F00036C0A4F83AC00379012B84B018D0022BEF
:1095000001D0002012E0836813F0010F02AA4FF08F
:10951000060314BF61468021FFF7E2FC0028F0D06B
:10952000029ABDF80C30C4F83620638704B010BD31
:10953000836890F910E0417C03F00103019302ABD2
:109540000093624606237046FAF784FAE6E700BF06
:1095500010B584B00023044600680293CDF80B30A8
:109560000279012A1ED0022A19D1836813F0010F53
:1095700002AA4FF0070314BF4E21CE21FFF7B0FC23
:10958000BDF80910BDF80B20BDF80D30C9BAD2BA2C
:10959000DBBA0120E1862287638704B010BD1A463A
:1095A0001946F6E7836890F910C0417C02AA03F0DF
:1095B0000103009201934E2207236046FAF74AFA0C
:1095C000DEE700BF00B500680379012B85B00DD040
:1095D000022B07D1012303AAFF21FFF781FC05B06D
:1095E0005DF804FB002005B05DF804FB8268417C57
:1095F00090F9100002F00102019203AA0092FF22EA
:10960000FAF728FA05B05DF804FB00BF30B5044650
:1096100000680379012B85B02DD0022B0ED0224B90
:109620006FF00102C3F80C212049214AD1F87033B0
:1096300015683233AB422CD305B030BD826812F0CE
:10964000010F18BF512103AA08BFD121FFF748FC21
:109650000028E4D0BDF80C30134A5BBA9BB2C2F8C4
:109660000C31D2F80C31B3F5C87FDDDD4FF0FF339C
:10967000C2F80C31D8E78368417C90F9100003F000
:109680000103019303AB009351220223FAF7E2F99D
:10969000DEE701F55A72C1F87053206800235121AA
:1096A000FFF7A6FB05B030BDCC150020887F002059
:1096B0000836002000B500680379012B85B02DD055
:1096C000022B24D1826812F0010F18BF002103AAD7
:1096D00008BF8021FFF704FC1B4B83F8200198B1E1
:1096E000BDF80C305BBA9BB2B3F5FA6F24D2174ABF
:1096F0001749A2FB0323DB0807EE903AF8EEE77A5E
:10970000FDEEE77AC1ED447A05B05DF804FB0E4B3F
:10971000002283F8202105B05DF804FB8368417CBA
:1097200090F9100003AA03F00103CDE900230223FE
:109730000022FAF78FF9CFE7054B4FF0FF32C3F85D
:10974000102105B05DF804FB887F0020CDCCCCCC87
:10975000CC15002010B500680379012B84B00C46AD
:109760001FD0022B02D0002004B010BD826812F07E
:10977000010F18BF002103AA08BF8021FFF7B0FB2B
:109780000028F0D05CB19DF80D309DF90C20DB096C
:1097900003EB830302EB820203EB4203238004B05A
:1097A00010BD8368417C90F9100003F00103019320
:1097B00003AB009300220223FAF74CF9E0E700BF65
:1097C00070B50446234894F9103003EB830300EB93
:1097D0008300A368D0F8CC6115469A070DD53046B2
:1097E00062F034FA012300222946304662F048F93B
:1097F000A3689B0716D5012070BD636913B11A6871
:109800009B885383144B154A1B6850684FEAC30C5E
:10981000134BA3FB0C3C4FEA9C1C53681B1A9C4542
:10982000FBD2DCE70C4B0D491A680D4B4FF4FA7074
:1098300000FB02F2A3FB0232486892094B681B1A34
:109840009A42FBD26369002BD5D01A689B88138398
:10985000012070BDCC150020CC3A0020001000E0A3
:10986000D34D621010B50379012B82B08E460DD016
:10987000022B02D0002002B010BD8368DB0758BF66
:1098800041F0800102B0BDE8104099E714468268BB
:10989000009402F00102417C90F91000019272469E
:1098A000FAF7D8F802B010BDF0B583B015460DF147
:1098B00007021C4606460F46FFF7D4FF9DF8072017
:1098C00005EA0203A34201D103B0F0BD22EA05027A
:1098D00022433946304603B0BDE8F040FFF766B991
:1098E00010B582B004466A4600680821FFF7BAFF47
:1098F0009DF80030DB0602D4002002B010BD2068C5
:1099000006236A460021FFF743FB0028F4D09DF8A8
:1099100001209DF800109DF802309FED386A120278
:1099200002EB01421344140248BF03F17F4307EEE8
:10993000903AF8EEE77A9DF804109DF803409DF800
:1099400005202F4BC7EE866A090201EB04410A4449
:10995000090248BF02F17F4207EE902AB3F938208E
:1099600007EE102AB3F93420F8EEE77A05EE102A54
:1099700087EE864AB3F93020B8EEC77AB8EEC55AFA
:1099800093ED0B6AD3ED0A7AA6EE875AF8EEC65A23
:1099900004EE902AE5EE265AB3F93220F8EEE77A83
:1099A00006EE102AB3F93620E5EEA67A03EE902AE9
:1099B000B3F92620F8EEE44AF8EEE33A07EE102A6F
:1099C000B8EEC66AB3F92420A6EEA36AE4EE247AC0
:1099D00005EE902AB8EEC77A66EE846AF8EEE55A8C
:1099E00027EE047AB6EE005AA5EE857AE6EE867A80
:1099F00083ED107AC3ED0F7A02B010BD00007848F5
:109A0000887F002030B5002385B00446C0F836308A
:109A100043870DF1070200680221FFF723FF18B109
:109A20009DF80730DB0703D40025284605B030BD7C
:109A3000062302AA03212068FFF7AAFA20680DF185
:109A400007020921FFF70EFF05460028ECD09DF81C
:109A5000073013F00C0FE7D1BDF80820BDF80C302B
:109A6000BDF80A102068C2EB8232C3EB83339B003F
:109A700092008900E2862187638701220A21FFF78D
:109A800095F8284605B030BDF0B54B4D95F8183126
:109A900083B03BB195F87463012E044639D0022E91
:109AA00057D00EB103B0F0BD012280210068FFF74E
:109AB0007DF820680122FF21FFF778F83246314611
:109AC0002068FFF773F895F8752320689121FFF758
:109AD0006DF8314620680122FFF768F832462068A9
:109AE000FF21FFF763F8324620688021FFF75EF818
:109AF000314620680122FFF759F8304B30491A6887
:109B000081F800010123C5F8782385F8743303B088
:109B1000F0BD01AA00682A4F0021FFF7A3FE9DF8BF
:109B2000043087F80001DA073DD5D5F87C33002BE7
:109B3000B8D0224AD5F87813126892B2521A9342DA
:109B4000B0D24FF0FF320023C7F8042185F87433F8
:109B5000A8E700681A4F01AA1321FFF783FE9DF8BA
:109B6000043087F800015B07DFD02068334601AA84
:109B70001E21FFF70DFABDF80430206801220B21E9
:109B80005CBAFFF713F80F4B87F80001A4B2A3FBF0
:109B90000434E40801220023C7F8044185F81921A0
:109BA00085F874337EE7054A02231268C5F87823E6
:109BB00085F8743376E700BF887F002008360020E0
:109BC000CC150020CDCCCCCC30B504460068037950
:109BD000012B85B062D0022B03D00025284605B0AA
:109BE00030BD826802AD12F0010F18BF19462A4637
:109BF00008BF8221FFF7E4FD0028EED09DF8083071
:109C0000DA07EAD52A46206807230321FFF7C0F9BF
:109C100005460028E1D0206811220A21FEF7C6FF80
:109C20009DF80E301B07D8D42A49BDF80830B1F88A
:109C3000802313FB02F3284A93423FDBB3F5000F66
:109C40003ADA002BB8BFFF331B125B421BB2BDF8E0
:109C50000A20E386B1F8823312FB03F31E4A9342D3
:109C600030DBB3F5000F31DA002BB8BFFF3343F31D
:109C70000F22BDF80C30B1F884132287164A13FB6B
:109C800001F393421CDBB3F5000F1DDA002BB8BFC4
:109C9000FF331B125B421BB263879FE7826890F918
:109CA00010C0417C02F0010202AD019200956046B5
:109CB0000222F9F7CFFE9FE7084BC8E7084BC6E73B
:109CC000074BE9E7064AD4E7044BE5E747F6FF729E
:109CD000CFE700BF887F002001FF7FFF0180FFFFEB
:109CE0000080FFFF10B5044686B0006800238DF8A1
:109CF0000F300379012B31D0022B02D0002006B0A7
:109D000010BD8368D9070DF10F024CBF2721A72191
:109D1000FFF756FD0028F1D09DF80F301B07EDD559
:109D20002068062304AA2821FFF732F928B3BDF9D9
:109D30001030BDF91220002BB8BF03339B10E3860F
:109D4000BDF91430002AB8BF0332002BB8BF03336B
:109D500092109B102287638706B010BD826890F92D
:109D600010C0417C02F0010201920DF10F0200923D
:109D700060462722F9F76EFECCE7C4F8360060870C
:109D80000020BCE730B504464FF0000C0068C4F872
:109D900036C0A4F83AC00379012B87B02AD0022B31
:109DA00002D0002007B030BD8368D9070DF10F0243
:109DB0004CBF61468021FFF703FD0028F1D09DF8DC
:109DC0000F301B07EDD52068062304AA0121FFF7F9
:109DD000DFF80028E5D0BDF81430BDF81010BDF84C
:109DE00012205BBA49BA52BA5B42E1862287638786
:109DF00007B030BD8568417C90F9100005F0010581
:109E000001950DF10F0562460095F9F723FED4E7A1
:109E100010B5044600230068C4F836306387037920
:109E2000012B86B023D0022B02D0002006B010BD3B
:109E30008368D9070DF10F024CBF06218621FFF779
:109E4000BFFC0028F1D09DF80F305B07EDD52068EE
:109E5000062304AA0021FFF79BF80028E5D0049A06
:109E6000BDF81430C4F83620638706B010BD826890
:109E700090F910C0417C02F0010201920DF10F0235
:109E8000009260460622F9F7E5FDDAE710B50446D0
:109E900000230068C4F8363063870379012B86B04D
:109EA00012D0022B0DD18368DB070DF10B024CBFE2
:109EB0003421B421FFF784FC18B19DF90B30002B3D
:109EC00011DB002006B010BD826890F910C0417C03
:109ED00002F0010201920DF10B0200926046342261
:109EE000F9F7B8FDE8E72068092303AA2421FFF762
:109EF0004FF80028E5D09DF810209DF80F109DF830
:109F00001330120442EA0162C2F30F429DF81210AC
:109F100022871B049DF80D2043EA01639DF80C1075
:109F2000120442EA0162C2F30F42C3F30F43E28616
:109F3000638706B010BD00BF2DE9F041DFF8BC809B
:109F40002C4E2D4D41F0010284B000210446FEF755
:109F50002DFED8F80070C6F8787319E0022B3FD1B7
:109F6000A368DB070DF10F024FF0130120465EBF1F
:109F70000DF10F0293212046FFF722FC9DF80F30D0
:109F800085F8000113F0070319D1D6F87C234ABBEA
:109F90002379012BE2D1A268617C94F9100002F0D0
:109FA000010201920DF10F0200921322F9F752FD06
:109FB0009DF80F3085F8000113F00703E5D001226A
:109FC0000B212046FEF7F2FD002211462046FEF747
:109FD000EDFD012385F80001184604B0BDE8F081CD
:109FE0000020CBE7D8F8001089B2C91B8A42CFD233
:109FF000F2E700BF887F0020CC1500200836002043
:10A0000010B50368DA6B82B0044612B1904740B1D4
:10A0100023685B6B1BB1214601A8984718B9FF2341
:10A02000E38202B010BDBDF80630013B9BB2F7E7FA
:10A03000F0B5044683B018460D4616461F466AF032
:10A040005FFC2844D4F800C0A073E67320460024C7
:10A050000094DCF814403B4632462946A04703B042
:10A06000F0BD00BF38B58B68016004460D469847C7
:10A0700000230B4A226123752B6B13B120469847AE
:10A080002075084B93F888331BB1237D23F001031F
:10A0900023750023E3822046BDE83840B0E700BFC7
:10A0A0000001FF00887F002010B5154BD3F88C43CA
:10A0B00084B084B12379012B10D0022B0BD1A1687D
:10A0C00011F00101024618BF8021204604B0BDE80E
:10A0D0001040FEF715BD002004B010BDA268617CE1
:10A0E0008DF80F0002F0010294F910000DF10F0439
:10A0F000CDE900428022F9F79DFA04B010BD00BFFF
:10A10000887F0020F0B5294BD3F88C5385B09DB1E2
:10A11000B02280212846FEF749FD402280212846B2
:10A12000FEF744FD002280212846FEF73FFD102265
:10A1300080212846FEF73AFD4FF480642DB9013C9A
:10A14000A4B2002CFBD105B0F0BD00270DF10F0625
:10A150002B79012B08D0022B04F1FF3217D094B2D7
:10A16000002CF0D0012BF6D1AA6895F91000697C7B
:10A170008DF80F7002F00102013CCDE90062A4B23B
:10A180004022F9F757FA002CE2D105B0F0BDAA68D9
:10A19000013C12F0010218BF002240212846A4B25F
:10A1A000FEF7AEFC002CD3D105B0F0BD887F0020B7
:10A1B0000B4B10B5D3F88C438CB15038C2B2802110
:10A1C0002046FEF7F3FC002280212046FEF7EEFC3D
:10A1D00020461022BDE810408021FEF7E7BC10BDEC
:10A1E000887F0020F0B5264B264CD3F88C532038BE
:10A1F00000EB8000661D85B00444064425B9013497
:10A20000A642FCD105B0F0BD0DF10F072B792278E5
:10A21000012B1BD0022B0AD00134A642F7D1002219
:10A220004021284605B0BDE8F040FEF7BFBCAB6852
:10A23000DB074FF04001284619D50134FEF760FCDA
:10A24000A642E3D1002DEAD105B0F0BD8DF80F2074
:10A25000AA6895F91000697C02F00102CDE900724C
:10A2600001344022F9F7E6F9B442CFD1D7E70134FF
:10A27000FEF746FCB442C9D1002DE5D0CFE700BFC0
:10A28000887F002050700708F0B5754BD3F88C53C9
:10A2900085B0002D00F09680D42280212846FEF75C
:10A2A00085FC802211462846FEF780FCA8228021EA
:10A2B0002846FEF77BFC3F2280212846FEF776FCED
:10A2C000D32280212846FEF771FC002280212846F7
:10A2D000FEF76CFC402280212846FEF767FC8D22A9
:10A2E00080212846FEF762FC142280212846FEF7D2
:10A2F0005DFCA12280212846FEF758FCC82280215F
:10A300002846FEF753FCDA2280212846FEF74EFC51
:10A31000122280212846FEF749FC8122802128460E
:10A32000FEF744FCCF2280212846FEF73FFCD922CD
:10A3300080212846FEF73AFCF12280212846FEF7CC
:10A3400035FCDB2280212846FEF730FC40228021AC
:10A350002846FEF72BFCA42280212846FEF726FC87
:10A36000A62280212846FEF721FCAF228021284624
:10A37000FEF71CFCA62280212846FEF717FCAE2221
:10A3800080212846FEF712FC202280212846FEF775
:10A390000DFC002280212846FEF708FCB022802117
:10A3A0002846FEF703FC402280212846FEF7FEFBEC
:10A3B000002280212846FEF7F9FB10228021284642
:10A3C000FEF7F4FB4FF4806435B9013CA4B2002CD5
:10A3D000FBD1012005B0F0BD00270DF10F062B7950
:10A3E000012B2AD0022B04F1FF3214D094B2002C9E
:10A3F000F6D1812280212846FEF7D8FBC822802191
:10A400002846FEF7D3FBAF2280212846FEF7CEFB7D
:10A41000012005B0F0BDAA68013C12F0010218BF8E
:10A42000002240212846A4B2FEF76AFB002CD6D1B8
:10A43000002DDED1012005B0F0BDAA6895F910000D
:10A44000697C8DF80F7002F00102013CCDE90062D9
:10A45000A4B24022F9F7EEF8002CC0D1C9E700BF42
:10A46000887F0020FEF714B9FEF712B9FEF710B985
:10A47000FEF70EB9FEF70CB9FEF70AB938B52B4C4A
:10A480002B483622002168F083F9D4F820320020CE
:10A49000984728B9D4F844329847012108B938BD03
:10A4A000002124204A42234B234D024000FB01445B
:10A4B0001344C5F8C833D4F840229047836853B397
:10A4C00005F5647C04886246614600230878032809
:10A4D00001F1060121D00133092BF7D1601E80B2B2
:10A4E00000231178022902F1060209D00133092B59
:10A4F000F7D1D5F8CC33082B0DD05A1CC5F8CC2396
:10A50000062202FB03CC022200238CF80020ACF8C8
:10A510000230ACF80400012038BD062101FB0353D2
:10A52000B3F89203013880B2DAE700BFCC150020FF
:10A5300018830020EC170020887F0020F0B170B550
:10A5400006680F4B06F13F4202F57E0203EB9223B1
:10A550000C4682B0054693F8B4025DF01DFF620917
:10A56000C4F30013A9883046CDE90032C4F3810357
:10A5700004F0030261F044F802B070BD704700BF00
:10A580004070070838B50409013C042C1CD8104D54
:10A5900005EB440200F00F03B2F8BC0240FA03F2EC
:10A5A00012F0010212D0012202FA03F3013B18401B
:10A5B00025446BF01DF995F8C832064A184400EBA3
:10A5C000400002EB800038BD002038BD104638BD89
:10A5D00040700708002A002010B503681A79022A83
:10A5E000044603D000232371236010BD987AFFF73F
:10A5F000C9FF0028F6D040F61A610022C18002721D
:10A600002021FFF79BFF00232371236010BD00BFB3
:10A61000F0B50668194B144606F13F4202F57E027A
:10A6200003EB9223074683B093F8B4020D465DF026
:10A63000B3FEB988B1FA81F3C3F11F03C3F3CC02AF
:10A6400006EB820203F0070330469B00166A0F27D1
:10A650009C4007FA03F326EA03031362136A1C43C0
:10A660001462C5F300136A09CDE90032C5F3810312
:10A6700005F0030260F0C4FF03B0F0BD40700708AE
:10A680002DE9F04FB44EB54CA64285B057D21D46C9
:10A6900002E00C36A64252D273798B42F9D133795B
:10A6A000834201D00028F4D1F3799342F1D1346888
:10A6B000002C44D000236360A360E36023616361E6
:10A6C000A361E36126603379237196F80690C4F89C
:10A6D0000890327AE260012B33D0022B2FD1F07A2E
:10A6E000FFF750FF96F90970A061B07A2774FFF761
:10A6F00049FF06466061F8B1DFF880A207EB8703E7
:10A700000AEB8303BA00D3F8CC810092B8F1000FB2
:10A7100012D093F8DE21EAB10E220023F2713372D7
:10A72000B57109213046FFF709FF3368B2881A83F3
:10A73000204605B0BDE8F08F2046FFF74DFF00240E
:10A74000F6E7F07AFFF71EFF727AB37A6374A061BE
:10A750002274EDE793F8D4B158465DF01DFE4FEA40
:10A760005B1201230BF01F0B023A03FA0BF3032ACF
:10A7700008D8DFE802F0ADA7B30279494A6922EAB6
:10A7800003034B61BB003B440AEB830393F8D10105
:10A79000FFF7F8FE791C0246C9B218B140F60A3339
:10A7A0000172C380BB003B440AEB8303CDE9002167
:10A7B00093F8D301FFF7E6FEDDE90021834620B1DF
:10A7C000017240F60A50ABF8060009F0040300934A
:10A7D000BB0003EB07090AEB8909CDE9022199F8CF
:10A7E000D201FFF7CFFEDDE9022199F8D591019062
:10A7F000002800F0D580019B197240F60A41D980EB
:10A80000009B002B70D0002A00F0C58010464A2122
:10A810004A46FFF7FDFEBBF1000F04D058464A46FA
:10A820002A21FFF7F5FE01984A460A21FFF7F0FEBC
:10A83000BB003B440AEB830393F8D0B1BBF1000F9C
:10A840006AD1484B984571D0474B984500F09880A5
:10A85000464B984575D0464B984500F0BE80454B19
:10A86000984500F0AF80444B984500F0D180009BA4
:10A87000B8F80020002B02F441520CBF0323002340
:10A88000134343F44573A8F80030B8F81C3023F4A0
:10A8900000631B041B0CA8F81C300723A8F8103019
:10A8A000B8F800309BB243F04003A8F80030BBF189
:10A8B000000F28D1BB003B440AEB8303012283F83D
:10A8C000DE2129E726490A6A22EA03030B6259E7D7
:10A8D00023494A6A22EA03034B6253E720490A6983
:10A8E00022EA03030B614DE722B110460A214A46D2
:10A8F000FFF78EFEBBF1000F95D058464A460A215D
:10A90000FFF786FE8FE75846FFF73CFE0028D1D0C0
:10A91000026883881383CDE75846FFF733FE00288B
:10A920008FD04A460921FFF773FE8AE703F5843387
:10A930005A6A42F480525A625A6A22F480525A6227
:10A9400095E703F5FE331A6A42F400421A621A6A66
:10A9500022F400421A628AE7BC9008086092080854
:10A96000003802400030014000380040003C004008
:10A97000003401400050014000540140CC1500203B
:10A9800003F500331A6A42F480421A621A6A22F40A
:10A9900080421A626BE7BBF1000F7FF43FAF42E7E2
:10A9A000009B2BB322B110464A214A46FFF730FEE6
:10A9B000BBF1000F3FF43CAF58464A462A21FFF74F
:10A9C00027FE35E703F568435A6A42F480125A625B
:10A9D0005A6A22F480125A6249E703F582335A6AAE
:10A9E00042F400525A625A6A22F400525A623EE716
:10A9F000CAB110460A214A46FFF70AFEBBF1000F12
:10AA00003FF416AF58464A460A21FFF701FE0FE70A
:10AA100003F564435A6A42F400125A625A6A22F4F5
:10AA200000125A6223E7BBF1000FEBD100E700BF31
:10AA30002DE9F04F83B01F46BDF830309DF834A0AB
:10AA40000093064689469046FBF7C0F8002800F0C0
:10AA50006F81DFF86CB39BF8D0430B2C00F263815D
:10AA60005C2202FB04B20021C2F8D41382F8D8138E
:10AA7000611CC9B2054630798BF8D0130191FFF7FC
:10AA800081FD002800F0478101990172022180F8C0
:10AA90000690C171BAF1000F2DD111210190FFF77D
:10AAA0004DFD019A116892884A835C2000FB04B036
:10AAB0004246C0F8D45339462846F7F775FC6D680E
:10AAC000A97901F00202003A18BF012211F0040036
:10AAD00015D04FF0000C500061464FF0040E664652
:10AAE0006F792A68032F00F24F81DFE817F0D80052
:10AAF0009A005C000E00327AFFF78AFDD5E751001C
:10AB00004FF4807C86460126EAE70E43118C21F43F
:10AB100080510904090C1184118C9588908B21F4C3
:10AB200000510904090C41EA063120F4E640A14E27
:10AB30000004000CB242ADB240F4C04000F01F81EE
:10AB400006F58066B24200F01A81009B95809083E2
:10AB500013641184908B20F400600004000C40F416
:10AB600000609083B2F844006FEA40406FEA5040C2
:10AB700080B2A2F844001146128892B242F001025B
:10AB800021F8402B8C4804EB4402C4EBC20200EBDA
:10AB900082005C2202FB04B30022C3F8DC130A60CB
:10ABA00003B0BDE8F08F0E43118C824F21F4807109
:10ABB0000904090C1184118C21F400710904090C99
:10ABC00041EA06259688918B21F073010904090C4E
:10ABD000BA42B6B241F0600100F0B78007F5806775
:10ABE000BA4200F0B280009B96809183D3631584B3
:10ABF000908B20F008000004000C40F008009083C7
:10AC0000B2F844006FEA40406FEA504080B2A2F8C8
:10AC100044001146128892B242F0010221F83C2B06
:10AC2000B0E70E43118C634F21F010010904090CA9
:10AC30001184118C21F020010904090C41EA061548
:10AC40009688118B21F4E6410904090CBA42B6B288
:10AC500041F4C04100F0868007F58067BA4200F0F9
:10AC60008180009B9680118393631584108B20F460
:10AC700000600004000C40F400601083B2F844004F
:10AC80006FEA40406FEA504080B2A2F8440011469B
:10AC9000128892B242F0010221F8382B72E70E437B
:10ACA000118C444F21F001010904090C1184118C0D
:10ACB00021F002010904090C41EA06059688118B6E
:10ACC00021F073010904090CBA42B6B241F06001E7
:10ACD00030D007F58067BA422CD0009B9680118354
:10ACE00053631584108B20F008000004000C40F022
:10ACF00008001083B2F844006FEA40406FEA504009
:10AD000080B2A2F844001146128892B242F00102C9
:10AD100021F8342B36E7BAF1000F7FF4C6AE1121CB
:10AD2000FFF70CFCC1E6254A00210420FAF7A0FE3B
:10AD3000002035E74FF6F3772F4026F4407607439F
:10AD400046EA0C064EEA0705C7E725F4006545EA22
:10AD5000002525F4806526F4405645EA0E2546EA8E
:10AD60000C1640E725F0800545EA001525F0400562
:10AD700026F4406645EA0E1546EA8C0671E725F48E
:10AD8000804545EA8C15E0E6B2F844106FEA41418F
:10AD90006FEA514189B2A2F8441011885C2000FB8F
:10ADA00004B48BB2002043F001031380C4F8DC0329
:10ADB0000060FFDE000001405C830020981A080854
:10ADC000887F002030B50368284D294C2DED028B7B
:10ADD000AB42246883B0F0EE408AB0EE608A10D0B7
:10ADE00005F58065AB420CD005F57055AB4208D037
:10ADF00005F58065AB4204D005F58065AB4218BF10
:10AE00006408B4FBF1F303F57F43FF331B0CB4FB81
:10AE1000F3F40023B4FBF1F5019200932246ABB2A8
:10AE20000221FFF705FEE0B1B5EE408A07EE904A39
:10AE3000F1EE10FAF8EE677A0ABF07EE105A28EE24
:10AE4000278AB8EE478A9FED0B7AC8EE076A01237E
:10AE5000037127EE667AC0ED046AA8EEA77A80ED4A
:10AE6000037A03B0BDEC028B30BD00BF000001408F
:10AE7000300C002000007A44074B53F8203021B1F9
:10AE80004BB11A689B8853837047002BFCD01A681B
:10AE90009B88138370477047347007082DE9F04F83
:10AEA000864FA7B000210A260C4607F624054FF06E
:10AEB000050B01968BE0BAF1000F19D143F0400366
:10AEC000BEF18C0F87F8283C00F2E48004F1010CFD
:10AED00098340DEB040A0CF198040DEB040C744645
:10AEE0004FF0040E0AF88CEC0CF88C3C04F1020EC6
:10AEF000BEF18C0F42F0020C00F2CC8004F19803FA
:10AF00006B4403F88BCC04F1040CBCF18C0F03F8F8
:10AF10008CBC00F2BF800EF198060DEB060E4FF0D0
:10AF2000060A0EF88CAC04EB0A0E4FEA8909BEF152
:10AF30008C0F5FFA89F603F8890C00F2AB8004F1FC
:10AF40009C0CEC444FF007090CF88C9C04F1080CA5
:10AF5000BCF18C0F03F8876C00F29C800EF1980610
:10AF60000DEB060E0EF88CBC03F8852C04F10A02DA
:10AF70008C2A00F28F8004F1A0060DEB060C0CF871
:10AF80008CAC03F8830C04F10C008C2800F2828056
:10AF900004F1A20204F1A3036A446B4402F88C9CFE
:10AFA000044603F88C8C480901F01F0C55F820303A
:10AFB000012202FA0CF223EA020345F82030019B39
:10AFC000013B01936ED00131B1F5F07F6AD23C2292
:10AFD0002846FAF721F8011E5FDB07EB410297F8DC
:10AFE000283CB2F860C81CF0040FC1F30722C8B2B5
:10AFF0005FFA8CF94FEA1C2803F0400A04F1020EB4
:10B000007FF459AFBAF1000F03D103F0380CCC45EF
:10B0100019D003F0870343EA0903BEF18C0F87F8C8
:10B02000283C37D804F1010C0CF1980698346C4494
:10B030000DEB060C4FF0040904F88C9C74460CF8D8
:10B040008C3C0EF1020EBEF18C0F23D804F1980354
:10B050000DEB030C231D8C2B0CF88B2C0CF88CBCEB
:10B0600018D80EF198020DEB020E06220EF88C2C69
:10B070000CF8890CA0188C280CD804F19C0304F15E
:10B080009D026B446A44072403F88C4C044602F882
:10B090008C8C88E76FF0004485E7204614B927B010
:10B0A000BDE8F08FD7F8200C234603AA002160F0FA
:10B0B00085FD012027B0BDE8F08F00BF887F00200C
:10B0C000F0B5284CD4F8200C83B010B194F8263C8D
:10B0D0000BB103B0F0BD01230DF10702842184F808
:10B0E000263CFEF7BFFB94F8282CD4F8200C042152
:10B0F0000A43FDF75BFDD4F8200C0DF10702842113
:10B10000FEF7B0FB9DF8073013F00406F3D1164D9F
:10B1100084F8283C3C223146284667F039FB324609
:10B12000124E05F13A0005F2FA374FF0010E30F8F1
:10B13000023F334002F01F019BB24FEA521C0EFA4D
:10B1400001F1013223B155F82C300B4345F82C3076
:10B15000B842ECD1FFF7A2FE0028FBD184F8260C00
:10B1600003B0F0BD887F0020AC87002004DFFFFF24
:10B1700070B5414DD5F8204C82B09CB395F8243C75
:10B18000012B43D0022B2FD1082194F910303B4AD8
:10B1900085F8271C03EB830302EB8303A2688DF879
:10B1A0000510002040F2044192078DF80400ADF82C
:10B1B0000610D3F8CC0142D504230DEB0302002185
:10B1C00060F05EFCA3689B0722D52D483C22FF213E
:10B1D00067F0DEFA95F8253C23B9FFF771FF0123EC
:10B1E00085F8253C02B070BD0DF10302A021204678
:10B1F000FEF738FB9DF8033003F00503012B37D031
:10B20000002B2FD1D5F8204C0821BEE74821BCE700
:10B210001C4B1D491A681D4B48684FF4FA7606FB13
:10B2200002F2A3FB023292094B681B1A9A42FBD22C
:10B230006369002BC9D01A689B881383C5E76369CB
:10B2400013B11A689B8853830E4B0F491A680F4B32
:10B250004E68D200A3FB023292094B689B1B9A42B4
:10B26000FBD2A9E70A4A126840F2DC539A42B9D9E4
:10B27000D5F8204C482188E7887F0020CC15002095
:10B28000AC870020CC3A0020001000E0D34D6210C3
:10B29000083600202DE9F041334D95F8263C82B068
:10B2A00003B1FEE7012285F8262C95F8272C0446E9
:10B2B00002F0F702D5F8200C85F8272C0E46194627
:10B2C000FDF774FCE2B207460921D5F8200CFDF722
:10B2D0006DFCB4F5807F3FD0D5F8200CDFF88C8072
:10B2E00050220821FDF762FCD5F8200C0DF1070271
:10B2F000A021FEF7B7FA48B9D8F88C31B8F89021F8
:10B3000059690A4214BF5A831A83EDE79DF8074032
:10B3100014F02004F0D1E2B20A21D5F8200CFDF798
:10B3200045FC3219D5F8200CC0210134FEF79AFAF9
:10B33000362CF0D157B995F8272CD5F8200C02F00F
:10B34000F702394685F8272CFDF730FC002385F8F5
:10B35000263C02B0BDE8F081D5F8200C40220A213D
:10B36000FDF724FCB8E700BF887F0020002A0020FA
:10B370002DE9F04F604D95F8267CC3B007B1FEE78C
:10B3800095F8272C044602F0F7020123D5F8200C8B
:10B3900085F8272C0E46394685F8263CFDF706FC35
:10B3A000FF2C4FF009038DF8054088BFA40801AABF
:10B3B0008CBF04F0C008B84602204FF0000C4FF0DC
:10B3C0000A0B0DF1050A4FF00B09137014E0B1F5EB
:10B3D000827F02F800B00AF8003016F80C3017D857
:10B3E0000CF1010CBCF1360F02F8079004F10604D1
:10B3F00002F80E30084614D0871C48EA0C03B7F553
:10B40000827F00F104010446DBB200F1030EDED9B5
:10B410000CF1010C6FF00041BCF1360F374C0846BF
:10B42000EAD1B4F5827F63D8082353540DF10503A4
:10B43000A0211954831CD5F8204C314E94F91010DA
:10B4400001EB810106EB8101D1F8CC01A1688907EC
:10B4500022D5002160F014FBA3689B0731D5294C4D
:10B46000D5F8200C0DF10302A021FEF7FBF948B935
:10B47000D4F88C31B4F8902159690A4214BF5A8328
:10B480001A83EDE79DF8033013F02003F0D185F81F
:10B49000263C43B0BDE8F08F616911B10E68898820
:10B4A00071831949194F0E681949D7F804C0F6007D
:10B4B000A1FB0616B6097968A1EB0C018E42FAD2FF
:10B4C000C7E7114B11491A68114B48684FF4FA76D7
:10B4D00006FB02F2A3FB023292094B681B1A9A4246
:10B4E000FBD26369002BBAD01A689B881383B6E736
:10B4F0006FF000439FE700BF887F002001000080BD
:10B50000CC150020002A0020CC3A0020001000E0DA
:10B51000D34D621038B5837913F0010F044603F060
:10B520002002C36B406B1FD0002A5D680CBF422114
:10B53000022110B12A7AFFF76BF8012384F86032F8
:10B54000A4F85C326A790C48296810440A8C90F897
:10B55000D00283409BB292B222EA03020A840A8C90
:10B5600092B213430B8438BD002A5D680CBF2221C0
:10B5700002210028DED1E0E740700708F8B58368B3
:10B580001C686579A80744D4ED0700D4F8BD94F889
:10B590005C32002BFAD194F85D320133DBB2092B17
:10B5A00084F85D3277D00A2BF0D194F85F52B4F86A
:10B5B0006632002D00F08D80980502D4DA0700F184
:10B5C000F580B4F86A320133A4F86A3201239D424F
:10B5D000A4F85C32DAD1E66BA179002384F85F32FB
:10B5E00001F0010130465CF021FE7268764B507923
:10B5F000116803440A8C93F8D03205FA03F39BB226
:10B6000092B222EA03020A840A8C92B213430B8498
:10B61000F8BD94F86112002934D1A26A636A94F8E3
:10B620006002934200F09180531CA669A362B65C4D
:10B630002269A779934228BF00237600A3620A23D8
:10B6400046F4007684F862320123A4F8646284F838
:10B65000613208B13A074CD47B0695D509224020C7
:10B6600087EA06037608A4F86462DE07A16B2AD491
:10B6700011B10B688988598384F86222002883D02D
:10B680002AB181E794F96222002A40F095800023D4
:10B6900084F8613278E794F85F32002B7FF476AF5C
:10B6A00094F85E32082B3FF671AFB4F866220120A1
:10B6B00000FA03F101330A43D9B2082992B2F7D94B
:10B6C000A4F86622F8BD0029D6D00B6889881983B2
:10B6D000D2E743F001009905A4F866024AD4E36A70
:10B6E0004008002B53D0216BC0B2984794F85F52AA
:10B6F0006CE7E26BD2F804E0334A9EF80500DEF80E
:10B7000000C00244606B92F8D0229340BCF8202025
:10B7100092B222EA0303ACF82030BCF820309BB28E
:10B72000ACF8203018B19EF80820FEF771FF002316
:10B7300084F86032236CA06B2BB35B681A7A002804
:10B740008AD00121FEF764FF86E700287FF41CAF52
:10B75000A37919077FF518AF216CA36B41B32BB107
:10B760004A680146127A1846FEF752FF2046FFF754
:10B77000D1FE09E7B4F86A3201221344A4F85C222E
:10B78000A4F86A32F8BD0121FEF7D8FE64E7E36948
:10B790006269C0B2D054E369E26894F85F52013341
:10B7A000B3FBF2F102FB1133E3610FE7184696E7B2
:10B7B0001846FEF7C3FED9E7A779B4F86462013AE8
:10B7C00007F0400052B24BE74070070838B5044616
:10B7D0004068304B0568304A9D421268084610D0D8
:10B7E00003F580639D420CD003F570539D4208D051
:10B7F00003F580639D4204D003F580639D4218BF2A
:10B8000052081346B3FBF0F1B1F5803F0FD289B275
:10B810002046F6F7C9FD23681A685379DBB9937996
:10B820004BB92B889BB243F001032B8038BD012B11
:10B83000EAD95B08E6E71A061ED41849CA18302070
:10B8400082F800035809012203F01F0302FA03F3F0
:10B8500041F82030E5E7190615D410485C0900EBE3
:10B86000030C012103F01F0301FA03F330218CF8CC
:10B87000001340F82430D2E7094A03F00F031A44BA
:10B8800030231376CDE7064903F00F031944302324
:10B890000B76C4E700000140300C002000E100E01E
:10B8A000FCEC00E00346C06B99608FE7002ABCBF48
:10B8B00080185242002B30B503EB010503DA0C4629
:10B8C0005B42294625460028B7BF121A8418144641
:10B8D0000020A4F11D0C0029BCBF2B460021BCF1A7
:10B8E000000FC4BFA2EB0C021418A5F10F02002A2E
:10B8F000C4BF9B1A5D1884421EDBC1F1010C0F4AC4
:10B90000AC44C1EB0113CCEB0C1C00EB4303013442
:10B910004FEA4C0C02EB43024FF0200E8D42A8BFC1
:10B92000002304DB22F813E01E339C45FAD10130DA
:10B93000A04202F10202F1D130BD00BFE887002031
:10B940001B4B1C48196C1C4A10B441F08051012457
:10B95000196404625321FF24CA2054625062516268
:10B960005B6FDB0085B013D400231449029302916E
:10B97000029A134804320292029A136003930391CD
:10B98000039B0393039B186005B05DF8044B70475D
:10B990000A4B002201920193019B0193019A084BEB
:10B9A00012689A42E0D105B05DF8044B704700BFC1
:10B9B0000038024000000E4200280040502800409D
:10B9C00076614E692DE9F04F2DED028BA74BA84C07
:10B9D0001B78A84FA84EB1B04FF000080293A146C3
:10B9E000C246A4F1100BD9F80050002357F83320B9
:10B9F000954203D001330E2BF8D1FF23334493F843
:10BA00002C3C012B00F0AF80022B09D1D9F80C306F
:10BA10005A0705D523F0040343F00803C9F80C3096
:10BA20004846FBF70FFC48B90AEB8A030BEB83038C
:10BA3000D96901F00C03042B00F0A1800AF1010A7E
:10BA4000BAF10C0F09F11409CDD1DDF8089004F119
:10BA5000F007254609E02868EA60FBF7F3FC50444C
:10BA60005FFA80F81435BD4220D02846FBF7EAFB88
:10BA70000028F7D1EB68580703F00C02F2D5042A2E
:10BA8000F0D023F0080242F0040208F10100C145A1
:10BA900011465FFA80FA23F00403DCD82868EB60D3
:10BAA00019461435FBF7CEFCBD42DED10023734DA1
:10BAB000DFF8F4A11F46994698469B462046FBF7BF
:10BAC000C1FB00287BD1E368590763D5029A55F87A
:10BAD0000C0C42457AD81A075ED4B9F1000F55F81C
:10BAE0000C3C40F38F8023A9002202E04A4500F07D
:10BAF000898051F8040F0068834202F10102F5D1F8
:10BB00000BF1010BBBF10C0F04F1140405F114054A
:10BB1000D4D1564BCDF80C9093F80090B9F10C0F9E
:10BB200000F31982564B574A9B791370032B75D932
:10BB30001A1F022A00F28682052B00F03882062B9B
:10BB40000CBF4FF47A544FF47A644F494F480022A7
:10BB50004A6000254E4AB2FBF4F200240A60C0E9B4
:10BB600000454C4A5BE0D9F80C3019077FF558AF17
:10BB700023F0080343F00403C9F80C3050E72846CB
:10BB8000FBF760FC08F101085FFA88F880445FFA6F
:10BB900088F853E71907B3D5002F55F80CEC24DDCE
:10BBA00017A9002201E0BA421FD051F8040F006823
:10BBB000864502F10102F6D15B07A1D58DE75B4610
:10BBC000524601210420F9F753FF99E723F00801B9
:10BBD000E160FBF737FCE36808F101081A075FFA38
:10BBE00088F8D9D45B078BD577E730AB03EB8902B4
:10BBF00008217046E16042F8304C09F10109FBF779
:10BC000021FC7DE7184630AB03EB87020421E1609D
:10BC100042F8604C0137FBF715FC71E71E4AC6F885
:10BC20003C2C1E4A12F81330002B00F0C781B94596
:10BC300000F30482B9F1000F7ED09FED198ADFF87E
:10BC40006CB0184D0DF15C0800240E4BDBF804209D
:10BC50001B7858F8040FC2F30072062B00F25982C9
:10BC6000DFE803F08E857C59262626009000001020
:10BC7000DC15002018630708887F0020E8150020E5
:10BC800084420020FA4000200041002008410020AA
:10BC900040420F00B1740008F588000808630708E7
:10BCA0006F12833A340C0020D41A08089800001050
:10BCB000052B00F05C81C449C44F062B08BF3946F0
:10BCC0000027019200970A4614230221FEF7B0FED6
:10BCD0000290002800F04D81029AD2F800C0DCF8F2
:10BCE00004E03B46DEF800A0DEF81070590105EBD9
:10BCF00043106A587A4012F47C5F03F1010300F0AC
:10BD0000A080102BF2D10023CCF80C30B04B029A5B
:10BD100043F834200DE0DFEDAF0AAF4BB0EE600A20
:10BD20009988FFF74FF8AA4B43F83400002800F039
:10BD300023810134A14588D196F8403C4BBBA74AEA
:10BD400002210420F9F794FE96F83A0CB0FA80F03C
:10BD5000400931B0BDEC028BBDE8F08FDFEDA00AE9
:10BD60009FEDA00A4FF4FA61FFF72CF8DBE7DFED57
:10BD70009E0A4FF47A71B0EE600AFFF723F8D2E71B
:10BD80009FED9A0AF0EE480A4FF4C871FFF71AF8CF
:10BD9000C9E796F8419C96F8423C09F10109A9EBE4
:10BDA0000309B9F1100F0BDD102302210093904A13
:10BDB00086F83A1C4B4600210420F9F759FEC3E7E8
:10BDC00096F84C3C012B00F0F580022B00F0DE8051
:10BDD000884AC6F8502C002B40F0E380039B99451D
:10BDE00000F33281B9F1000FAEDD834FDFF848B2C6
:10BDF000DFF8088223AD002404E001344C4547F805
:10BE0000040BA1D0DBF80430B6F8441CC3F3007275
:10BE1000B6F8463C01920091B8FBF3F3774A55F827
:10BE2000040F9BB20321FEF703FE0028E5D1052590
:10BE30000146734A86F83A5C23460420F9F718FE57
:10BE400082E7037FCCF80C00002B7FF45FAFBAF8D9
:10BE500044306FEA43436FEA53439BB2AAF844303D
:10BE6000BAF800309BB243F08003AAF800309EF885
:10BE70000520644B9EF806E004929A181EF0040F09
:10BE800092F8D022BAF820E014BF04230123934093
:10BE90009BB21FFA8EFE2EEA030EAAF820E0BAF833
:10BEA000202092B21343AAF82030BAF8003042683A
:10BEB0009BB243F00103AAF80030534B9A4200F0C2
:10BEC000D580524B52481A6B42F480021A6301F13A
:10BED00018024FF0070E20F802E01A6B42F48002BD
:10BEE0001A636A184B4892F91430C2F818C0002B34
:10BEF000D060C0F2B480484A580902EB030C4FF0FE
:10BF0000010E03F01F030EFA03F34FF0300E8CF80E
:10BF100000E342F8203029448B6805931846F6F771
:10BF20000FFC059B1A6822F001021A601846F6F70A
:10BF300007FCDDE904130022CDE91222CDE9142229
:10BF40000C921092032900F2E180DFE811F0DC008E
:10BF5000D900D600A100314ACDF800B0012186F801
:10BF60003A1C4B4600210420F9F782FDE4E62C49F7
:10BF7000A6E6174B43F83400052186F83A1C294AF7
:10BF8000234600210420F9F773FDD5E65DF0C2F9E0
:10BF9000254A96F84C3CC6F8502C13F0FD0F3FF4A0
:10BFA0001DAF224A02210420F9F762FDCCE64FF4CE
:10BFB000FA54CAE55DF0AEF91D4AEAE71D4A0221CE
:10BFC0000420F9F755FDB7E6C0C62D00001BB700E9
:10BFD0004041002000000000844200209C1B080813
:10BFE000ACC5A737ACC5A7366F1203396F12833AB9
:10BFF000B81B08087D7400086080002040420F00D4
:10C00000581C0808407007080060024000380240D1
:10C01000380C0020D102000800E100E0EC1A08080A
:10C02000808D5B00741B080895740008E41B0808E9
:10C03000F5EC0208181B080898000010374A009712
:10C0400003218CE7364AEAE5039B00930420354A36
:10C0500086F83A0C4B460021F9F70AFD74E6324A9D
:10C0600003F00F031A443023137654E7A3F520534B
:10C070002E481A6B42F400121A6301F118024FF0B5
:10C08000070E20F802E01A6B42F400121A6328E748
:10C090000AF1400A264A0493FFB202EB87024FF4EA
:10C0A000804ED2F8D4220792029ACDF820A002F155
:10C0B000140712220B924FF480620D924FF48052BB
:10C0C000CDE90E2E402218460A9207A94FF40032FD
:10C0D000119209975CF034F9049B1A6842F010023F
:10C0E0001A6038464822002166F052FB029A01236A
:10C0F0001371104B43F834201BE60AF13C0AC9E7E0
:10C100000AF1380AC6E70AF1340AC3E74FF0000A19
:10C11000C0E7084A002342F834302DE7381B0808EE
:10C12000AD740008201C0808FCEC00E0380C00206E
:10C13000407007084041002010B5104CD4E904239A
:10C14000A16882B002FB03F38B428DF8070012D086
:10C150006368E0680DF10701184464F001FF63684B
:10C160002269A16813446269B3FBF1F0013201FB5B
:10C1700010336360626102B010BD00BF184100203F
:10C1800010B50379012B84B00C4627D0022B23D1A4
:10C190008368DB070DF10F024CBF01218121FDF700
:10C1A0000FFB9DF80F300022C3F3001161F307026B
:10C1B000C3F3800161F30F220F49C3F3C00C6CF38A
:10C1C000174281F80001C3F3801161F31F62DB099C
:10C1D0002260237104B010BD0020E2E782680DF1F7
:10C1E0000F0102F00102CDE900121A46417C90F9DC
:10C1F0001000F7F72FFCD4E7CC1500202DE9F04113
:10C2000082B014460E4601AA50210546FDF72AFBCE
:10C210009DF80430DFF8F080394F01335B00DBB26A
:10C220004621238001AA2846FDF71CFB23789DF8B0
:10C23000042008FB03F303F5FA73A7FB0313013291
:10C240009909DB0902FB0133A280A7FB03239B09A9
:10C2500001AAE360512102232846FCF799FE2378C6
:10C26000BDF8040008FB03F340BA03F5FA73A7FB1B
:10C270000323C2B2C0F307208240013292B2980970
:10C28000DB0902FB0033A7FB03739B097021E280EB
:10C29000238201AA2846FDF7E5FA9DF80430013310
:10C2A0005B00DBB201AA6380712102232846FCF700
:10C2B0006FFEBDF80430134AF17882F800015BBAD2
:10C2C000DAB2C3F307239A40013292B2228119B144
:10C2D000E388D21A92B222810B48A378084900FB66
:10C2E00003F303F5FA73A1FB03039809DB0902FBCF
:10C2F0000033A1FB03139B09638202B0BDE8F08108
:10C30000D34D6210CC150020002F3A002DE9F047E4
:10C31000DFF89882DFF89892A34F8CB0054600268C
:10C320004FF4FA7307AA89210068C8F87C3388F8AB
:10C330001861FDF797FA9DF81C20286842F0010269
:10C340008921FCF733FC324688212868FCF72EFC53
:10C35000012280212868FCF729FC0122FF2128689E
:10C36000FCF724FC324631462868FCF71FFC07AA7C
:10C3700091212868FDF776FA9DF81C30286888F826
:10C38000753331460122FCF711FC3246FF21286843
:10C39000FCF70CFC324680212868FCF707FC07AA52
:10C3A00060212868FDF75EFA9DF81C20286842F09D
:10C3B00012026021FCF7FAFB4FF40053ADF81C3079
:10C3C00007AA022344212868FCF712FDFF2201215D
:10C3D0002868FCF7EBFB2C68012280212046FCF743
:10C3E000E5FB0122FF212046FCF7E0FB3246314607
:10C3F0002046FCF7DBFB0622FF212046FCF7D6FB9C
:10C4000007AA83212046FDF72DFA9DF81C208321E1
:10C4100042F004022046FCF7C9FB0722FF21204618
:10C42000FCF7C4FB012281212046FCF7BFFB01225F
:10C4300080212046FCF7BAFB6B2294212046FCF7B2
:10C44000B5FB324683212046FCF7B0FBD9F80060EB
:10C45000C8F878632379012B00F09880022B0FD065
:10C4600000209DF81C3087F80001DBB9D9F80030B6
:10C470009BB29B1BB3F5FA7FECD90CB0BDE8F087FB
:10C48000A368DB0707AA4FF0830120465EBF07AA17
:10C4900083212046FDF794F99DF81C3087F80001B0
:10C4A000002BE3D0012283212046FCF77FFB07AA63
:10C4B00092212046FDF7D6F90022812120469DF8E1
:10C4C0001CA0FCF773FB0622FF212046FCF76EFB45
:10C4D00007AA83212046FDF7C5F99DF81C2083217A
:10C4E00002F0FB022046FCF761FB0122FF212046FF
:10C4F000FCF75CFB012200212046FCF757FB0022E1
:10C50000FF212046FCF752FB204600228021FCF749
:10C510004DFB0623B02105AA2868FCF739FD01224E
:10C52000FF212868FCF742FB00224F212868FCF716
:10C530003DFB2C224E212868FCF738FB0022FF210E
:10C540002868FCF733FB4FEADA162868B422B621D4
:10C55000FCF72CFB0024002E18BF0C260AF07F0AE3
:10C56000A1464FF0010EC4F3C40330336B44E2B272
:10C5700013F81C0C04F0070C0EFA0CF1964220EA9A
:10C58000010117D903F81C1C0134ECE7A268617C97
:10C5900094F9100002F00102019207AA009283228E
:10C5A000F7F758FA5DE700BFCC150020887F002020
:10C5B00008360020D14540FA0CF200F01183D30771
:10C5C00044BF09F101095FFA89F90134302CCAD15D
:10C5D000062305AAB0212868FCF70AFC0122FF21E6
:10C5E0002868FCF7E3FA002211462868FCF7DEFA17
:10C5F0000022FF212868FCF7D9FA002209212868C7
:10C60000FCF7D4FA002210212868FCF7CFFA0022A8
:10C6100011212868FCF7CAFA012224212868FCF7B6
:10C62000C5FAFF2225212868FCF7C0FA00227521EF
:10C630002868FCF7BBFA0122FF212868FCF7B6FA4C
:10C640002C224E212868FCF7B1FA002248212868E4
:10C65000FCF7ACFA214620222868FCF7A7FA002252
:10C66000FF212868FCF7A2FA214609222868FCF776
:10C670009DFA002254212868FCF798FA04223121FF
:10C680002868FCF793FA032232212868FCF78EFA17
:10C69000832240212868FCF789FA25224621286850
:10C6A000FCF784FA002260212868FCF77FFA002258
:10C6B00027212868FCF77AFA062250212868FCF71F
:10C6C00075FA002251212868FCF770FA962252214F
:10C6D0002868FCF76BFA082256212868FCF766FAEE
:10C6E000224657212868FCF761FA00226121286858
:10C6F000FCF75CFA002262212868FCF757FA002256
:10C7000064212868FCF752FA002265212868FCF7AA
:10C710004DFAA02266212868FCF748FA0122FF2181
:10C720002868FCF743FA322222212868FCF73EFAF7
:10C73000142247212868FCF739FAFF22492128688A
:10C74000FCF734FA00224A212868FCF72FFA00226D
:10C75000FF212868FCF72AFA0A227A212868FCF7C8
:10C7600025FA00227B212868FCF720FA2122782173
:10C770002868FCF71BFA0122FF212868FCF716FA4B
:10C78000342223212868FCF711FA0022422128686C
:10C79000FCF70CFAFF2244212868FCF707FA26224E
:10C7A00045212868FCF702FA052246212868FCF793
:10C7B000FDF9402211462868FCF7F8F906220E21FF
:10C7C0002868FCF7F3F91A2220212868FCF7EEF913
:10C7D000402243212868FCF7E9F90022FF2128685C
:10C7E000FCF7E4F9032234212868FCF7DFF944223E
:10C7F00035212868FCF7DAF90122FF212868FCF7C7
:10C80000D5F9042231212868FCF7D0F909224B21FF
:10C810002868FCF7CBF905224C212868FCF7C6F9FB
:10C8200004224D212868FCF7C1F90022FF21286865
:10C83000FCF7BCF9002244212868FCF7B7F9202254
:10C8400045212868FCF7B2F9082247212868FCF73F
:10C85000ADF9282248212868FCF7A8F900226721B1
:10C860002868FCF7A3F9042270212868FCF79EF9D8
:10C87000012271212868FCF799F9FE2272212868AB
:10C88000FCF794F9002276212868FCF78FF9002242
:10C8900077212868FCF78AF90122FF212868FCF734
:10C8A00085F901220D212868FCF780F90022FF217B
:10C8B0002868FCF77BF9012280212868FCF776F9CB
:10C8C000F82201212868FCF771F90122FF2128686C
:10C8D000FCF76CF901228E212868FCF767F9012228
:10C8E00000212868FCF762F90022FF212868FCF784
:10C8F0005DF9002280212868FCF758F904220A21FA
:10C900002868FCF753F92C6807AA84212046FCF715
:10C91000A9FF9DF81C20204602F0EF028421FCF7BD
:10C9200045F901220B212868FCF740F92C6803A97E
:10C930002046FFF725FC07AA03A92046FFF75EFC67
:10C940009DF80C30002B00F05C810A9C04F68454A6
:10C950009DF80E30002B00F04A810A9B03F2B223AF
:10C9600004EB43049DF80F3023B1BDF82C3003F5E0
:10C9700025731C449DF8103023B1BDF82E3003F20E
:10C9800026231C44E82201212868C8F8544CFCF7EF
:10C990000DF9286821465CF0D3FF01221146286872
:10C9A000FCF704F9402187F800012868FDF7C4FA74
:10C9B00000283FF462AD012128680222FCF7F6F856
:10C9C000002187F800012868FDF7B6FA00283FF437
:10C9D00054ADE82201212868FCF7E8F84FF4005331
:10C9E00007AAADF81C30442102232868FCF700FA9E
:10C9F0002C6803A92046FFF7C3FB07AA03A920461A
:10CA0000FFF7FCFB502257212046FCF7CFF8082205
:10CA100056212046FCF7CAF8082250212046FCF790
:10CA2000C5F8BDF82C204FF47A7148F20E6301FB73
:10CA30000233794A934240F2EB80784AA2FB0332F8
:10CA4000120C013AFF2A4FF0000306DD52080133B1
:10CA5000FF2A9BB2FAD81B029BB21343C3F30722EF
:10CA6000DBB28DF808208DF8093002AA022351218B
:10CA70002046FCF7BDF90A9A4FF47A7148F20E632A
:10CA800001FB0233664A934200F2C080634AA2FB74
:10CA90000332120C013AD2B246212046FCF786F846
:10CAA0002046D8F8541C5CF04BFF02AA0121204616
:10CAB000FCF7D8FE02229DF8086001212046FCF711
:10CAC00075F800212046FDF737FA3246204601214D
:10CAD000FCF76CF82C6803A92046FFF751FB07AA66
:10CAE00003A92046FFF78AFB482211462046FCF79F
:10CAF0005DF8082247212046FCF758F8032232212E
:10CB00002046FCF753F8072230212046FCF74EF868
:10CB10000122FF212046FCF749F82022302120463F
:10CB2000FCF744F80022FF212046FCF73FF80622DC
:10CB300070212046FCF73AF8BDF82E10394A4FF420
:10CB40007A7046F6440300FB0133A2FB03239DF8F1
:10CB50000F201B0B1AB1BDF8222013449BB2002BEF
:10CB600052D05A1EFF2A4FF0000306DD520801334F
:10CB7000FF2A9BB2FAD81B029BB21343C3F30722CE
:10CB8000DBB28DF808208DF8093002AA022371214A
:10CB90002046FCF72DF9D8F8541C20465CF0D0FE56
:10CBA00002AA01212046FCF75DFE9DF808500222F2
:10CBB00001212046FBF7FAFF00212046FDF7BCF9D2
:10CBC0002A4601212046FBF7F1FF6422012387F862
:10CBD0000001C8F87C2388F818310CB0BDE8F08754
:10CBE0000EFA0CFC20EA0C0003F81C0CEDE49DF896
:10CBF0000D30002B3FF4B6AE0A9B03F525731C44A1
:10CC0000B0E640F63634A3E61A46BAE7FF2243E719
:10CC100000231A4625E700BF1B0C0100950370F4A2
:10CC20001B280D014963A41310B5174C84F8691231
:10CC3000017952BAA4F86A2201294FF0000282B0A9
:10CC400084F8682210D0022903D06FF00C0002B0E3
:10CC500010BD042304F51A72FF21FCF771F80028B7
:10CC6000F3D0002002B010BD8268417C90F9100022
:10CC700004F51A7402F00102CDE900420423FF22F8
:10CC8000F6F7D8FCEBE700BF887F00202DE9F04FD6
:10CC90009D4F9E4D06683C464FF0000885B0834688
:10CCA00085F81A815B37C4F12D0905F51A7A13E06E
:10CCB000022B0FD1B26812F0010F4FF0030352465E
:10CCC0004FF0FF01304601BF03235246FF2130469B
:10CCD000FCF736F8A7421AD0337985F8688209EB59
:10CCE0000401012B14F8012F85F8691285F86A22D6
:10CCF000DED1B368717C96F9100003F00103CDE931
:10CD000000A3FF220323F6F795FCA742E4D14FF4DA
:10CD10000743A5F86832402385F86A325246032358
:10CD2000FF213046FCF764F800238DF80E300DF13A
:10CD30000E0130465CF0CEFD9DF80E30002BF6D093
:10CD40004FF40643A5F868320123714A85F86A3228
:10CD5000FF2103233046FCF74BF84FF407436C4A9E
:10CD6000A5F8683200240323FF21304685F86A4283
:10CD7000FCF73EF84FF40063A5F868320923644AD3
:10CD800085F86A32FF2103233046FCF731F84FF46F
:10CD90003063A5F868325E4A85F86A42304603235C
:10CDA000FF21FCF725F8002800F0AC80DBF80040FC
:10CDB0000DF10E025E212046FCF7D0F9BDF80E30D1
:10CDC000B3F5D77F00F08C806AD8512B00F08480B7
:10CDD00078D81D2B7ED10F2608BB0A224B21204676
:10CDE000FCF728F80F2260212046FCF723F80D22DB
:10CDF00063212046FCF71EF8B82269212046FCF783
:10CE000019F840F60D7278212046FFF70DFF40F625
:10CE10000E627A212046FFF707FF00286DD0DBF86D
:10CE2000000021215CF0ACFCDBF800400DF10E02AB
:10CE3000DE212046FCF792F9BDF80E309FED357AE1
:10CE4000C3F3090303EB8303DB0007EE903AF8EE2C
:10CE5000E77A4FF4D84267EE877AA5F86822FCEEAD
:10CE6000E77A524617EE903A1BBAC5F86A32FF21AC
:10CE700006232046FBF7BCFF4FF407414023DBF8B5
:10CE80000000A5F8681285F86A3252460323FF2194
:10CE9000FBF7AEFFB0B385F81A0105B0BDE8F08F1F
:10CEA00040F2E132934219D01CD840F2D922934289
:10CEB00014D040F2E122934202D0B3F5E67FAED126
:10CEC000642689E7AD2B0BD0D62B01D0602BA6D1E1
:10CED000212681E71E2BA2D114267DE7C8267BE7F9
:10CEE000322679E740F28F42934203D040F29152CA
:10CEF000934294D14FF4FA766EE7314620465CF0C7
:10CF00003FFC8CE70020C6E733730708887F0020CA
:10CF1000F08100209A99893F03682DE9F041DF698B
:10CF20001FB13B46BDE8F0411847002A164611DD07
:10CF300004460D460E4400E023689B68204698474F
:10CF40000028F9D0236815F8011B1B682046984774
:10CF5000B542F1D1BDE8F081DEE700BFBFF34F8FEE
:10CF60000549064BCA6802F4E0621343CB60BFF385
:10CF70004F8F00BFFDE700BF00ED00E00400FA05A1
:10CF800008B572B600224FF0FF31930003F1604301
:10CF900003F561430132082AC3F88010C3F88011F9
:10CFA000F3D1FFF7DBFF00BF012108B50846F7F713
:10CFB000C7FAFFF7E5FF00BF00B583B00D490022B7
:10CFC00000920091009B04330093009B1B68012B8F
:10CFD00002D003B05DF804FB01920191019B064968
:10CFE00004330193019B1A600B6883F308884B6834
:10CFF0009847FEE7502800400000FF1F10B4EFF3F1
:10D000001183102282F31288094C0A4822684FF0DB
:10D01000E021013222608A69C0F8582C0022C0F851
:10D020005C2C0A69DBB283F311885DF8044B70470E
:10D0300008360020887F002030B4EFF311821023DF
:10D0400083F312884FF0E023D2B29969186910F483
:10D05000803F0D481EBF0121C0F85C1C99690B4B35
:10D060001D68D0F85C3C82F31188094804684FF4CD
:10D070007A7202FB04F02B44401A0021B0FBF4F05A
:10D0800030BCE3FB02017047887F00200836002097
:10D09000CC3A0020124B5B68C3F30803FBB9EFF3F3
:10D0A0001183E3B930B40F4A0F4C4FF0E02C1368F2
:10D0B000DCF8180011688B42F9D1D4F8581C88426A
:10D0C000F5D80A4A15684FF47A7404FB05F200217A
:10D0D000101AB0FBF5F0E3FB040130BC7047ABE77E
:10D0E00000ED00E008360020887F0020CC3A0020C8
:10D0F00090B170B5461EFFF7CDFF04460D46FFF711
:10D10000C9FF001B61EB0501B0F57A7F71F10001E9
:10D11000F5D3013EEFD270BD704700BF2DE9F0415D
:10D12000076888B08046B6227E213846FBF73EFD70
:10D130006426FFF7AFFF04460D46FFF7ABFF001B69
:10D1400061EB0501B0F57A7F71F10001F5D3013E85
:10D15000EFD102213846FBF77FFC7B6913B11A68D7
:10D160009B885383FFF796FF04460D46FFF792FF17
:10D17000001B61EB0501B0F57A7F71F10001F5D379
:10D180007B6913B11A689B8813830A26FFF782FF15
:10D1900004460D46FFF77EFF001B61EB0501B0F56D
:10D1A0007A7F71F10001F5D3013EEFD132467C2147
:10D1B0003846FBF7FBFCFFF76DFF04460D46FFF713
:10D1C00069FF001B61EB0501B0F57A7F71F1000189
:10D1D000F5D3002259213846FBF7E8FCFFF75AFF48
:10D1E00004460D46FFF756FF001B61EB0501B0F545
:10D1F0007A7F71F10001F5D35E22002371498DF829
:10D2000007200DF10702CDE902320122CDE90531F7
:10D21000049202A94FF4A472384607925EF080FC93
:10D220000A26FFF737FF04460D46FFF733FF001BC2
:10D2300061EB0501B0F57A7F71F10001F5D3013E94
:10D24000EFD1012259213846FBF7B0FCFFF722FF4E
:10D2500004460D46FFF71EFF001B61EB0501B0F50C
:10D260007A7F71F10001F5D38C2240213846FBF71B
:10D270009DFCFFF70FFF04460D46FFF70BFF001B59
:10D2800061EB0501B0F57A7F71F10001F5D303225E
:10D2900041213846FBF78AFCFFF7FCFE04460D46A9
:10D2A000FFF7F8FE001B61EB0501B0F57A7F71F125
:10D2B0000001F5D3444CD8F8382098F83500B4FB79
:10D2C000F2F2092391B2414AF9F768FD4388B4FBB1
:10D2D000F3F4C8F840400279422142F0C0023846D7
:10D2E000FBF764FCFFF7D6FE04460D46FFF7D2FEBF
:10D2F000001B61EB0501B0F57A7F71F10001F5D3F8
:10D30000082243213846FBF751FCFFF7C3FE0446D1
:10D310000D46FFF7BFFE001B61EB0501B0F57A7FFC
:10D3200071F10001F5D3042258213846FBF73EFC89
:10D33000FFF7B0FE04460D46FFF7ACFE001B61EBA5
:10D340000501B0F57A7F71F10001F5D30A2253216E
:10D350003846FBF72BFCFFF79DFE04460D46FFF712
:10D3600099FE001B61EB0501B0F57A7F71F10001B8
:10D37000F5D300227C213846FBF718FCFFF78AFE24
:10D3800004460D46FFF786FE001B61EB0501B0F574
:10D390007A7F71F10001F5D306227D213846FBF733
:10D3A00005FCFFF777FE04460D46FFF773FE001BF2
:10D3B00061EB0501B0F57A7F71F10001F5D308B09A
:10D3C000BDE8F0819073070840420F00D874070849
:10D3D0002DE9F043836B0768A04AA14CB4FBF3F13D
:10D3E00083B080460F2389B290F83500F9F7D6FC58
:10D3F00000214388B4FBF3F48146C8F84040384626
:10D40000FBF72AFB002276213846FBF7CFFB0F22E1
:10D410004E213846FBF7CAFB0F26FFF73BFE0446BA
:10D420000D46FFF737FE001B61EB0501B0F57A7F73
:10D4300071F10001F5D3013EEFD199F805204F219C
:10D4400002F00F023846FBF7B1FB0F26FFF722FE72
:10D4500004460D46FFF71EFE001B61EB0501B0F50B
:10D460007A7F71F10001F5D3013EEFD199F80520E3
:10D47000502102F00F023846FBF798FB0F26FFF70A
:10D4800009FE04460D46FFF705FE001B61EB050192
:10D49000B0F57A7F71F10001F5D3013EEFD1FF22A3
:10D4A00052213846FBF782FB0F26FFF7F3FD0446B7
:10D4B0000D46FFF7EFFD001B61EB0501B0F57A7F2C
:10D4C00071F10001F5D3013EEFD198F8351007292D
:10D4D00041D0644D95F82101FAF762F80446012223
:10D4E00076213846FBF762FBA2780C213846FBF721
:10D4F0005DFB22790D213846FBF758FBA279A38802
:10D50000120142EA1322D2B20E213846FBF74EFB3B
:10D510004FF4807195F82101FAF742F8044602228F
:10D5200076213846FBF742FBA2785200032102F035
:10D53000FE023846FBF73AFB227904213846FBF716
:10D5400035FBA279A388120142EA13220521D2B247
:10D550003846FBF72BFB002276213846FBF726FBEB
:10D56000032214213846FBF721FB0F26FFF792FD1B
:10D5700004460D46FFF78EFD001B61EB0501B0F57B
:10D580007A7F71F10001F5D3013EEFD1324663217C
:10D590003846FBF70BFB6426FFF77CFD04460D467F
:10D5A000FFF778FD001B61EB0501B0F57A7F71F1A3
:10D5B0000001F5D3013EEFD1082265213846FBF783
:10D5C000F5FA64210DF107023846FCF74BF99DF896
:10D5D000072022F0100242F06002642138468DF8E4
:10D5E0000720FBF7E3FA0F26FFF754FD04460D462C
:10D5F000FFF750FD001B61EB0501B0F57A7F71F17B
:10D600000001F5D3013EEFD10DF106024D21384660
:10D61000FCF728F99DF8062002F03F0242F0400294
:10D620004D2138468DF80620FBF7C0FA0F26FFF78C
:10D6300031FD04460D46FFF72DFD001B61EB050192
:10D64000B0F57A7F71F10001F5D3013EEFD10321EE
:10D650003846FBF701FA03B0BDE8F0831075070800
:10D6600040420F00887F0020F0B5002283B00746BB
:10D670000A210068FBF79AFA1426FFF70BFD04460F
:10D680000D46FFF707FD001B61EB0501B0F57A7F42
:10D6900071F10001F5D3013EEFD138680F220A2164
:10D6A000FBF784FA0A26FFF7F5FC04460D46FFF760
:10D6B000F1FC001B61EB0501B0F57A7F71F100010F
:10D6C000F5D3013EEFD13868032301AA1021FBF7FF
:10D6D0005FFC0A26FFF7DEFC04460D46FFF7DAFC86
:10D6E000001B61EB0501B0F57A7F71F10001F5D304
:10D6F000013EEFD19DF804209DF805009DF806102D
:10D70000194B803280308031A3F88023A3F8820344
:10D710003246A3F8841338680A21FBF747FA0A2631
:10D72000FFF7B8FC04460D46FFF7B4FC001B61EBA5
:10D730000501B0F57A7F71F10001F5D3013EEFD11B
:10D740000DF1030238680221FCF78CF80DF1030299
:10D7500038680921FCF786F8386811220A21FBF79E
:10D7600025FA012003B0F0BD887F0020F0B500222B
:10D7700083B007460A210068FBF718FA1426FFF762
:10D7800089FC04460D46FFF785FC001B61EB050193
:10D79000B0F57A7F71F10001F5D3013EEFD1386821
:10D7A0000F220A21FBF702FA0A26FFF773FC044650
:10D7B0000D46FFF76FFC001B61EB0501B0F57A7FAA
:10D7C00071F10001F5D3013EEFD13868032301AABE
:10D7D0001021FBF7DDFB0A26FFF75CFC04460D4633
:10D7E000FFF758FC001B61EB0501B0F57A7F71F182
:10D7F0000001F5D3013EEFD1324638680A21FBF72C
:10D80000D5F90A26FFF746FC04460D46FFF742FC11
:10D81000001B61EB0501B0F57A7F71F10001F5D3D2
:10D82000013EEFD10DF1030238680221FCF71AF82E
:10D830000DF1030238680921FCF714F83868012259
:10D840000A21FBF7B3F9012003B0F0BDF8B5782247
:10D85000074600210068FBF7A9F90526FFF71AFC27
:10D8600004460D46FFF716FC001B61EB0501B0F501
:10D870007A7F71F10001F5D3013EEFD138682022A3
:10D880000121FBF793F90526FFF704FC04460D463A
:10D89000FFF700FC001B61EB0501B0F57A7F71F129
:10D8A0000001F5D3013EEFD1324638680221FBF783
:10D8B0007DF96426FFF7EEFB04460D46FFF7EAFB11
:10D8C000001B61EB0501B0F57A7F71F10001F5D322
:10D8D000013EEFD10120F8BD70B52422044641215C
:10D8E0000068FBF763F990B90526FFF7D3FB044600
:10D8F0000D46FFF7CFFB001B61EB0501B0F57A7F0A
:10D9000071F10001F5D3013EEFD1012070BD206817
:10D9100020223021FBF74AF90028E5D020680622B2
:10D920003121FBF743F90028DED0206800223421A2
:10D93000FBF73CF9D8E700BFF8B5072207460A21F4
:10D940000068FBF733F90526FFF7A4FB04460D46F4
:10D95000FFF7A0FB001B61EB0501B0F57A7F71F1C9
:10D960000001F5D3013EEFD1386824224121FBF7B5
:10D970001DF90526FFF78EFB04460D46FFF78AFBCF
:10D98000001B61EB0501B0F57A7F71F10001F5D361
:10D99000013EEFD13868C0224221FBF707F9052686
:10D9A000FFF778FB04460D46FFF774FB001B61EBA5
:10D9B0000501B0F57A7F71F10001F5D3013EEFD199
:10D9C0000120F8BDF8B50122074610210068FBF7D9
:10D9D000EDF800B9F8BD1426FFF75CFB04460D46D0
:10D9E000FFF758FB001B61EB0501B0F57A7F71F181
:10D9F0000001F5D3013EEFD13868A022BDE8F84020
:10DA00001121FBF7D3B800BFF0B583B00023074660
:10DA10008DF802301426FFF73DFB04460D46FFF754
:10DA200039FB001B61EB0501B0F57A7F71F1000154
:10DA3000F5D3013EEFD131460DF102023868FBF714
:10DA400011FF0DF1020280213868FBF70BFF4FF444
:10DA5000F842ADF8042038688DF80660032301AA67
:10DA60006021FBF7C5F91426FFF714FB04460D46A9
:10DA7000FFF710FB001B61EB0501B0F57A7F71F138
:10DA80000001F5D3013EEFD131460DF103023868B4
:10DA90008DF80360FBF7E6FE4CF26243ADF804300C
:10DAA00004238DF806303868032301AA6021FBF7B0
:10DAB0009FF91426FFF7EEFA04460D46FFF7EAFA3F
:10DAC000001B61EB0501B0F57A7F71F10001F5D320
:10DAD000013EEFD131460DF1030238688DF8036045
:10DAE000FBF7C0FE4FF4E853ADF8043008238DF87F
:10DAF0000630386801AA03236021FBF779F9142660
:10DB0000FFF7C8FA04460D46FFF7C4FA001B61EBA5
:10DB10000501B0F57A7F71F10001F5D3013EEFD137
:10DB20000DF10302314638688DF80360FBF79AFE69
:10DB300038680DF102021E21FBF794FE012003B0AC
:10DB4000F0BD00BF2DE9F047C2B282B00E233121F3
:10DB50000220FCF795FDDFF85CA10746CAF8240116
:10DB6000002864D00321FAF777FF4FF00008C14680
:10DB70003226FFF78FFA04460D46FFF78BFA001B9B
:10DB800061EB0501B0F57A7F71F10001F5D3013E3B
:10DB9000EFD19F23019397F91030404C8DF801602D
:10DBA00003EB830304EB8303D3F8CC01BB689A0730
:10DBB00058D504230DEB030269465DF061FFBB6895
:10DBC0009B0738D59DF802109DF80130344A0902B0
:10DBD000002741EA03419DF803302780C4E901771B
:10DBE0001943304BA781994204D1B2F80480B2F8AE
:10DBF0000690012752F8083F002BF4D1002F44D0A3
:10DC0000A4F80080A4F80C90B8F1000F3DD04FEAC2
:10DC10000922A37302FB08F3C4E90123B3F1807F57
:10DC20004FF48072628032D801238AF82831384656
:10DC300002B0BDE8F0871C4B1C491A681C4B4FF41E
:10DC4000FA7000FB02F2A3FB0232486892094B68AB
:10DC50001B1A9A42FBD27B69002BB3D01A689B88AF
:10DC60001383AFE77B6913B11A689B8853830E4B0C
:10DC70000E491A680E4B4D68D200A3FB023292097E
:10DC80004B685B1B9A42FBD293E70027CFE7012347
:10DC9000B7208AF83031F9F78DFDC5E7CC150020A3
:10DCA0006C7507081620C200CC3A0020001000E076
:10DCB000D34D6210887F00202DE9F041C2B282B0BE
:10DCC0000E2332210220FCF7DBFCDFF8A48007469C
:10DCD000C8F8340168B3002301933226FFF7DAF95C
:10DCE00004460D46FFF7D6F9001B61EB0501B0F5C0
:10DCF0007A7F71F10001F5D3013EEFD104230DEBE2
:10DD000003029F213846FBF743F99DF806309DF842
:10DD10000510154A1B0243EA01439DF807100B4307
:10DD2000934209D0C8E91A66A8F86460A8F8706040
:10DD3000304602B0BDE8F0810C4BC8F864300126D3
:10DD400040214FF400324FF00063C8E91A23A8F8CD
:10DD5000701088F8726088F83861FAF78FF83046EA
:10DD600002B0BDE8F08100BF21AAEF000004000866
:10DD7000887F002070B5006801220921FAF716FF9C
:10DD80006426FFF787F904460D46FFF783F9001B69
:10DD900061EB0501B0F57A7F71F10001F5D3013E29
:10DDA000EFD170BD2DE9804883B0431C0193DFF8AB
:10DDB00030810A230093D8F88011D8F88C31B8F854
:10DDC0008401B8F89021DDF804B048834FF0320A9E
:10DDD0001A834FF00509D8F88031B8F884215969C1
:10DDE0000A4214BF5A831A83D8F88C31B8F89021AC
:10DDF00059690A4214BF5A831A8356465746FFF799
:10DE000049F904460D46FFF745F9001B61EB050192
:10DE1000B0F57A7F71F10001F5D3013FEFD1D8F869
:10DE20008031B8F8842159690A4214BF5A831A8391
:10DE3000D8F88C31B8F8902159690A4214BF5A8336
:10DE40001A83FFF727F904460D46FFF723F9001B55
:10DE500061EB0501B0F57A7F71F10001F5D3013E68
:10DE6000EFD1B9F1000F1CD0B9F10109B3D14FF4D2
:10DE7000FA76FFF70FF904460D46FFF70BF9001B82
:10DE800061EB0501B0F57A7F71F10001F5D3013E38
:10DE9000EFD14FF0FA0ABBF1000F07D04FF00009A5
:10DEA00099E70BF1FF3BBBF1000FF7D14FF47A7606
:10DEB000FFF7F0F804460D46FFF7ECF8001B61EBA6
:10DEC0000501B0F57A7F71F10001F5D3013EEFD184
:10DED000009B013B00937FF46EAFFFF765F800BF36
:10DEE000002A0020437A5A1C0344D2B2427299722B
:10DEF000037A934200D97047002AFCD010B504463B
:10DF000004F10A01D0E9003098470023637210BD84
:10DF10002E4E3568F06880B529F06AFE284629F053
:10DF200067FEF76879798B0747D500210846FCF72B
:10DF3000A3FF00210120FCF79FFF254C3B683846DA
:10DF40005B68984758B92B6828465B689847F8B9CA
:10DF5000F7683B6838465B6898470028F3D0F0685C
:10DF6000D4F88C210368B4F89011DB68518398478A
:10DF70002B6801461B6828469847D4F88C31B4F8C2
:10DF800090211A832B6828465B6898470028DFD0C9
:10DF9000D4F880212B68B4F88411DB6851832846BB
:10DFA00098470146F06803681B689847D4F88031A9
:10DFB000B4F88421F7681A83C0E73B6838469B6948
:10DFC00041F002019847F768AFE700BF60A4002066
:10DFD000002A00201D4B30B59E4684461D461C4637
:10DFE000BEE80F00CCF80000CCF80410BEE8030037
:10DFF000CCF80820CCF80C30CCF81000CCF8141079
:10E000000FCDCCF81A00CCF81E1003CDCCF822208E
:10E01000CCF82630CCF82A00CCF82E100FCCBEF865
:10E0200000E0ACF818E0ACF832E0CCF83400CCF802
:10E03000381003CCCCF83C20CCF84030ACF84CE0A5
:10E04000CCF84400CCF8481030BD00BF4C7607082F
:10E050000FB410B582B004AB0B4C53F8042BA06B7B
:10E060000A4901935DF034FEA46B627A32B1D4E9BF
:10E07000003004F10A0198470023637202B0BDE842
:10E08000104004B0704700BF60A40020E5DE000827
:10E09000F8B504460F46164600252046202166F0B6
:10E0A000EFFA0446C8B10378202B03D114F8013FDE
:10E0B000202BFBD02046F8F791F9B0F5617F10DBFB
:10E0C00040F63403984211DD30231A46C5B17B7007
:10E0D0003378013333702046F8BD002DFBD1012584
:10E0E000DBE700231A46002DF1D109E0074AA0F52D
:10E0F0006173A2FB0323DA08C3F3C703002DE6D143
:10E100003A70337801333370E9E700BF1F85EB5174
:10E1100070B5054608460E4666F0F2FB31460446E9
:10E1200002462846F7F73EFE68B92B5DA3F13002A0
:10E13000092A00D870BD23F02003413B192BF9D9DF
:10E140000134281970BD002070BD00BF70B110B53A
:10E1500004798C4209D344799442964605D30368E6
:10E16000DB6813B1BDE81040184710BD704700BF11
:10E1700038B190F806C08C4503D303681B6903B11E
:10E180001847704718B103685B6903B118477047B7
:10E1900018B10368DB6903B118470020704700BF5E
:10E1A00018B103681B6A03B118470020704700BF0D
:10E1B00038B50B4D0C4620B10368DB6A0BB19847AC
:10E1C00060B90020C4E90000C4E90200C4E90655B2
:10E1D0002D2230232061227584F8203038BD00BF05
:10E1E0009C7008080178F1B1F8B50F4F054600267C
:10E1F00002E015F8011FA9B1BC6B637A5A1C2344D5
:10E20000D2B262729972237A9342F2D804F10A016F
:10E21000002AEED0D4E900309847667215F8011F45
:10E220000029E9D1F8BD704760A4002070B504460C
:10E230000E48FFF7D7FF2046FFF7D4FF0C48FFF743
:10E24000D1FF0C4B9E8F16B970BD013EFCD0FEF77E
:10E2500021FF04460D46FEF71DFF001B61EB050183
:10E26000B0F57A7F71F10001F5D3EEE7801C080864
:10E27000147B080860A4002070B50E4C05460E46BD
:10E280000D48FFF7AFFF2A460C49A06B33465DF0FF
:10E290001FFDA56B6A7A32B12B68686805F10A0127
:10E2A000984700236B7294F83E3013B1012384F831
:10E2B0003F3070BD60A40020881C0808E5DE00081F
:10E2C0000FB470B582B006A951F8040B0191FFF7A5
:10E2D000D3FF0E48FFF786FF0D4B9E8F36B902B075
:10E2E000BDE8704004B07047013EF8D0FEF7D2FEA2
:10E2F00004460D46FEF7CEFE001B61EB0501B0F5AE
:10E300007A7F71F10001F5D3EEE700BF147B0808B6
:10E3100060A4002070B5C379044603F007008CB0F8
:10E320001546062800F29B80DFE800F0092433350B
:10E33000384004004F480CB0BDE8704088E60E78C5
:10E3400013F0C0031BD0402B21D13146237A462B3A
:10E350005FD8494A02EBC30393F8B821914258D2DF
:10E36000D3F8B43153F82100002852D00CB0BDE8E6
:10E3700070406DE613F0C00391F90060E3D13F48AF
:10E380003146FFF765FE15B1E3793F2B4FD90CB04D
:10E3900070BD0E88D4E7B1F90060D1E7096813F0C9
:10E3A000C0030E463FD0402BD0D0F0E791ED000ADD
:10E3B0006846F7F7EFFE01462E48FFF749FE002DAD
:10E3C000E5D0E3793F2BE2D8237A2B4D05EB83038D
:10E3D0006846B3F91C3000EE103AB8EEC00AF7F701
:10E3E000D9FE01462648FFF733FEE37903F0C00368
:10E3F000402B2BD0637A05EB830595ED070AB8EE29
:10E40000400A6846F7F7C6FE01461D48FFF720FEA2
:10E41000BDE7694620461CF08BFC1A486A46314627
:10E42000FFF74EFFB3E71848FFF712FEABE7217A7C
:10E43000114B627A154803EB820203EB8103D26928
:10E44000B3F91C100CB0BDE8704001E6237A05EB6F
:10E45000C30595F8B831013B00EE103ACFE713F051
:10E46000C00304D0402B92D100210E466EE71E4619
:10E4700085E700BFF02B08084C7607081828080825
:10E48000305608089C1C08080C220808941C080830
:10E49000002841D00378002B3ED02DE9F04F87B003
:10E4A000594905AA62F0E8FC0446002800F0A18062
:10E4B0004FF0000BDFF880A1DFF88091DFF8488192
:10E4C0005D465F464FF0FF360FE0BBF1000F03D112
:10E4D0002046F7F783FF064605AA4146002062F072
:10E4E000CBFC0BF1010B0446E8B1BBF1010F15D0D9
:10E4F000BBF1020FE9D15146204666F00BF8002827
:10E500005FD045F001054946204666F003F8002833
:10E5100050D045F00205DFE73C48D1E62046F7F74A
:10E520005DFF0746D8E770B2394A002392F9001020
:10E53000814225D00133072B02F10C02F6D1002FC6
:10E5400046D0002D08BF03250023EDB2CDE90153CD
:10E5500000971A46194629F0DBF8044600284ED0E9
:10E560002C48DFF8DC803A463146F7F749FA314665
:10E570002948F7F745FAD8F80000214658F082FEFE
:10E58000DFF8BC8003EB430308EB83035C6C002CD7
:10E59000D5D022483146F7F733FA15B16179A9424F
:10E5A0001DD1E36A002BE2D01D48F7F729FA0023BA
:10E5B000E362DCE71B49204665F0ACFF0028A8D1E8
:10E5C0008AE71949204665F0A5FF002899D19AE706
:10E5D00016483146F7F714FA07B0BDE8F08F2A461F
:10E5E0001348F7F70DFA2368E9B29B69204698476C
:10E5F000D7E74FF0FF3025462746064694E73146D9
:10E600000C48F7F7FDF9E7E7EC710808BC1C0808AF
:10E61000A0A400201C1D08088C1D08083C1D08082B
:10E62000741D0808D01C0808983E0808D41C080867
:10E63000541D0808FC1C0808C81C0808CC1C080845
:10E6400060A40020A0B32DE9F04F037887B0054601
:10E650003BB300F10040514C0138294603E09F4292
:10E660002AD1814212D011F8013BA3F14102192AAB
:10E6700014F8012BA2F1410698BF2033192E02F1A4
:10E680002007ECD99A4217D1002BEAD1444B002243
:10E69000C3F8202E83F8292EA3F8272E07B0BDE853
:10E6A000F08F0021012007B0BDE8F04F58F044BEC4
:10E6B0000021012058F040BE3A4C294603E09F4219
:10E6C0001AD1814212D011F8013BA3F14102192A5B
:10E6D00014F8012BA2F1410698BF2033192E02F144
:10E6E0002007ECD99A4207D1002BEAD1012007B0CC
:10E6F000BDE8F04F4BF008BC2B4C294603E09F428D
:10E7000058D1814212D011F8013BA3F14102192ADC
:10E7100014F8012BA2F1410698BF2033192E02F103
:10E720002007ECD99A4245D1002BEAD11C4B00229C
:10E7300093F9274E83F8202E1846164693F8D214E4
:10E740000129A1F1030509D0052D07D90EB180F8E3
:10E75000274E164807B0BDE8F04FB1E593F8D31443
:10E76000A52903F1140303D00132782AE6D1EDE79D
:10E77000012C03D0013C64B20126F5E70C4980F876
:10E78000204E0023013280F8212E81F8943080F849
:10E79000273E07B0BDE8F04F4BF018BCBC1D080881
:10E7A00038930020C41D0808882D0808BC1C0808E0
:10E7B00060A40020DFF8C8B22846F7F70FFE9BF9E7
:10E7C00094A00AFA80F6772E074600F2DB802846EE
:10E7D000202165F055FF0446002800F02A810378C7
:10E7E000202B03D114F8013F202BFBD02046F7F754
:10E7F000F5FD01255FFA80F82046202165F040FFF5
:10E800000446002800F013810378202B03D114F86C
:10E81000013F202BFBD02046F7F7E0FD01350190AA
:10E82000EDB22046202165F02BFF0446002800F0C1
:10E83000FC800378202B03D114F8013F202BFBD060
:10E840002046F7F7CBFD01350290EDB2204620219E
:10E8500065F016FF0446002800F0E5800378202BC1
:10E8600003D114F8013F202BFBD02046F7F7B6FD6B
:10E8700001350390EDB22046202165F001FF0446EA
:10E88000002800F0CE800378202B03D114F8013F3C
:10E89000202BFBD02046F7F7A1FD013503B20493EE
:10E8A000EDB22046202165F0EBFE0446002800F082
:10E8B000B0800378202B03D114F8013F202BFBD02C
:10E8C0002046F7F78BFD20210346204605931CB216
:10E8D00065F0D6FE0135059BEDB20246002859D001
:10E8E0001378202B03D112F8013F202BFBD01046C8
:10E8F0000592F7F773FD059A0FFA80F9202110466B
:10E9000065F0BEFE00284CD00378202B03D110F810
:10E91000013F202BFBD0F7F761FD05F0FD05042D2D
:10E9200008BFC3B27FF415AFB8F1010F0AD9B8F12F
:10E93000040F07D0A8F10502032A03D9B8F1030F89
:10E940007FF407AF23B1A52B44D0482B7FF401AF50
:10E95000002E39D1474A82F8276E82F8D284019975
:10E96000C2F8C0140299C2F8C4140399C2F8C814BA
:10E970000499A2F8CC14A2F8CE44A2F8D09482F85C
:10E98000D3348BE63C493D487723002207B0BDE8ED
:10E99000F04F95E4062D7FF4DCAE8146DBB20446F1
:10E9A000C2E7052D7FF4D5AEB8F1010F0AD9B8F151
:10E9B000040F07D0A8F10503032B03D9B8F1030F07
:10E9C0007FF4C7AE0346C3E72A4A06EB860602EB8E
:10E9D0008602C2E786BB2748019AC0F8C024029A83
:10E9E000C0F8C424039AC0F8C824049A80F8D33429
:10E9F00080F8D284A0F8CC24A0F8CE44A0F8D0941B
:10EA000001230AF101023A448BF8942080F8273E52
:10EA100044E6202165F034FE024600287FF460AF12
:10EA200097E604903DE7039025E702900EE70190FA
:10EA3000F7E605468046DFE60E48019906EB8606B6
:10EA400000EB8602C2F8C01482F8D334029990F821
:10EA5000273EC2F8C4140399C2F8C81401330499BC
:10EA600082F8D284A2F8CC14A2F8CE44A2F8D094B2
:10EA70005BB2C6E738930020CC1D0808D81D0808F3
:10EA800060A400202DE9F04782B03C4901AA62F061
:10EA9000F3F9002863D04FF0000A4FF0FF34374DF0
:10EAA000D1465646D0462746BAF1040F37D8DFE89C
:10EAB0000AF0423C310B03000378482B41D0562B1F
:10EAC0002DD14FF0010904E0F7F788FC3F280646F6
:10EAD00025D8002001AA29460AF1010A62F0CCF9E2
:10EAE0000028E1D1BAF1040F2ED0BAF1050F40D1C0
:10EAF000234AB301962103F47C6308F03F0801FB2D
:10EB0000074443EA080302EB440243EA4933A2F80C
:10EB1000983007E0F7F762FC3F288046D9D91948BA
:10EB2000FFF7CEFB02B0BDE8F087F7F757FC95285A
:10EB30000446CED9F3E7F7F751FC03280746C8D9B6
:10EB4000EDE74FF00009C4E70D4A962303FB0743A6
:10EB500002EB4303B3F89890C9F34039C9E74FF08B
:10EB6000FF373C46084923463A46012058F070FCDE
:10EB7000D8E7BAF1030FD2D0F4E700BFEC71080870
:10EB800060A40020BC1C0808F8A400202DE9F04F68
:10EB90008FB0DFF8A8829D4E9D4C0091074603E0A0
:10EBA0000C34444500F0AD80B56B6A7A32B12B6805
:10EBB000686805F10A01984700236B72E27902F058
:10EBC0003803BB42ECD1924BA4EB030C914B4FEAC0
:10EBD000AC0C03FB0CFC1FFA8CFCBCF1150F40F2D3
:10EBE00008818D4D0120162302E0302800F0D580E9
:10EBF00015F8011F0B449BB29C45014600F1010032
:10EC0000F3D2864B03EB4103B3F8EC538448854BB6
:10EC1000834204D3F6E01433834280F0F3801988F2
:10EC2000C1F30B01A942F6D12046D3F808B00192F6
:10EC30001CF03EF981460BEB000A20461CF090F9CF
:10EC4000019A0146009802F0070300F02005062B08
:10EC500014D8DFE803F08088786F59049100D1ED73
:10EC6000007A9AED007AB4EE677AF1EE10FA0CBFF2
:10EC700001230023002D50D0002B91D102AD294655
:10EC800020461CF055F8009B5A0614D566482946C4
:10EC9000FFF7DEF92B68654A934200F0818000227D
:10ECA00051462046FFF736FB6148FFF79BFAB38FCA
:10ECB000002B40F089805F482946FFF7C9F9002200
:10ECC00051462046FFF726FB5948FFF78BFAB38FD2
:10ECD000002B3FF465AF9A46FEF7DCF905468946FE
:10ECE000FEF7D8F9401B61EB0901B0F57A7F71F1AD
:10ECF0000001F5D3BAF1010AEED10C3444457FF49A
:10ED000053AF0FB0BDE8F08F0A685BF809309B1A6B
:10ED1000B3FA83F35B09002DAED102AD294620463C
:10ED200001931CF005F8009B5B06C4D5019B002BEA
:10ED3000C1D1ABE7B1F900203BF909309B1AB3FA16
:10ED400083F35B0996E70A883BF809309B1AB3FA0C
:10ED500083F35B098EE70A781BF809309B1AB3FA34
:10ED600083F35B0986E791F900201BF909309B1AB0
:10ED7000B3FA83F35B097DE702F0C002402A274B18
:10ED800039D0627A03EB8203DA690132504662F0CD
:10ED900021FCB0FA80F35B096CE74FF6FF7535E7AD
:10EDA0002B79002B7FF47BAF1BF80930202B7FF4ED
:10EDB00076AF21485146FFF74BF91D48FFF712FA8D
:10EDC000B38F002B3FF477AF9B460194FEF762F9B7
:10EDD00004468946FEF75EF9001B61EB0901B0F5B8
:10EDE0007A7F71F10001F5D3BBF1010BEED1019CEB
:10EDF00061E70A250AE7227A03EBC20393F8B821F8
:10EE0000013AC2E700239B68FFDE00BF60A4002038
:10EE10003C8A0708ABAAAAAA987A07084C76070882
:10EE2000088C08081C870808041E08086E616D65B8
:10EE3000147B0808F81D0808101E080874A60708A7
:10EE40002DE9F0413B4F3B68002B70D01B6A98477F
:10EE50008368002B50D03848DFF8EC80FFF7C2F908
:10EE60003648FFF7BFF9B8F83C60D6B939F0AEFACA
:10EE70003B6813B15B68984710BB6426FEF70AF93C
:10EE800004460D46FEF706F9001B61EB0501B0F5DF
:10EE90007A7F71F10001F5D3013EEFD1E8E7013E41
:10EEA000E4D0FEF7F7F804460D46FEF7F3F8001B32
:10EEB00061EB0501B0F57A7F71F10001F5D3EEE762
:10EEC0001F48FFF78FF91D48FFF78CF9B8F83C6031
:10EED0001EB9BDE8F081013EFBD0FEF7DBF8044629
:10EEE0000D46FEF7D7F8001B61EB0501B0F57A7F00
:10EEF00071F10001F5D3EEE71248FFF773F90F48FF
:10EF0000FFF770F9104B9E8F002EE2D0FEF7C2F88B
:10EF100004460D46FEF7BEF8001B61EB0501B0F597
:10EF20007A7F71F10001F5D3013EEFD1D1E70748B7
:10EF30008EE700BF508300202C1E0808147B0808B1
:10EF4000381E0808181E080860A4002050A40020DD
:10EF500080B51848184DFFF745F91848FFF742F9F2
:10EF6000AC6B627A32B12146606851F80A3B98472F
:10EF7000002363722F683B6838465B699847B0B9D5
:10EF80000A26FEF787F804460D46FEF783F8001BB5
:10EF900061EB0503B0F57A7F73F10003F5D3013E11
:10EFA000EFD13B6838465B6998470028E8D00120DC
:10EFB00006F002FF401E080860A400205C1E08083E
:10EFC00030B42B4C94F84835012B86B002D006B0F3
:10EFD00030BC704794F84D350A2B04D0254806B054
:10EFE00030BCFFF7FFB82449244A08780092002378
:10EFF000B22103228DF80400CDF80730CDF80B3094
:10F00000CDF80F30ADF813308DF805108DF80620CF
:10F010000DF1FF3C0DF1120541F221001CF8012F0A
:10F02000082183EA02231AB2002A4FEA4303B6BF3B
:10F0300080EA42029BB293B20139F4D1AC45EDD1E2
:10F04000C3F307228DF814308DF81320EC461523F6
:10F05000C4F8B835BCE80F00094D0FC59CE80300A3
:10F0600045F8040B0748297006B030BCFFF7BAB862
:10F0700060A40020681E080834180020A64115EB83
:10F08000C8A90020781E080880B52D482D4FFFF72D
:10F09000A9F82D48FFF7A6F8BE8F002E40D1BC6B13
:10F0A000627A32B12146606851F80A3B98470023E2
:10F0B0006372002587F8BC55C7F8FC5587F80056E1
:10F0C00023F042F92148FFF78DF8BC6B627A2AB130
:10F0D0002146606851F80A3B984765723F683B6873
:10F0E00038465B699847B0B90A26FDF7D3FF044656
:10F0F0000D46FDF7CFFF001B61EB0503B0F57A7FEE
:10F1000073F10003F5D3013EEFD13B6838465B69EC
:10F1100098470028E8D0002006F04EFE013EBED001
:10F12000FDF7B8FF04460D46FDF7B4FF001B61EB89
:10F130000501B0F57A7F71F10001F5D3EEE700BF6C
:10F14000941E080860A40020147B08085C1E0808B0
:10F15000F8B5324C94F83E301BB194F83F30002B98
:10F160004FD12F48FFF73EF8012384F8073684F883
:10F170003C36F7F719FC40B9F7F716FC28B9F7F752
:10F1800013FC10B90520FEF70DFEF7F799FB0028D8
:10F19000F8D0244B24481A68C4F81426002601230A
:10F1A00084F83C6684F8076684F83236FFF71AF86C
:10F1B000A56B6A7A2AB1D5E9003005F10A019847B2
:10F1C0006E7227683B6838465B699847B0B90A2673
:10F1D000FDF760FF04460D46FDF75CFF001B61EB89
:10F1E0000501B0F57A7F71F10001F5D3013EEFD151
:10F1F0003B6838465B6998470028E8D0002006F055
:10F20000DBFD0A48FFF75CF80948FFF759F80023CF
:10F2100084F83E3084F83F30F8BD00BF60A4002081
:10F22000181F0808083600205C1E0808C01E0808C1
:10F23000F81E0808F8B5394B394F1B68D7F8404617
:10F24000002B69D01B6A9847A28861884468521ACB
:10F2500002FB0444002C4AD03248FEF7C3FF324878
:10F26000FEF7C0FF3148FEF7BDFFBE8F86BB3048BA
:10F27000FEF7B8FFBC6B627A002A45D14FF47A766C
:10F28000FDF708FF04460D46FDF704FF001B61EB88
:10F290000501B0F57A7F71F10001F5D3013EEFD1A0
:10F2A000386828F0A5FC234B1A784AB12249304629
:10F2B00051F836300BB19B68186001369642F7D191
:10F2C00002210120F5F73CF9FDF75AFE013ECED0B0
:10F2D000FDF7E0FE04460D46FDF7DCFE001B61EB8A
:10F2E0000501B0F57A7F71F10001F5D3EEE713481F
:10F2F000FEF778FFBD6B6A7A2AB12B68686805F162
:10F300000A0198476C72F8BD2368606804F10A012D
:10F31000984700236372B1E7094895E750830020BE
:10F3200060A40020801C0808201F0808147B08081F
:10F330005C1E08089000001040410020401F080893
:10F3400050A400202DE9F84F1A4FDFF870A0DFF825
:10F3500070B0DFF8709007F5407802E0103747454D
:10F3600026D03868FEF73EFF796811B15846FEF79F
:10F370006FFEB96811B11048FEF76AFE4846FEF705
:10F3800031FFBAF83C60002EE8D0FDF783FE04465A
:10F390000D46FDF77FFE001B61EB0501B0F57A7F9E
:10F3A00071F10001F5D3013EEFD110374745D8D1B7
:10F3B000BDE8F88FC87A0708781F080860A4002005
:10F3C000701F0808147B080870B50C48FEF70AFF88
:10F3D0000B4B9E8F16B970BD013EFCD0FDF75AFE57
:10F3E00004460D46FDF756FE001B61EB0501B0F526
:10F3F0007A7F71F10001F5D3EEE700BF147B0808B6
:10F4000060A4002070B525490522044665F036FA4F
:10F4100010BB234C94F83E3023B9012284F83E20DF
:10F4200084F83F301F48FEF7DDFE1F48FEF7DAFE86
:10F43000A68F16B970BD013EFCD0FDF72BFE044629
:10F440000D46FDF727FE001B61EB0501B0F57A7F45
:10F4500071F10001F5D3EEE714490322204665F06F
:10F460000DFAA8B90E4C94F83E3013B194F83F3021
:10F4700053B90F48FEF7B6FEFFF7A6FF002384F846
:10F480003E3084F83F3070BD0A48FEF719FFF5E7BB
:10F49000BDE870400848FEF713BF00BF801F080892
:10F4A00060A40020881F0808147B08081C36080880
:10F4B000A01F0808C01E0808B41F0808800601D550
:10F4C000002930D10CB470B5184C1949A06B82B02A
:10F4D00007AB069A01935CF0FBFBA56B6A7A32B12D
:10F4E0002B68686805F10A01984700236B72114880
:10F4F000FEF778FEA68F3EB9012002B0BDE870404D
:10F5000002B07047013EF7D0FDF7C4FD04460D463A
:10F51000FDF7C0FD001B61EB0501B0F57A7F71F1CD
:10F520000001F5D3EEE70020704700BF60A4002083
:10F53000E5DE0008147B0808F0B5064683B060B32A
:10F5400004785CB300F1004E444C0EF1FF3E0146DE
:10F5500003E0984236D1714513D011F8013BA3F175
:10F560004102192A14F8012BA2F1410C98BF203353
:10F57000BCF1190F02F12000EBD99A4222D1002BE5
:10F58000E9D1374B374AC3F84426C3F84826C3F8B5
:10F590004C26C3F8502603B0F0BD0446324D334E1E
:10F5A00035F8243005EB8402002152880120CDE992
:10F5B0000032234632460134FFF780FF042CEFD19E
:10F5C00003B0F0BD3046F6F709FF0328074639D8E7
:10F5D0002021304665F054F8044600283BD00378DB
:10F5E000202B03D114F8013F202BFBD02046F6F747
:10F5F000F5FE012605462021204665F041F8D8B1E8
:10F600000378202B03D110F8013F202BFBD0F6F715
:10F61000E5FE8EB1A5F2EE2240F2DC539A420BD801
:10F62000A0F2EE229A4207D80D4B03EB8703A3F812
:10F630004456A3F84606AEE70D4803B0BDE8F040D7
:10F64000FEF73EBE0B490C480323002203B0BDE881
:10F65000F040FEF735BE0646CDE700BFBC1D0808EA
:10F6600060A40020E803D007A4AA0020C41F080853
:10F67000BC1C0808D81F0808D81D08082DE9F0434D
:10F6800085B040B3037806462BB300F1004C574CCD
:10F690000CF1FF3C014603E0984232D1614512D0A3
:10F6A00011F8013BA3F14102192A14F8012BA2F130
:10F6B000410598BF2033192D02F12000ECD99A4260
:10F6C0001FD1002BEAD14A486022002105B0BDE8D5
:10F6D000F04363F05DB8464D464E0024D5E9012164
:10F6E00015F80C3B0093CDE9012123463246002159
:10F6F00001200134FFF7E2FE082CEFD105B0BDE890
:10F70000F0833046F6F76AFEC3B2072B054657D89A
:10F710002021304664F0B4FF0446002859D0037815
:10F72000202B03D114F8013F202BFBD02046F6F705
:10F7300055FE071E18BF012701262046202164F030
:10F740009FFF044600284ED00378202B03D114F8E5
:10F75000013F202BFBD02046F6F740FE01368046C5
:10F76000F6B22046202164F08BFF0446A0B3037854
:10F77000202B03D114F8013F202BFBD02046F6F7B5
:10F780002DFE0136814620212046F6B264F078FF36
:10F7900008B10136F6B2032E05D0174805B0BDE812
:10F7A000F043FEF78DBD154B6DB205EB450503EB40
:10F7B000850383F85476C3F85886C3F85C969DE7B2
:10F7C0000F4910480723002205B0BDE8F043FEF7BB
:10F7D00077BD06460746B0E7202164F051FFA146F9
:10F7E0000028D6D1D9E78046BBE700BFBC1D08087A
:10F7F000B4AA0020E01F0808BC1C080860A4002070
:10F80000F81F0808D81D080870B588B0002841D036
:10F8100003780446002B3DD000252D2B54D0A3F1B6
:10F820003002092A50D9202B62D163780134002B91
:10F83000F3D1052DBDF914305AD19AB20F2A57D8F9
:10F84000BDF91610A1F5FA7292B2B2F5FA6F4FD85F
:10F85000BDF91800A0F5FA7292B2B2F5FA6F47D866
:10F86000BDF91A40A14243DCA04241DBBDF91C5066
:10F8700005F17D0292B2FA2A3AD8204A02EBC3037C
:10F88000A3F8B416A3F8B606A3F8B84683F8BA5698
:10F8900008B070BD1A4C1B4E002594F90600B4F94F
:10F8A0000410B4F9022034F9083BCDE90210CDE987
:10F8B000003200212B46324601200135FFF7FEFDC4
:10F8C000102DEAD108B070BD042D11DC2046F6F7EA
:10F8D00085FD08AB03EB4503013523F80C0C14F848
:10F8E000013FA3F13002092AF9D9002B95D1A0E7F5
:10F8F000054808B0BDE87040FEF7E2BC60A40020F7
:10F9000014AB002008200808BC1C080870B58AB099
:10F91000064664F0F5FF10F0FF0414D13B4D3C4E59
:10F92000AB68D5E900210120CDE9012100933246E1
:10F93000234600210134FFF7C1FD082C05F10C0519
:10F94000EED10AB070BD334C06F1050C314603E030
:10F9500098422AD1614512D011F8013BA3F141022E
:10F96000192A14F8012BA2F1410598BF2033192D53
:10F9700002F12000ECD99A4217D1002BEAD1264897
:10F98000264A904238BF40F2FF3103D3D9E7143002
:10F990009042D6D20388C3F30B038B42F7D11B49A5
:10F9A0000AB0BDE87040F7F7D5B91D4905AA304641
:10F9B00061F062FA78B11A4E06AD0024F6F70EFD3A
:10F9C00005AA45F8040B31460020013461F054FAD1
:10F9D00030B1042CF2D11348FEF772FC0AB070BDAE
:10F9E000042CF8D1069B072BF5D80849DDE9074020
:10F9F00003EB430301EB830241F823009460099B6E
:10FA000009485360FFF782FF9BE700BF94AB0020DB
:10FA100020200808BC1D08081C870808088C080856
:10FA2000EC710808BC1C0808207908082DE9F04191
:10FA300084B0584903AA61F01FFA00286ED0F6F787
:10FA4000CDFC0D2805462AD8524903AA002061F0B2
:10FA500013FA002864D05049504E044603E09E45F6
:10FA600023D1B14213D011F8013BA3F14102192A6D
:10FA700014F8012BA2F1410C98BF2033BCF1190FEF
:10FA800002F1200EEBD99A420FD1002BE9D10024CC
:10FA9000404903AA002061F0EFF900285DD04048FA
:10FAA000FEF70EFC04B0BDE8F0813E493E4F04462F
:10FAB00003E09C4516D1B94212D011F8013BA3F1E5
:10FAC0004102192A14F8012BA2F1410698BF2033F4
:10FAD000192E02F1200CECD99A4203D1002BEAD165
:10FAE0000124D5E73149324F03E09E42D7D1B942D4
:10FAF00012D011F8013BA3F14102192A10F8012B91
:10FB0000A2F1410498BF2033192C02F12006ECD950
:10FB10009A42C4D1002BEAD10224B9E74FF0FF3555
:10FB2000DFF89880234F244E00240EE03B5D08EB65
:10FB300083033246D3F87C3700930021234601200B
:10FB40000134FFF7BBFC0E2CACD06B1CEED0A542F1
:10FB5000ECD001340E2CFAD1A4E7164B174E164FF9
:10FB60005C555C19854200F1010002D00E28F9D1E4
:10FB700098E7237806EB83033A46D3F87C37009363
:10FB800000212B460120FFF799FC0D2D05F1010006
:10FB9000E8D187E7EC71080834200808332008888A
:10FBA000BC1C08083C2008083B200888346F080863
:10FBB000336F0888B48B0020442008084C7607086F
:10FBC00010F040002FD00CB470B50C4682B029B1B3
:10FBD000002002B0BDE8704002B07047174EB56B10
:10FBE0006B7A5A1C2B44D2B223216A7299722B7AF7
:10FBF000934219D9069A124907AB284601935CF043
:10FC000067F8B46B627A32B1D4E9003004F10A01CA
:10FC1000984700236372FFF7D7FB012002B0BDE8CD
:10FC2000704002B070477047002AE3D0D5E9003039
:10FC300005F10A0198476C72B56BDBE760A4002000
:10FC4000E5DE00082DE9F04FDFF8F0A087B093461D
:10FC500081460D46164600270AF28C744FF01908AB
:10FC600095F800C0BBF1000F52D03078604551D0FC
:10FC70000021002302E00133392B5AD004EBC302E8
:10FC80004FEAC30C12798242F5D1F37805914FF413
:10FC9000617218FB03230393B378D44418FB032346
:10FCA00002939CF8913772784846CDE90032224A97
:10FCB0003B46FFF785FF95F800C00599002302E059
:10FCC0000133392B35D004EBC302D80012796245D9
:10FCD000F6D1EB784FF4617218FB03230393AB78F2
:10FCE000504418FB032302936A7890F891374846F2
:10FCF000CDE900323B46104A0137FFF7DFFB282FE2
:10FD000005F1040506F10406AAD107B0BDE8F08F9D
:10FD10005946D3E76A7873789A42A9D1AA78B3781A
:10FD20009A42A5D1E978F378C91AB1FA81F1490963
:10FD30009FE700235B79FFDE5C2008084C7607080C
:10FD4000002871D0F0B5037883B00446002B43D06F
:10FD5000F6F744FB272805466ADC0023601C2021B7
:10FD60008DF8073064F08CFCAE00044658B103787F
:10FD7000202B03D114F8013F202BFBD02046F6F7AF
:10FD80002DFB002834DA2046202164F079FC04465B
:10FD9000A0B10378202B03D114F8013F202BFBD016
:10FDA0002046F6F71BFB152808D8264B334483F86A
:10FDB00095079DF8073001338DF80730224FB11CAD
:10FDC0000DF1070239442046FEF762F99DF807302D
:10FDD000042B08D103B0F0BD1B490022012003B061
:10FDE000BDE8F0402EE7002347F8253003B0F0BD12
:10FDF000164FC2B2002307F28C7001E0392BC2D03B
:10FE000000EBC3014FEAC30C4979914203F10103AE
:10FE1000F4D101238DF807300A4B6744334497F837
:10FE2000902783F89427AEE707490022012009E7CD
:10FE3000074908482723002203B0BDE8F040FEF739
:10FE40003FBA00BF60A40020F4AB00204C76070846
:10FE500070200808D81D08082DE9F04F89B0434EDE
:10FE6000434F079092460C46154602F1540894F908
:10FE70000430404A92F90010994202F10C0209D074
:10FE80009642F7D10C35454504F10C04EFD109B089
:10FE9000BDE8F08FBAF1000F51D095F904E0D5F824
:10FEA00000B06A79A879297A95F807C0734548D0D7
:10FEB0004FF0000907EB8C0C07EB8101DCF854399B
:10FEC000049307EB8000D1F85439039307EB8202C7
:10FED000D0F854390293D2F854390193264A07983E
:10FEE000CDF800B073464946FFF76AFE94F9043036
:10FEF000E279D4F800C007EB82024946D2F85429CF
:10FF00000492227A07EB82020C35D2F8542903922C
:10FF1000A27907EB82020C34D2F85429029214F829
:10FF2000070C154ACDF800C007EB8000D0F8540943
:10FF300001900798FFF7C2FA454598D1A7E7D14647
:10FF4000D6E723685B45B3D163799342B0D1A379F7
:10FF50008342ADD1237A8B42AAD194F80790A9EBC2
:10FF60000C09B9FA89F94FEA5919A3E7F4A400205A
:10FF70004C760708A0A4002078200808D8B10278A1
:10FF8000CAB12DE9F04F87B0451CF6F727FA5A4C55
:10FF9000014647B22246002392F90460BE4202F1B4
:10FFA0000C020CD00133072BF6D1544807B0BDE842
:10FFB000F04FFEF785B95049002201204CE703EBD2
:10FFC000430304EB830494E8070003AE86E80700CC
:10FFD00007462021284664F053FB834600287DD045
:10FFE0000278202A03D11BF8012F202AFBD02B2ACC
:10FFF00039D02D2A66D05846F6F7F0F90223074685
:020000040801F1
:100000000093E37994F8059094F8068094F808A09A
:10001000019300255846202164F032FB83460028D6
:1000200045D00278202A03D11BF8012F202AFBD0CB
:100030005846F6F7D3F9002203461146304804E04B
:100040000132112A1AD050F8041F9942F8D1022D1A
:100050005FFA82FC16D0032D16D0012D14BFE146A5
:10006000E0460135D6E70BF1010B5846F6F7B6F935
:1000700001228240022317430093C2E7BBB9022D3D
:100080009C46E8D1E246ECE7002369F3070368F3F6
:100090000F236CF317436AF31F630397CDF81130F6
:1000A00096E8070084E8070007B0BDE8F08F009BE2
:1000B0002B44DBB2012B14D1124807B0BDE8F04F3E
:1000C000FEF7FEB80BF1010B5846F6F787F901224F
:1000D0008240022327EA0207009392E7012300935C
:1000E0008FE70023019A69F3070368F30F2362F394
:1000F00017436AF31F63D0E70880002098200808A0
:10010000A07F0708BC1C08082DE9F04F89B0DFF874
:10011000D0A0079281460C46154600264FF01908DC
:100120004FF461773AE0A97894F802B02B786A78B6
:10013000E87895F804C095F805E08B4534D04FF089
:10014000000B18FB027218FB0373CDE90232CDE9F4
:10015000040CCDE900E13346524659464846FFF7C4
:100160002FFD23790593E37804936278237818FBB5
:10017000027218FB0373CDE90232A378019363790D
:10018000009352463346594648460136FFF796F9E2
:10019000142E04F1060405F106051ED0079B002B62
:1001A000C1D1DDF81CB0DCE794F800B09B45C6D1A6
:1001B00094F801B09345C2D194F803B08345BED101
:1001C00094F804B0E345BAD194F805B0ABEB0E0B4C
:1001D000BBFA8BFB4FEA5B1BB3E709B0BDE8F08FBE
:1001E000AC200808002800F0AD802DE9F047037826
:1001F00082B00446002B71D0F6F7F0F813280546BC
:1002000000F3A48000EB40060023601C20218DF841
:10021000073064F035FADFF850814FEA46096F0085
:1002200008EB4606044658B10378202B03D114F896
:10023000013F202BFBD02046F6F7D0F8032877D9D2
:100240002046202164F01CFA044658B10378202B84
:1002500003D114F8013F202BFBD02046F6F7BEF85F
:10026000152859D920460DF107023146FDF710FF38
:10027000202164F005FA0446002870D00378202B72
:1002800003D114F8013F202BFBD02046F6F7A6F847
:100290003B289DF807A032D92046202164F0F0F9D0
:1002A000B0B10378202B03D110F8013F202BFBD0F5
:1002B000F6F794F815280BD82A4B2F440AF1010AB7
:1002C00003EB47035FFA8AFA8DF807A083F8380832
:1002D000BAF1060F09D102B0BDE8F0872249002229
:1002E000012002B0BDE8F0470EE72048002348F89F
:1002F0000930B38002B0BDE8F047FDF7E1BF194B0C
:100300007A190AF1010A03EB42035FFA8AFA8DF8BF
:1003100007A083F83708BFE79DF80720114B01328B
:100320008DF807207A1903EB420383F8360899E722
:100330000C4B7A1903EB420383F8390801238DF83B
:1003400007307DE7084900220120DDE60849094819
:100350001323002202B0BDE8F047FDF7B1BF9DF8BE
:1003600007A099E760A4002094AC0020BC1C0808FA
:1003700070200808D81D08082DE9F04F2DED088BD6
:1003800099B082460C461546002607925DE0F4EED1
:100390004A8AF1EE10FA74D1B4EE6A9AF1EE10FACC
:1003A0006FD1F4EE4B9AF1EE10FA0CBF012100214F
:1003B00014A80691F5F7EEFEB0EE4A0A074610A81B
:1003C000F5F7E8FE0DF130098346B0EE6A0A4846BB
:1003D000F5F7E0FE0DF120080590B0EE4B0A40461F
:1003E000F5F7D8FE059A0390CDE901B206992B4A9C
:1003F000009733465046FFF7E3FBB0EE480A14A8D7
:10040000F5F7C8FEB0EE680A074610A8F5F7C2FE79
:10041000B0EE490A83464846F5F7BCFEB0EE690ADD
:1004200081464046F5F7B6FE3346CDE90290CDE968
:10043000007B1A4A002150460136FFF73FF80C2E88
:1004400004F1100405F1100522D094ED008AB5EEF8
:10045000408AF1EE10FA1BD0079BD4ED018A94ED8F
:10046000029AD4ED039A73B195ED000A95ED01AAB5
:10047000D5ED02AA95ED03BAB4EE408AF1EE10FA7A
:1004800085D0002194E70DF130090DF12008B4E783
:1004900019B0BDEC088BBDE8F08F00BFCC20080878
:1004A0002DE9F04198B30378054683B36E4C00F113
:1004B000050E014603E0984237D1714513D011F87B
:1004C000013BA3F14102192A14F8012BA2F1410CBE
:1004D00098BF2033BCF1190F02F12000EBD99A42EA
:1004E00023D1002BE9D1614A92F8CE1B4FF4C8709A
:1004F00000FB01F102F6AC0302F66C120B440A4455
:10050000002143F8101F9342FBD1BDE8F081574909
:1005100091F8CE3B4FF4C87000FB0311BDE8F041E9
:10052000002201F6BC01012026E72846F5F756FF18
:100530000B28064600F28D802021284664F0A0F8A2
:100540000446002800F08D800378202B03D114F896
:10055000013F202BFBD02046F5F78CFE434A92F852
:10056000CE3B03EB830303EB8303334402EB031221
:1005700002F6BC02012582ED000A2046202164F02B
:100580007FF80446C0B10378202B03D114F8013F53
:10059000202BFBD02046F5F76DFE344A92F8CE3B77
:1005A00003EB830303EB8303334402EB031202F6F2
:1005B000BC02013582ED010A2046202164F060F87A
:1005C0000446C0B10378202B03D114F8013F202B3F
:1005D000FBD02046F5F74EFE244B03F6AC0293F811
:1005E000CE3B03EB830303EB8303334402EB0313A0
:1005F000013583ED060A2021204664F041F8C0B1A0
:100600000378202B03D110F8013F202BFBD0174C8F
:1006100094F8CE7BF5F72EFE07EB870303EB8303FD
:1006200004F6AC04334404EB0313032D83ED070AF3
:1006300004D0BDE8F0410E48FDF742BE4FF4C87348
:1006400003FB074404F110010022BDE8F041012042
:1006500092E6BDE8F041074907480B230022FDF769
:100660002FBE054689E700BFBC1D080860A4002016
:10067000BC1C080870200808D81D08082DE9F04F98
:1006800091B0DFF834B1079282460C4690460025BF
:1006900009AF0BAE3AE01A4643493046F5F7D0F9B8
:1006A000079B002B49D098F800C02378634547D0BA
:1006B0004FF000093D4B059300230493B8F9123025
:1006C0000393B8F910303A4A02930192CDF800C072
:1006D0002B465A4649465046FFF772FA0597237D46
:1006E0000493B4F912300393B4F9102014F8203BAA
:1006F0000093CDE901622B465A46494650460135E2
:10070000FEF7DCFE082D08F120084AD004F1150997
:1007100004224946384664F05FF90022A3688DF848
:100720002820E268082B72F10001B4D32149304639
:10073000F5F786F9079B002BB5D1DDF81C90CDE7C6
:10074000D4E90202D8E902139A4208BF8842AFD125
:10075000227D98F814309A42AAD199F8002098F88E
:1007600015309A42A4D199F8012098F816309A428F
:1007700009F101099CD119F8012F98F817309A4214
:1007800096D199F8012098F818309A4290D12269B0
:10079000D8F81030A2EB0309B9FA89F94FEA5919D0
:1007A00088E711B0BDE8F08F1828080820790808FC
:1007B00040170808E0200808EC20080898B32DE945
:1007C000F04F037883B0804633B300F1004CA54D61
:1007D0000CF1FF3C014603E0984228D1614512D05C
:1007E00011F8013BA3F14102192A15F8012BA2F1DE
:1007F000410798BF2033192F02F12000ECD99A420B
:1008000015D1002BEAD198484FF48072002103B033
:10081000BDE8F04F61F0BCBF93490022012003B056
:10082000BDE8F04F2AE790490022012026E7404624
:10083000F5F7D4FD83B2072B074600F2EE802021A6
:10084000404663F01DFF8146002800F0F8800378E1
:10085000202B03D119F8013F202BFBD04846F5F798
:10086000BDFD01250FFA80F82021484663F008FFFE
:10087000002800F0E7800378202B03D110F8013F17
:10088000202BFBD0002B00F0E7800026014600F172
:10089000100C3446A3F13002D2B2092AA3F1610E42
:1008A0000CD9BEF1050FA3F15702A3F1410E04D9F3
:1008B000BEF1050F11D8A3F13702D2B211F8013FF2
:1008C000240144EA167442EA0616002B00F0B480B4
:1008D000202B00F0B1806145DCD10023019301356C
:1008E000EDB2202163F0CCFE8246002800F0B280F9
:1008F0000378202B03D11AF8013F202BFBD0504660
:10090000F5F76CFD01350FFA80F9EDB25046202164
:1009100063F0B6FE8346002800F09A800378202B0F
:1009200003D11BF8013F202BFBD05846F5F756FDAD
:1009300001350FFA80FAEDB25846202163F0A0FE8F
:100940008346002800F082800278202A03D11BF819
:10095000012F202AFBD05846F5F740FD013543B260
:100960000093EDB25846202163F08AFE034600282A
:100970006AD00278202A03D113F8012F202AFBD055
:100980000135EDB2032D51D91FFA88F2022A4DD854
:1009900009F2262292B2B2F5E16F47D80AF2262276
:1009A00092B2B2F5E16F41D89DF800B0BBF1060FED
:1009B0003CD81846009363F0A3FF042836D8019B67
:1009C000002B33D0294A009B294D3FB202F54061EC
:1009D00078010E5001EB47114C6002EB47110A46BB
:1009E00081F8F88BA1F8089CA1F80AAC81F80CBC3E
:1009F00002F60C42591E033311F8010F2C5C04F06F
:100A00000304022C08BF203802F8010F087808B14F
:100A10009942F1D103B0BDE8F08F1649164807237B
:100A2000002203B0BDE8F04FFDF74ABC134803B005
:100A3000BDE8F04FFDF744BC012301934FE70546A5
:100A4000804611E701904CE70D4B9BE7009089E74A
:100A5000824671E7814659E71E461C4601230193F1
:100A60003DE700BFBC1D080858B0002060A400206E
:100A7000D113080810210808D81D0808BC1C080854
:100A8000207908082DE9F04FDFF8AC9087B0924646
:100A900080460C4615460026BAF1000F35D06B7A19
:100AA000617AB5F90AC0B5F90CE095F808B0994239
:100AB000D5E900202BD00027CDE90020CDE9023C6C
:100AC000CDE904EB33464A4639464046FFF778F80D
:100AD000237A0593B4F90C300493B4F90A300393E4
:100AE000637A0293626854F8103B3946CDE90032CC
:100AF000404633464A460136FEF7E0FC112E05F12A
:100B00001005C9D107B0BDE8F08F5746E0E721686E
:100B10009142D0D161688142CDD1B4F90A106145CA
:100B2000C9D1B4F90C107145C5D1277AA7EB0B07D1
:100B3000B7FA87F77F09BFE720210808A0B32DE99E
:100B4000F04F037883B005463BB300F1004E804C74
:100B50000EF1FF3E014603E0984229D1714513D0C2
:100B600011F8013BA3F14102192A14F8012BA2F15B
:100B7000410C98BF2033BCF1190F02F12000EBD9D2
:100B80009A4215D1002BE9D172484FF488720021A6
:100B900003B0BDE8F04F61F0FBBD6E4900220120BB
:100BA00003B0BDE8F04F6DE76A490022012069E714
:100BB0002846F5F713FCC3B2102B064600F2AC80B2
:100BC0002021284663F05CFD0446002800F0B18037
:100BD0000378202B03D114F8013F202BFBD02046B3
:100BE000F5F7FCFB012507462046202163F048FD70
:100BF0000446002800F09B800378202B03D114F8D2
:100C0000013F202BFBD02046F5F7E8FB013580465D
:100C1000EDB22046202163F033FD0446002800F0A9
:100C200084800378202B03D114F8013F202BFBD0C4
:100C30002046F5F7D3FB0128814667D80135EDB290
:100C40002046202163F01CFD0446002874D0037860
:100C5000202B03D114F8013F202BFBD02046F5F7C1
:100C6000BDFB00F5B473B3F5347F82464ED8013531
:100C7000EDB22046202163F003FD834600285DD0BD
:100C80000378202B03D11BF8013F202BFBD05846C3
:100C9000F5F7A4FB00F5B473B3F5347F044635D8FB
:100CA0000135EDB25846202163F0EAFC8346002866
:100CB00046D00378202B03D11BF8013F202BFBD01B
:100CC0005846F5F78BFB031E18BF01230135584624
:100CD00020210193EDB263F0D3FC08B10135EDB2F0
:100CE000062D13D11C4B019A76B203EB0613C3F801
:100CF000F87CC3F8FC8C83F8019DA3F802ADA3F83F
:100D0000044D83F8002D03B0BDE8F08F134803B005
:100D1000BDE8F04FFDF7D4BA114912481023002264
:100D200003B0BDE8F04FFDF7CBBA814688E78046B7
:100D30006FE70546074657E782469AE70446B1E75C
:100D4000202163F09DFC0028E0D0CDF804B0C5E779
:100D5000BC1D080858B1002060A40020BC1C080875
:100D600040210808D81D08082DE9F04F8FB00C4627
:100D7000099207901546002630E02868BDF8281033
:100D80000C9080B2AB88ADF834308142B5F90230B6
:100D900095F801C095F804E02A7834D00021CDE917
:100DA000023ECDE9002C07981E4ACDF8108033464C
:100DB0000891FEF705FF08991A4A0798CDF80090A8
:100DC0003346CDE903B8CDE901A70136FEF776FB3E
:100DD000202E04F1060405F106051FD0B4F90270B7
:100DE000A388206894F801A094F804B094F90580D1
:100DF00094F800900A90ADF82C307FB1099B002B3D
:100E0000BBD10999D8E79F42C8D1BDF82C10BDF8D5
:100E10003400091AB1FA81F14909C0E70FB0BDE801
:100E2000F08F00BF54210808F0B589B0064663F082
:100E300067FD10F0FF020DD1474991F8CE3B4FF40A
:100E4000C87000FB031101F67C11012009B0BDE858
:100E5000F04089E7414C751D314603E09E452AD19B
:100E6000A94213D011F8013BA3F14102192A14F849
:100E7000012BA2F1410C98BF2033BCF1190F02F1F4
:100E8000200EEBD99A4216D1002BE9D1324A344BCD
:100E900092F8CE1B4FF4C87000FB012218689988A5
:100EA00002F67C1302F63C221860998006339342C6
:100EB000FAD109B0F0BD2B4901AA30465FF0DCFF42
:100EC0004FF0FF33079380B1264E02AD0024F5F7B3
:100ED00085FA034645F8043B002001AA3146013457
:100EE0005FF0CAFF30B1062CF1D11F48FDF7E8F9D9
:100EF00009B0F0BD042CF8DD029B1F2BF5D8039A36
:100F00000F2AF2D8049C262CEFD8059F07F57A719A
:100F1000B1F5FA6FE9D8069EFF2EE6D8079D691C49
:100F20004029E2D80C4991F8CE0B4FF4C87E0EFB55
:100F300000F04FF0060E0EFB03030B440B4883F842
:100F40007C2983F87D49A3F87E7983F8806983F84A
:100F50008159FFF769FFACE760A40020BC1D0808B9
:100F6000E47F0708EC710808BC1C08082079080811
:100F70002DE9F04F9FB098460F908B4692464FF068
:100F8000000910920AE0C8450BD009F10109B9F136
:100F9000400F0BF1140B0AF1140A7AD0B8F1FF3F9D
:100FA000F1D15D460FCD14AC0FC42B6823609BF8C4
:100FB00013300B939BF810300C939BF911300D9369
:100FC0009BF81230DBF808200E93109B0A929BF8D6
:100FD0000C209BF8047008900992002B46D0DAF898
:100FE00000301193DAF80830129356469AF813300D
:100FF00013930FCE19AD0FC5189C33689AF804C02F
:101000009AF80CE02B605C4034F07F442CD16745AB
:101010002ED00B9B07930A9B0693099B0593089B75
:101020001D4A0F98CDE903730E9B02930D9B01930C
:101030000C9B009321464B46FEF7C2FD0B9B07938A
:101040000A9B0693099B0593089B134A0F98CDE9C9
:1010500003730E9B02930D9B01930C9B00932146FF
:101060004B46FEF72BFA90E70024D2E7109CE5E709
:10107000089B8342CDD1099B7345CAD10A9B129A22
:101080009342C6D10B9B139A9C1AB4FA84F4640958
:10109000BFE71FB0BDE8F08F6C2108082DE9F041D3
:1010A0008AB005460C4663F02BFC10F0FF0011D10E
:1010B000524991F83E2022B1631C3BD10AB0BDE8F1
:1010C000F0814FF0FF3301F6086101200AB0BDE85E
:1010D000F0414DE74A4C681D294603E09E452CD15E
:1010E000884213D011F8013BA3F14102192A14F8E8
:1010F000012BA2F1410C98BF2033BCF1190F02F172
:10110000200EEBD99A4218D1002BE9D13D483E4A36
:10111000904203D3D2E714309042CFD20388C3F376
:101120000B03B3F57E7FF6D138490AB0BDE8F04134
:10113000F5F710BE23460246C5E735496A462846FC
:101140005FF09AFE78B1324E6D460024F5F746F90D
:101150006A4645F8040F3146002001345FF08CFEEA
:1011600038B1092CF2D12B48FDF7AAF80AB0BDE836
:10117000F081092CF7D101993F29F4D8029B012B6A
:10118000F1D80398421C402AEDD8049F342FEAD8A6
:10119000DDF814E0BEF1070FE5D8DDF818C01E4CED
:1011A0000CF5742202F51072A242DCD8079E072EBD
:1011B000D9D8089D05F5742202F51072A242D2D842
:1011C000099CFF2CCFD80D4A4FF0140808FB0122D0
:1011D00009B282F8190E114882F8183E82F81A7E78
:1011E00082F80CEEC2F808CE82F8146EC2F8105ED7
:1011F00082F81B4EFFF752FF60E700BF60A400209B
:10120000BC1D08081C870808088C080868B2002064
:10121000EC710808BC1C080880841E0020790808AE
:101220004FF0FF313AE700BF2DE9F04FA5B08B46F4
:10123000119092464FF000091292DBF808300C939F
:101240009BF80C300B93BBF810300D93BBF81230A9
:101250000E93BBF814300F935D46BBF81630109315
:101260000FCD16AC0FC495E80700129BDBF8007099
:101270009BF804809BF8186084E80700002B4DD091
:10128000DAF800301393DAF80830159355469AF8D7
:101290000C3014930FCD1DAC0FC495E807009AF8DD
:1012A00018E09AF804C0B64584E8070038D0002456
:1012B000109B08930F9B07930E9B06930D9B059322
:1012C0000C9B04930B9B214A1198CDE90273CDE945
:1012D00000684B462146FEF773FC109B08930F9B5A
:1012E00007930E9B06930D9B05930C9B04930B9BFE
:1012F000164A1198CDE90273CDE900684B462146A4
:1013000009F10109FEF7DAF8B9F1040F0BF11C0B32
:101310000AF11C0A91D125B0BDE8F08F129CDCE7E0
:10132000E045C4D1139B9F42C1D10B9B149A9342B9
:10133000BDD10C9B159A9342B9D11A9A8242B6D16B
:101340001B9C641AB4FA84F46409B1E7902108087C
:101350002DE9F0478CB0064663F0D2FA10F0FF0298
:1013600005D1544901200CB0BDE8F0475CE7524C70
:10137000751D314603E09E4529D18D4213D011F8E9
:10138000013BA3F14102192A14F8012BA2F1410CEF
:1013900098BF2033BCF1190F02F1200EEBD99A420D
:1013A00015D1002BE9D14548454A904203D328E0A6
:1013B0001430904225D20388C3F30B03B3F57E7F2C
:1013C000F6D13C490CB0BDE8F047F5F7C3BC3D4948
:1013D00001AA30465FF050FD80B13A4E02AD0024C4
:1013E000F4F7FCFF034645F8043B002001AA314610
:1013F00001345FF041FD38B10A2CF1D13248FCF7DD
:101400005FFF0CB0BDE8F0870A2CF7D1029B032BDD
:10141000F4D803990129F1D8049C072CEED8059F34
:101420002A4807F5742202F510728242E6D8DDF8E8
:1014300018E0BEF1070FE1D8DDF81CC00CF57422EE
:1014400002F510728242D9D8DDF82090B9F5004F2C
:10145000D4D2DDF82480B8F5004FCFD2DDF828A033
:10146000BAF5004FCAD20B9EB6F5004FC6D21C206B
:1014700000FB03F30020164A05466AF30F0566F3E6
:101480001F4502F504761A44103382F8281282F8B8
:101490001442C2F8107282F81CE2C2F818C269F352
:1014A0000F00F21868F31F40F0500A485560FFF72C
:1014B0004FFFA6E768B70020BC1D08081C87080876
:1014C000088C0808EC710808BC1C080880841E0001
:1014D00058B50020207908082DE9F04FA1B08346C7
:1014E000884600240DF1500A164608EB44174FEACF
:1014F000441C796858F80C00BA68FB6810AD0FC539
:1015000038697969BA69FB690FC5002E5ED006EBB0
:101510000C0756F80C007968BA68FB68BDF846906D
:101520000FC538697969BA69FB699DF840700FC5C4
:101530009DF848009DF860100A90BDF84A000B9095
:101540009DF84C000C90B942BDF84E00BDF84230F9
:101550009DF844200D903BD000250D9907910C99E2
:1015600006910B9905910A990292CDE90391CDE973
:1015700000732D4ACDF820A0234629465846FEF791
:101580001FFB9DF84C30BDF84E10BDF84A20069365
:101590009DF84830CDE9071ACDE90432BDF8461070
:1015A0009DF84430BDF84220CDE902319DF840302D
:1015B0002946CDE90032584623461B4A0134FDF73F
:1015C0007DFF032C91D121B0BDE8F08F3546D8E7DF
:1015D000BDF862109942BFD19DF864109142BBD111
:1015E000BDF866104945B7D19DF868100A98814248
:1015F000B2D1BDF86A100B988142ADD19DF86C1044
:101600000C988142A8D1BDF86E100D988142A3D1EB
:101610001CA95046CDE90E3260F022F8B0FA80F5F0
:10162000DDE90E326D0998E7B42108082DE9F04193
:1016300090B0044663F064F910F0FF0205D144490C
:10164000012010B0BDE8F04146E7424901AA20461A
:101650005FF012FC40496A465FF00EFC002866D03D
:101660003D4E05AD0024F4F7B9FE034645F8043FAE
:1016700000206A46314601345FF0FEFB002854D05A
:10168000092CF0D1334901AA00205FF0F5FB054693
:10169000002852D063F034F9044600284FD104F1F9
:1016A00040030DEB0304069B0022022B04F8382CA8
:1016B0003DD8079A072A3AD80899FF2937D8099CB4
:1016C000072C34D8DDF82880B8F1FF0F2FD80B9FF6
:1016D000072F2CD8DDF830E0BEF1FF0F27D8DDF85A
:1016E00034C0BCF1020F22D80E9EFF2E1FD81B481B
:1016F00000EB431302AD83F88442A3F8868203F51E
:10170000247483F88872A3F88AE283F88CC2A3F861
:101710008E6283F88022A3F8821295E80F0084E895
:101720000F000F48FFF782FF04E0092CAAD00D48F4
:10173000FCF7C6FD10B0BDE8F0810446AFE70F2806
:1017400028BF0F242246294602A85FF009FCA6E71D
:10175000D8B700202C4B0808EC71080858B50020B9
:1017600020790808BC1C08080FB470B582B006AB1D
:10177000164C53F8042B1649A06B01935AF0A8FAA3
:10178000A56B6A7A32B12B68686805F10A0198473F
:1017900000236B720F48FCF725FDA68F36B902B007
:1017A000BDE8704004B07047013EF8D0FBF772FC12
:1017B00004460D46FBF76EFC001B61EB0501B0F51E
:1017C0007A7F71F10001F5D3EEE700BF60A400203D
:1017D000E5DE0008147B08082DE9F041C37913F019
:1017E000C00225D0402A21D1047A1F48462C36D881
:1017F000FCF7F8FC1D4B03EBC40393F8B8518DB113
:10180000D3F8B4711A4EDFF87480002402E0404629
:10181000FCF7E8FC57F8241030460134FCF718FCBC
:10182000A542F4D1BDE8F041FDF7CEBDBDE8F081A1
:101830000E4C427A03F0070304EB8202062BD269B6
:1018400008D0037A0B4804EB8304B4F91C10BDE8FC
:10185000F04189E7BDE8F0410748114684E7FCF70D
:10186000C1FC00231B79FFDE102208084C76070814
:1018700030560808F8210808E8210808202208083E
:101880002DE9F04F0378202B8FB0054603D115F8D2
:10189000013F202BFBD000242B464C4EDFF8488123
:1018A000DFF848B1DFF848A125461C4602E00C36B7
:1018B00046452FD002A9304619F03AFA214602A82F
:1018C00062F028FE0028F2D0414802A9FCF7C0FBD4
:1018D000029B5B45304622D019F042FBDFF80491B1
:1018E000014600223046FCF715FD5046FCF77AFC15
:1018F000B9F83C7067BB3046FFF76EFF5046FCF707
:1019000071FCB9F83C30002B37D10C36464505F157
:101910000105CFD1002D45D00FB0BDE8F08F9DF867
:101920000C30002BD8D119F01BFB2A4A2A4BDFF8C8
:10193000B49001460078202814BF10461846FCF7E2
:1019400087FB5046FCF74EFCB9F83C70002FD2D014
:10195000CDE90065FBF79EFB05460E46FBF79AFBBB
:10196000401B61EB0601B0F57A7F71F10001F5D300
:10197000013FEFD1DDE90065BDE799460096FBF731
:1019800089FB06460F46FBF785FB801B61EB0701D1
:10199000B0F57A7F71F10001F5D3B9F10109EED10B
:1019A000009EB2E70D48FCF71DFC0D48FCF71AFC41
:1019B000FDF70AFD0B4B93F83E20002AACD0012224
:1019C00083F83F200FB0BDE8F08F00BF3C8A0708C6
:1019D000FC1D0808F02B0808101E0808881C0808C1
:1019E0002422080860A4002074A607086E616D65B3
:1019F000147B08082DE9F04F0478202C8FB00546A1
:101A000003D115F8014F202CFBD0284662F078FF57
:101A10008246002800F09E80012800F098803D2139
:101A2000284662F02DFE0446002800F02D8110F8B3
:101A3000013C202B40F0AD81431E1A4613F8011DD6
:101A40002029FAD06378202BA2EB050204F10104CF
:101A500003D114F8013F202BFBD0DFF858A3D3B2F9
:101A60000193564600270DF1080840F25A2B05E075
:101A700001375F4506F10C0600F0638141463046B0
:101A800019F056F9404662F03BFF41468146024656
:101A90002846F4F787F90028EAD1019B9945E7D158
:101AA0007B00019307EB47030AEB830B9BF807903E
:101AB00009F00705062D00F0A58019F0C00900F017
:101AC0008180B9F1400F40F08A809BF80820462AB7
:101AD00000F2C881B54B03EBC20393F8B891B9F19A
:101AE000000F7CD0D3F8B4310746A3F1040E6FF099
:101AF000004A5EF8041F204601EB0A0C05E0203284
:101B00009A4240F0CA808C4512D011F8013BA3F1F3
:101B10004102192A10F8012BA2F1410B98BF203382
:101B2000BBF1190FEBD99A4240F0B780002BEAD1F4
:101B3000304619F015FA0346052D00F2D080DFE893
:101B400015F08D018D018F018F01CD0083012A2CAD
:101B50007FF465AF9648974FDFF884B2DFF86C9258
:101B6000FCF740FB0DF10808FDF72EFC02E00C37F6
:101B7000BB4544D04146384619F0DAF841468E4814
:101B8000FCF766FA384619F0EBF95246014638463A
:101B9000FCF7C0FB8948FCF725FBB9F83C60002E38
:101BA000E5D0FBF777FA04460D46FBF773FA001B06
:101BB00061EB0501B0F57A7F71F10001F5D3013ECB
:101BC000EFD1D4E7227852B17D49204662F0C0FDC2
:101BD0000746204662F094FE874200F00381794870
:101BE000FCF700FB7848FCF7FDFA784B93F83E20B1
:101BF000002A4ED13046FFF7EFFDFDF7E5FB0FB0B1
:101C0000BDE8F08F204662F07BFEA346054680B11A
:101C10001BF8012BA2F16101192906D8203A0BF813
:101C2000012C204662F06CFE0546ABEB04029542A7
:101C3000EED8674940465FF013FD00285CD0654947
